:10000000FDC6000025C7000023C7000021C700006F
:100010001FC700001DC700001BC7000019C7000054
:1000200017C7000015C700000C94DE590C942C6B08
:100030000FC700000DC700000BC7000009C7000074
:1000400007C7000005C7000003C7000001C7000084
:10005000FFC60000FDC60000FBC60000F9C6000098
:10006000F7C60000F5C60000F3C60000F1C60000A8
:10007000EFC60000EDC60000EBC60000E9C60000B8
:10008000E7C60000E5C60000E3C60000E1C60000C8
:10009000DFC60000DDC600000555075509550B55A4
:1000A0000D550F551155145517551A551C551F55FB
:1000B0002255245527552A552C553F55445546550C
:1000C00048554A554D555155545557555A555D55F6
:1000D0006055635566556955224F6E20626F617297
:1000E00064206461746120666C617368220022552B
:1000F00053422052656D6F7465206D656D6F727926
:1001000022006364006D6F756E74006370006C7321
:10011000006C737C6D6F726500726D0064660073B5
:1001200070616365006D6B64697200746F756368FC
:1001300000617070656E6400636174006361747C5B
:100140006D6F72650063642E2E006469736B006DC1
:1001500061726B00676F746F006D760068656C701C
:1001600000666F726D61740073796E630070657202
:1001700066007265626F6F74006C737573620073F2
:10018000757370656E6400726573756D6500656E7C
:10019000756D6572617465006466755F6572617323
:1001A00065006466755F70726F67006466755F7383
:1001B00074617274006869645F646675006869647C
:1001C0005F676574005061737465204661696C0DEA
:1001D0000A00243E000C2D2D2D2D2D2D2D2D2D2DE5
:1001E0002D2D2D2D2D2D2D2D2D2D2D2D2D2D2D2D3F
:1001F0000D0A2020202041544D454C2041565220CC
:10020000755368656C6C0D0A2D2D2D2D2D2D2D2D02
:100210002D2D2D2D2D2D2D2D2D2D2D2D2D2D2D2D0E
:100220002D2D0D0A000C2D2D2D2D2D2D2D2D2D2D8F
:100230002D2D2D2D2D2D2D2D2D2D2D2D2D2D0D0A31
:10024000755368656C6C206E6F7420617661696CA3
:1002500061626C650D0A2D2D2D2D2D2D2D2D2D2D31
:100260002D2D2D2D2D2D2D2D2D2D2D2D2D2D0D0A01
:1002700000556E61626C6520746F206D6F756E74D1
:100280002064726976650D0A00447269766520649F
:100290006F6573206E6F742065786973740D0A0042
:1002A00043616E206E6F742065726173652C2069E6
:1002B0006620746865206E616D6520697320612019
:1002C0006469726563746F72792C20636865636B0F
:1002D00020697420697320656D7074790D0A00556A
:1002E0006E6B6E6F776E2066696C650D0A00436FEA
:1002F0006D6D616E64206E6F7420666F756E640D37
:100300000A00466F726D6174206661696C730D0A34
:10031000000D0A53696D706C6520746578742065F2
:100320006469746F722C20656E74657220636861F5
:100330007220746F20617070656E642C205E712075
:10034000746F206578697420616E642073617665CE
:100350000D0A000D0A2D2D2D2D20557368656C6C2E
:1003600020436F6D6D616E64733A0D0A2048454CF1
:10037000502020202020202020202020202020204D
:1003800020202050726F76696465732048656C7018
:1003900020696E666F726D6174696F6E20666F7230
:1003A00020557368656C6C20636F6D6D616E64734E
:1003B0002E0D0A2021202020202020202020202057
:1003C0002020202020202020202050726576696F78
:1003D000757320636F6D6D616E6420286869737436
:1003E0006F7279292E0D0A20242020202020202021
:1003F00020202020202020202020202020204E658A
:10040000787420636F6D6D616E6420286869737401
:100410006F7279292E0D0A0D0A2D2D2D2D2046697A
:100420006C652053797374656D7320436F6D6D61D6
:100430006E64733A0D0A204449534B20202020203B
:1004400020202020202020202020202020446973EC
:10045000706C61797320746865206E756D62657269
:10046000206F66206472697665732E0D0A204446FB
:10047000202020202020202020202020202020207C
:1004800020202020446973706C6179732066726546
:1004900065207370616365206F6620616C6C2063FA
:1004A0006F6E6E6563746564206472697665732E21
:1004B0000D0A20464F524D4154205B2F413A5D209A
:1004C000202020202020202020466F726D61747330
:1004D0002064726976652C202F41206472697665EC
:1004E000206C65747465722028612C20622C206554
:1004F00074632E292E0D0A204D4F554E54205B2F2C
:10050000413A5D20202020202020202020204D6FF7
:10051000756E74732064726976652C202F41206497
:1005200072697665206C65747465722028612C2070
:10053000622C206574632E292E0D0A205B2F413A10
:100540005D2020202020202020202020202020206E
:1005500020204D6F756E74732064726976652C204F
:100560002F41206472697665206C65747465722011
:1005700028612C20622C206574632E292E0D0A2000
:10058000535041434520202020202020202020209F
:10059000202020202020446973706C6179732064CE
:1005A000726976652063617061636974792E0D0AE2
:1005B000204C53205B7C4D4F52455D202020202055
:1005C00020202020202020446973706C61797320E2
:1005D00061206C697374206F662066696C65732096
:1005E000616E64207375626469726563746F7269A9
:1005F000657320696E2061206469726563746F722F
:10060000792E0D0A204344205B2E2E5D5B706174B1
:10061000685D2020202020202020204368616E6714
:100620006573207468652063757272656E742064EA
:1006300069726563746F72792E0D0A2043415420EC
:100640005B66696C65206E616D655D2020202020F1
:100650002020446973706C6179732066696C652031
:10066000636F6E74656E74732E0D0A204D4B444992
:1006700052205B646972206E616D655D20202020D0
:10068000202043726561746573206120646972651E
:1006900063746F72792E0D0A20544F554348205BC6
:1006A00066696C65206E616D655D202020202043A9
:1006B00072656174657320612066696C652E0D0A30
:1006C00020524D205B2A5D5B66696C65206E616D12
:1006D000655D202020202044656C65746573206F63
:1006E0006E65206F72206D6F72652066696C657330
:1006F000206F72206469726563746F726965732E0E
:100700000D0A20415050454E44205B66696C6520BF
:100710006E616D655D20202020417070656E647390
:100720002066696C652066726F6D207465726D69F4
:100730006E616C20696E7075740D0A204D41524BCC
:1007400020202020202020202020202020202020A9
:1007500020205265636F726420746865206375722F
:1007600072656E74206469726563746F7279206952
:100770006E20626F6F6B6D61726B0D0A20474F5474
:100780004F2020202020202020202020202020203A
:10079000202020476F20746F20626F6F6B6D617235
:1007A0006B6564206469726563746F72790D0A20E9
:1007B0004350205B66696C65206E616D655D5B70A2
:1007C0006174685C5D20436F7079732066696C6545
:1007D00020746F20626F6F6B6D61726B6564206453
:1007E00069726563746F7279206F7220746F207004
:1007F00061746820617267756D656E742E0D0A20D4
:100800004D56205B706174685D205B6E6577206E6D
:10081000616D655D202052656E616D65732066694E
:100820006C652066726F6D207061746820776974E2
:1008300068206E6577206E616D652E0D0A20535914
:100840004E43205B7372635F706174685D205B640C
:100850006573745F706174685D202053796E63689E
:10086000726F6E697A6573206120666F6C64657261
:1008700020636F6E74656E742077697468206F747E
:1008800068657220666F6C6465722E0D0A20504593
:100890005246205B2F413A5D205B2F413A5D20207C
:1008A00020202020506572666F6D7320746865206B
:1008B0007472616E73666572207261746520626520
:1008C000747765656E2074776F20646576696365FB
:1008D000732E0D0A205245424F4F542020202020D5
:1008E00020202020202020202020205265736574A5
:1008F00020746865206170706C69636174696F6EE3
:100900002E0D0A0D0A2D2D2D2D2055534220486FF6
:10091000737420436F6D6D616E64733A0D0A204CE1
:10092000535553422020202020202020202020200A
:100930002020202020446973706C61797320555306
:100940004220696E666F726D6174696F6E2E0D0A5A
:100950002053555350454E44202020202020202055
:100960002020202020202053757370656E64732032
:100970005553422062757320616374697669747996
:100980002E0D0A20524553554D4520202020202071
:1009900020202020202020202020526573756D65A6
:1009A00073205553422062757320616374697669C0
:1009B00074792E0D0A20454E554D4552415445201F
:1009C000202020202020202020202020466F72631D
:1009D00065732061207265736574206F6E205553B6
:1009E00042206C696E6520616E642072657374616B
:1009F00072742074686520656E756D6172617469CA
:100A00006F6E2E0D0A0D0A2D2D2D2D2055534220CF
:100A1000486F73742044465520436F6D6D616E645A
:100A2000733A0D0A204446555F45524153452020F4
:100A30002020202020202020202020457261736566
:100A4000207461726765742E0D0A204446555F500C
:100A5000524F47205B706174685D20202020202069
:100A60002050726F6772616D2074617267657420C7
:100A7000776974682061204845582066696C652E46
:100A80000D0A204446555F535441525420202020E3
:100A90002020202020202020205374617274207494
:100AA00061726765742E0D0A0D0A2D2D2D2D2055AE
:100AB000534220486F7374204849442047656E654F
:100AC00072696320436F6D6D616E64733A0D0A2025
:100AD0004849445F474554202020202020202020E2
:100AE00020202020202044697370616C7973206974
:100AF0006E666F726D6174696F6E2061626F75747E
:100B0000207468652074617267657420636F6E6E0F
:100B10006563746564206174204849442E0D0A2081
:100B20004849445F44465520202020202020202092
:100B3000202020202020456E7465727320696E206D
:100B4000444655206D6F6465207468652074617239
:100B500067657420636F6E6E65637465642061748D
:100B6000204849442E0D0A004E6F7420637572723E
:100B7000656E746C79206170706C696361626C651C
:100B800020746F20737570706F7274656420636F6A
:100B90006E6E656374656420646576696365287349
:100BA0002920696620616E790D0A006F6B0D0A00BD
:100BB0004641494C0D0A00446576696365207375AA
:100BC00070706F7274732072656D6F7465207761D9
:100BD0006B652D75700D0A00446576696365206448
:100BE0006F6573206E6F7420737570706F727420F0
:100BF00072656D6F74652077616B652D75700D0A78
:100C0000004465766963652069732073656C662DA1
:100C1000706F77657265640D0A0044657669636577
:100C2000206973206275732D706F77657265640D2E
:100C30000A005553422069732073757370656E64A2
:100C40006564210D0A004465766963652069732037
:100C500066756C6C2D73706565640D0A004465766D
:100C6000696365206973206C6F772D7370656564A7
:100C70000D0A0041544D454C202020415439305537
:100C80005342313238204D20532020302E30300056
:100C90008003021F0000001201000200000040EB70
:100CA000032320001001020301090259000301007F
:100CB0008032090400000103000200092111010033
:100CC0000122340007058103080025090401000200
:100CD0000806500007058202400000070503024095
:100CE00000000904020002030000000921110100B4
:100CF00001223500070584030800140705050308D1
:100D000000140C03410054004D0045004C003A0310
:100D100041005600520020005500530042002000C0
:100D20004B0045005900200043004F004D0050008B
:100D30004F00530049005400450020004400450086
:100D400056004900430045001C03300030003000CD
:100D50003000300030003000300030003000300013
:100D6000300030000403090405010902A101090152
:100D7000A100050919012903150025017501950335
:100D80008102750595018101050109300931093894
:100D90001581257F750895038106C0C006FFFF09F0
:100DA00001A10109020903150026FF007508950835
:100DB000810209040905150026FF007508950891B0
:100DC0000209060907150026FF0075089504B102FF
:100DD000C04649524D574152452E48455800423A67
:100DE0002F4F55542F00423A2F494E2F00413A2F92
:100DF0004F55542F00413A2F494E2F0011241FBE4A
:100E0000CFEFD0E2DEBFCDBF80E090E020E80FB6AC
:100E1000F89420936100809361000FBE81E017E099
:100E2000A0E0B1E0E6EBF5E001E00BBF02C0079007
:100E30000D92A83AB107D9F719E1A8EAB7E001C0C5
:100E40001D92A739B107E1F70E94007E0C94D98268
:100E5000D7C88FB7F89497EF94BF98E10FB6F8947E
:100E600090936000109260000FBE87FF01C07894DD
:100E70000895982F3FB7F89487EF84BF93FD02C081
:100E800028E001C028E29770292B88E190E00FB696
:100E9000F894A895809360000FBE2093600037FF00
:100EA00001C0789408950E94FA5B0E948E730E949C
:100EB000BF540E94B07D0E949E7C0E94A7760E9433
:100EC00077780E94227B0E949A7BEDCF0E94D65BAE
:100ED0000E949C730E947D550E94EF7D0E949A7C27
:100EE0000E9497770E94BB770E947E780C94957B36
:100EF000EDDFD9CF8091C8008078089580E190E03F
:100F00009093CD008093CC00E8ECF0E0808182608B
:100F1000808386E08093CA00E9ECF0E080818861FC
:100F2000808381E00895282F8091C80085FFFCCF41
:100F30002093CE00822F08958091C80087FFFCCFB8
:100F40008091CE000895CF93DF93AAE7B0E08C9113
:100F500080688C93ECE7F0E080818F7D80832BE7C5
:100F600030E0E90188818F77888380818F77808363
:100F70008081806480838C91877F8C938C91887F23
:100F80008C938C9185608C93DF91CF910895DC01D7
:100F9000FB018D9181934150E1F70895CF93DF9349
:100FA000EC0120E030E00FC0FE01E20FF31FDB0197
:100FB000A20FB31F90818C91981719F02FEF3FEF7C
:100FC00007C02F5F3F4F2417350770F320E030E054
:100FD000C901DF91CF910895809197199091981947
:100FE000A0919919B0919A1985559A4AAA4AB5457E
:100FF00069F41092971910929819109299191092F9
:101000009A19E0910001F09101010995089585E593
:101010009AEAAAEAB5E58093971990939819A09354
:101020009919B0939A1985E024DFFFCF20918400AD
:1010300030E040918500942F80E0282B392BC901A6
:1010400008959091EB0091609093EB008093EC00F9
:101050008091ED008270862B8093ED008091ED00F1
:1010600082608093ED008091EE00881F8827881FA2
:1010700008958091D8008F7B8093D8008091D9000B
:1010800081FF0BC01092E9008091EB0080FD05C04C
:101090001092E90082E060E3D4CF80E00895E9EAAD
:1010A000F0E09081916090838093AA00EBEAF0E0F9
:1010B00060838081826080838091AC008078089515
:1010C0008930910510F480E008958131910510F484
:1010D00081E008958132910510F482E00895813411
:1010E000910510F483E008958138910510F484E0AF
:1010F000089521E08130920710F485E00895815031
:10110000924010F087E0089586E0089520E030E0F6
:1011100041E050E0CA01022E02C0880F991F0A94D4
:10112000E2F78093A8001092A8002093A700809176
:10113000AB008D7F8093AB008091A9008E7F809360
:10114000A9002F5F3F4F2730310521F70895809187
:10115000F80020E030E0682F70E0422FCB01022E33
:1011600002C0959587950A94E2F780FD06C02F5F2F
:101170003F4F2730310589F748E0842F089580914B
:101180007C00807F80937C0080917C0081608093D4
:101190007C0080917A00806480937A0080917A004C
:1011A00084FFFCCF9091780080917900382F20E067
:1011B000290F311DC90108958091A80708950F9343
:1011C0001F938A011BD3C8018BD559D380E090E0CF
:1011D0001F910F9108950F931F938A01BBD0C801EF
:1011E00058D50DD180E090E01F910F9108950F9395
:1011F0001F938A01AFD0C80104D1182F00D120E07D
:1012000030E0112311F421E030E0C9011F910F916A
:1012100008959091A8078091A907981729F09093B5
:10122000A90723E030E008C05ED0813019F022E049
:1012300030E002C020E030E0C9010895FC018FEFEA
:101240009FE1A0E0B0E080839183A283B383E1CFEC
:1012500020C008950F931F93CF93DF938B019C01C0
:10126000EA018091A807882341F4C901B801C6D2D8
:10127000CE0136D3882321F40CD021E030E003C026
:10128000FED220E030E0C901DF91CF911F910F9194
:101290000895239884B1876184B985B18F6185B938
:1012A0008CB580618CBD8CB5837F8CBD8CB58C601A
:1012B0008CBD84B1866084B98CB58C7F8CBD8CB5B7
:1012C0008CBD8DB581608DBD8CB580648CBD109258
:1012D000AE071092AF0708952C9A8091AF0788232C
:1012E00009F42C9808950F931F931092AF0707ED00
:1012F00011E013C0F1DF0EBD0DB407FEFDCF1EBC23
:101300000DB407FEFDCF8EB58C73843319F02C9A83
:1013100080E008C02C9A1093AF078091AF07882314
:1013200049F381E01F910F910895D6DF87ED8EBDBF
:101330000DB407FEFDCF1EBC0DB407FEFDCF04C0EB
:101340001EBC0DB407FEFDCF0EB407FEF9CF2C9ADC
:101350008EB5089549E0660F771F881F991F4A953B
:10136000D1F76093AA077093AB078093AC07909373
:10137000AD071092AF078091AE0780FF04C08E7F4B
:101380008093AE07D2DFA8DF82ED8EBD0DB407FEDD
:10139000FDCF2091AB078091AC07880F922F991F4A
:1013A0009927991F892B8EBD0DB407FEFDCF822F83
:1013B00090E08E7F880F991F2170282B2EBD0DB4D1
:1013C00007FEFDCF8091AA078EBD0DB407FEFDCFAD
:1013D0008FEF8EBD0DB407FEFDCF8FEF8EBD0DB428
:1013E00007FEFDCF8FEF8EBD0DB407FEFDCF8FEF53
:1013F0008EBD0DB407FEFDCF8EB581E008952C9A09
:101400000895CF93DF93EC0198E0F8941EBC0DB4DF
:1014100007FEFDCF8EB58093F1001EBC0DB407FE14
:10142000FDCF8EB58093F1001EBC0DB407FEFDCF3D
:101430008EB58093F1001EBC0DB407FEFDCF8EB5B6
:101440008093F1001EBC0DB407FEFDCF8EB58093D6
:10145000F1001EBC0DB407FEFDCF8EB58093F100E8
:101460001EBC0DB407FEFDCF8EB58093F1001EBCEF
:101470000DB407FEFDCF8EB58093F1001EBC0DB4F8
:1014800007FEFDCF8EB58093F1001EBC0DB407FEA4
:10149000FDCF8EB58093F1001EBC0DB407FEFDCFCD
:1014A0008EB58093F1001EBC0DB407FEFDCF8EB546
:1014B0008093F1001EBC0DB407FEFDCF8EB5809366
:1014C000F1001EBC0DB407FEFDCF8EB58093F10078
:1014D0001EBC0DB407FEFDCF8EB58093F1001EBC7F
:1014E0000DB407FEFDCF8EB58093F1001EBC0DB488
:1014F00007FEFDCF8EB58093F1001EBC0DB407FE34
:10150000FDCF8EB58093F1001EBC0DB407FEFDCF5C
:101510008EB58093F1001EBC0DB407FEFDCF8EB5D5
:101520008093F1001EBC0DB407FEFDCF8EB58093F5
:10153000F1001EBC0DB407FEFDCF8EB58093F10007
:101540001EBC0DB407FEFDCF8EB58093F1001EBC0E
:101550000DB407FEFDCF8EB58093F1001EBC0DB417
:1015600007FEFDCF8EB58093F1001EBC0DB407FEC3
:10157000FDCF8EB58093F1001EBC0DB407FEFDCFEC
:101580008EB58093F1001EBC0DB407FEFDCF8EB565
:101590008093F1001EBC0DB407FEFDCF8EB5809385
:1015A000F1001EBC0DB407FEFDCF8EB58093F10097
:1015B0001EBC0DB407FEFDCF8EB58093F1001EBC9E
:1015C0000DB407FEFDCF8EB58093F1001EBC0DB4A7
:1015D00007FEFDCF8EB58093F1001EBC0DB407FE53
:1015E000FDCF8EB58093F1001EBC0DB407FEFDCF7C
:1015F0008EB58093F1001EBC0DB407FEFDCF8EB5F5
:101600008093F1001EBC0DB407FEFDCF8EB5809314
:10161000F1001EBC0DB407FEFDCF8EB58093F10026
:101620001EBC0DB407FEFDCF8EB58093F1001EBC2D
:101630000DB407FEFDCF8EB58093F1001EBC0DB436
:1016400007FEFDCF8EB58093F1001EBC0DB407FEE2
:10165000FDCF8EB58093F1001EBC0DB407FEFDCF0B
:101660008EB58093F1001EBC0DB407FEFDCF8EB584
:101670008093F1001EBC0DB407FEFDCF8EB58093A4
:10168000F1001EBC0DB407FEFDCF8EB58093F100B6
:101690001EBC0DB407FEFDCF8EB58093F1001EBCBD
:1016A0000DB407FEFDCF8EB58093F1001EBC0DB4C6
:1016B00007FEFDCF8EB58093F1001EBC0DB407FE72
:1016C000FDCF8EB58093F1001EBC0DB407FEFDCF9B
:1016D0008EB58093F1001EBC0DB407FEFDCF8EB514
:1016E0008093F1001EBC0DB407FEFDCF8EB5809334
:1016F000F1001EBC0DB407FEFDCF8EB58093F10046
:101700001EBC0DB407FEFDCF8EB58093F1001EBC4C
:101710000DB407FEFDCF8EB58093F1001EBC0DB455
:1017200007FEFDCF8EB58093F1001EBC0DB407FE01
:10173000FDCF8EB58093F1001EBC0DB407FEFDCF2A
:101740008EB58093F1001EBC0DB407FEFDCF8EB5A3
:101750008093F1001EBC0DB407FEFDCF8EB58093C3
:10176000F1001EBC0DB407FEFDCF8EB58093F100D5
:101770001EBC0DB407FEFDCF8EB58093F1001EBCDC
:101780000DB407FEFDCF8EB58093F1008091E80087
:101790008F778093E800789404C08091EB0080FFFD
:1017A00029C08091E80085FFF8CF915009F02DCE37
:1017B0006091AA077091AB078091AC079091AD073B
:1017C00060507E4F8F4F9F4F6093AA077093AB0777
:1017D0008093AC079093AD0721972C9A11F481E088
:1017E0000AC059E096958795779567955A95D1F7F0
:1017F000B1DD0ACE80E0DF91CF910895E9E0660F78
:10180000771F881F991FEA95D1F76093AA077093F5
:10181000AB078093AC079093AD071092AF07809110
:10182000AE0780FF04C08E7F8093AE077EDD54DD5F
:1018300082E88EBD0DB407FEFDCF2091AB078091ED
:10184000AC07880F922F991F9927991F892B8EBD5E
:101850000DB407FEFDCF822F90E08E7F880F991F79
:101860002170282B2EBD0DB407FEFDCF8091AA0755
:101870008EBD0DB407FEFDCF8EB581E0089517C073
:101880001EBC0DB407FEFDCF8091AA079091AB0757
:10189000A091AC07B091AD070196A11DB11D809339
:1018A000AA079093AB07A093AC07B093AD078091C4
:1018B000AA07882329F78091AB0780FDE1CF8EB579
:1018C0002C9A81E090E00090AF0702C0880F991F2A
:1018D0000A94E2F72091AE07282B2093AE070895D3
:1018E0000F931F93CF93DF93EC0101E010E098E09A
:1018F00004C08091EB0080FFC6C18091E80085FFA5
:10190000F8CFF8948091F1008EBD0DB407FEFDCFA5
:101910008091F1008EBD0DB407FEFDCF8091F100E6
:101920008EBD0DB407FEFDCF8091F1008EBD0DB4CC
:1019300007FEFDCF8091F1008EBD0DB407FEFDCFF7
:101940008091F1008EBD0DB407FEFDCF8091F100B6
:101950008EBD0DB407FEFDCF8091F1008EBD0DB49C
:1019600007FEFDCF8091F1008EBD0DB407FEFDCFC7
:101970008091F1008EBD0DB407FEFDCF8091F10086
:101980008EBD0DB407FEFDCF8091F1008EBD0DB46C
:1019900007FEFDCF8091F1008EBD0DB407FEFDCF97
:1019A0008091F1008EBD0DB407FEFDCF8091F10056
:1019B0008EBD0DB407FEFDCF8091F1008EBD0DB43C
:1019C00007FEFDCF8091F1008EBD0DB407FEFDCF67
:1019D0008091F1008EBD0DB407FEFDCF8091F10026
:1019E0008EBD0DB407FEFDCF8091F1008EBD0DB40C
:1019F00007FEFDCF8091F1008EBD0DB407FEFDCF37
:101A00008091F1008EBD0DB407FEFDCF8091F100F5
:101A10008EBD0DB407FEFDCF8091F1008EBD0DB4DB
:101A200007FEFDCF8091F1008EBD0DB407FEFDCF06
:101A30008091F1008EBD0DB407FEFDCF8091F100C5
:101A40008EBD0DB407FEFDCF8091F1008EBD0DB4AB
:101A500007FEFDCF8091F1008EBD0DB407FEFDCFD6
:101A60008091F1008EBD0DB407FEFDCF8091F10095
:101A70008EBD0DB407FEFDCF8091F1008EBD0DB47B
:101A800007FEFDCF8091F1008EBD0DB407FEFDCFA6
:101A90008091F1008EBD0DB407FEFDCF8091F10065
:101AA0008EBD0DB407FEFDCF8091F1008EBD0DB44B
:101AB00007FEFDCF8091F1008EBD0DB407FEFDCF76
:101AC0008091F1008EBD0DB407FEFDCF8091F10035
:101AD0008EBD0DB407FEFDCF8091F1008EBD0DB41B
:101AE00007FEFDCF8091F1008EBD0DB407FEFDCF46
:101AF0008091F1008EBD0DB407FEFDCF8091F10005
:101B00008EBD0DB407FEFDCF8091F1008EBD0DB4EA
:101B100007FEFDCF8091F1008EBD0DB407FEFDCF15
:101B20008091F1008EBD0DB407FEFDCF8091F100D4
:101B30008EBD0DB407FEFDCF8091F1008EBD0DB4BA
:101B400007FEFDCF8091F1008EBD0DB407FEFDCFE5
:101B50008091F1008EBD0DB407FEFDCF8091F100A4
:101B60008EBD0DB407FEFDCF8091F1008EBD0DB48A
:101B700007FEFDCF8091F1008EBD0DB407FEFDCFB5
:101B80008091F1008EBD0DB407FEFDCF8091F10074
:101B90008EBD0DB407FEFDCF8091F1008EBD0DB45A
:101BA00007FEFDCF8091F1008EBD0DB407FEFDCF85
:101BB0008091F1008EBD0DB407FEFDCF8091F10044
:101BC0008EBD0DB407FEFDCF8091F1008EBD0DB42A
:101BD00007FEFDCF8091F1008EBD0DB407FEFDCF55
:101BE0008091F1008EBD0DB407FEFDCF8091F10014
:101BF0008EBD0DB407FEFDCF8091F1008EBD0DB4FA
:101C000007FEFDCF8EB58091E8008B7F8093E800C2
:101C10008091E8008F778093E8007894915009F0E4
:101C20006CCE4091AA075091AB076091AC077091C0
:101C3000AD0740505E4F6F4F7F4F4093AA075093C0
:101C4000AB076093AC077093AD0721972C9A98016E
:101C50000090AF0702C0220F331F0A94E2F7809171
:101C6000AE07822B8093AE07209711F481E00CC061
:101C7000F9E07695679557954795FA95D1F7CB0199
:101C8000BA01BCDD34CE80E0DF91CF911F910F917E
:101C90000895FC0120E030E01EBC0DB407FEFDCF2E
:101CA0008EB580832F5F3F4F82E02030380711F0E0
:101CB0003196F2CF8091AA079091AB07A091AC0723
:101CC000B091AD0780509E4FAF4FBF4F8093AA0792
:101CD0009093AB07A093AC07B093AD0781E0089554
:101CE000FC0120E030E080818EBD0DB407FEFDCF09
:101CF0002F5F3F4F82E02030380711F03196F3CF4D
:101D00008EB58091AA079091AB07A091AC07B091D6
:101D1000AD0780509E4FAF4FBF4F8093AA0790935F
:101D2000AB07A093AC07B093AD0781E008958FEFA8
:101D300080932A1380933A1380934A1310922913A5
:101D4000089520912913322F41E06AE470E05FEF9B
:101D50001FC0A22FB0E084E0AA0FBB1F8A95E1F755
:101D6000A65EBC4E8C918F3F89F090E0869FF0017B
:101D7000879FF00D969FF00D1124EF54F94E81814D
:101D8000882311F040E003C05C9341113150215091
:101D90002223F9F630932913089520912913222341
:101DA000E1F08091F01788508230B8F08091D9002E
:101DB00081FD13C0EDE2F3E190E030E044E0220F5A
:101DC000331F4A95E1F72E0F3F1F03C08081980F04
:101DD0007096E217F307D1F701C090E0892F0895BC
:101DE000382F409129134423E9F18091F01788504E
:101DF0008230C0F18091D90081FD34C01092B007CB
:101E000080E02AC0E82FF0E054E0EE0FFF1F5A9563
:101E1000E1F7E65DFC4E9381282F2F5F3917D0F450
:101E20008093B00720812F3FE9F030932613209351
:101E3000B51030E08AE490E0289FF001299FF00D72
:101E4000389FF00D1124EF54F94E81818093A10049
:101E500081E00895391B822F8417A0F28093B00788
:101E600080E0089580E00895BBDF882311F481E0CD
:101E700008952091261330E08091B00790E0F90199
:101E8000EE0FFF1FE20FF31F64E0880F991F6A95A2
:101E9000E1F7E80FF91FE65DFC4E8581089590910A
:101EA000AA0082E08093551981E080935619109220
:101EB0005819109257199F70906890935919109261
:101EC0005A1910925C1910925B1910925D1981EFEA
:101ED00097E10E94C460E091B007F0E0A4E0EE0F4B
:101EE000FF1FAA95E1F7E65DFC4E81818093A70074
:101EF000E6EAF0E080818D7F8083E9EAF0E080818E
:101F0000886080830895E091B007F0E0B4E0EE0FC0
:101F1000FF1FBA95E1F7E45DFC4E80816FE170E050
:101F200045E053E10E94026990E0882309F491E0C2
:101F3000892F0895E9E0F3E19091091334978FE137
:101F4000DF011D928A95E9F785E5808383E580931B
:101F5000061382E48093071383E4809308139F5F42
:101F60009093091380912613809312130895CF92B2
:101F7000DF92EF92FF920F931F93DF93CF93CDB732
:101F8000DEB763970FB6F894DEBF0FBECDBFD2DFCA
:101F900092E190930D1380E88093111386E0809373
:101FA000131383E08093141390931813ACDF8823EA
:101FB00009F446C081E190E09A838983E091B007FB
:101FC000F0E024E0EE0FFF1F2A95E1F7E65DFC4EFE
:101FD00093E0C92ED12CCC0EDD1E81817E010894A8
:101FE000E11CF11CB701A6010E94DA698823B9F44B
:101FF0000D811F858DE090E09A838983E091B00781
:10200000F0E084E0EE0FFF1F8A95E1F7E65DFC4EFD
:102010008181B701A6010E94DA69882321F080320C
:1020200079F43DDF0DC0802F8F70823039F086301B
:1020300039F4183219F423E030E007C01A3319F0EC
:1020400021E030E002C022E030E0C90163960FB623
:10205000F894DEBF0FBECDBFCF91DF911F910F91DE
:10206000FF90EF90DF90CF900895AF92BF92CF9204
:10207000DF92EF92FF921F93DF93CF93CDB7DEB73E
:102080002F970FB6F894DEBF0FBECDBF11E05DE015
:10209000A52EB12C43E0C42ED12CCC0EDD1E7E012A
:1020A0000894E11CF11CBA82A982E091B007F0E02B
:1020B00034E0EE0FFF1F3A95E1F7E65DFC4E8181BB
:1020C000B701A6010E94DA69882339F0803281F5D0
:1020D000E6DE112369F110E0E6CF8B81853571F4DE
:1020E0008C81833559F48D81823441F420E08E81D6
:1020F000833509F021E081E0282701C020E090919C
:1021000009138F81981741F48885882329F48985DC
:10211000882311F48A85811120E08F85882329F492
:10212000222319F020E030E005C021DF9C0102C02D
:1021300021E030E0C9012F960FB6F894DEBF0FBE44
:10214000CDBFCF91DF911F91FF90EF90DF90CF90A7
:10215000BF90AF900895EF92FF920F931F93DF937C
:10216000CF9300D0CDB7DEB71092B1078091241382
:1021700080932613E0912513E093B007F0E0A4E0EC
:10218000EE0FFF1FAA95E1F7E65DFC4E808180937C
:10219000B51090E02AE430E0829FF001839FF00DBB
:1021A000929FF00D1124EF54F94E81818093A1008C
:1021B000E12C72E0F72E8E010F5F1F4F24C0FA82D0
:1021C000E982E091B007F0E064E0EE0FFF1F6A954E
:1021D000E1F7E65DFC4E8181B80140E050E00E94ED
:1021E000DA69882339F0803209F459DE3EDF21E0D4
:1021F00030E011C08091271390912813019790939C
:102200002813809327138091271390912813892BEB
:10221000B1F62BDF9C01C9010F900F90CF91DF9198
:102220001F910F91FF90EF900895EF92FF920F93FF
:102230001F93DF93CF93CDB7DEB728970FB6F894EF
:10224000DEBF0FBECDBF182F4D835E836F837887AF
:102250007901C6DD882309F478C02091261330E087
:102260008091B00790E0F901EE0FFF1FE20FF31F1E
:1022700024E0880F991F2A95E1F7E80FF91FE65D22
:10228000FC4E8681823008F060C08091B1078823BF
:1022900019F061DF812FA4DD802F90E0A0E0B0E095
:1022A00019E0880F991FAA1FBB1F1A95D1F78983C0
:1022B0009A83AB83BC833EDEFE0131968981809395
:1022C0000D13818180930E13828180930F1383817C
:1022D00080931013109211138AE0809313138AE2F3
:1022E00080931413FE0135968381809316138281A7
:1022F000809317138181809318138D818093191314
:1023000000931C1300DE8823D9F41FC0E091B007AE
:10231000F0E0B4E0EE0FFF1FBA95E1F7E45DFC4E8C
:10232000808160E072E0A7010E940269803219F4A6
:10233000B6DD9BDE0AC0015080E092E0E80EF91E97
:10234000002321F792DE9C0102C021E030E0C901A8
:1023500028960FB6F894DEBF0FBECDBFCF91DF91A8
:102360001F910F91FF90EF900895AF92BF92CF927F
:10237000DF92EF92FF920F931F93DF93CF9300D0E2
:1023800000D0CDB7DEB7082F6A017B01590128DDE7
:10239000882309F466C02091261330E08091B007AD
:1023A00090E0F901EE0FFF1FE20FF31F74E0880FBA
:1023B000991F7A95E1F7E80FF91FE65DFC4E16814B
:1023C000123008F04EC0212F30E040E050E0C7014D
:1023D000B6010E94527E29833A834B835C838091AD
:1023E000B107882319F0B7DE802FFADCA3DD812F37
:1023F00090E0880F991F80930E13109211138AE0BA
:10240000809313138AE280931413FE013196838123
:102410008093161382818093171381818093181300
:1024200089818093191381E080931C136CDD8823CC
:10243000C1F0E091B007F0E054E0EE0FFF1F5A95B5
:10244000E1F7E45DFC4E808160E072E0A5010E944E
:102450000269803219F423DD08DE03C006DE9C0128
:1024600002C021E030E0C9010F900F900F900F9053
:10247000CF91DF911F910F91FF90EF90DF90CF9060
:10248000BF90AF9008956F927F928F929F92AF927C
:10249000BF92CF92DF92EF92FF920F931F93DF9341
:1024A000CF9300D000D000D0CDB7DEB7182F4A01AF
:1024B0005B01390195DC882309F43BC18091B107A8
:1024C0008823A1F1E091B007F0E054E0EE0FFF1F88
:1024D0005A95E1F7E65DFC4E90818091251398179F
:1024E00011F590912413809126139817E1F420910F
:1024F0005A1330915B1340915C1350915D13821617
:102500009306A406B50678F08091271390912813BE
:10251000A0E0B0E0820F931FA41FB51F8816990694
:10252000AA06BB0628F017DE812F5ADCCC2402C095
:10253000C82CC21A8091B107882309F064C0209189
:10254000261330E08091B00790E0F901EE0FFF1FF5
:10255000E20FF31F24E0880F991F2A95E1F7E80F97
:10256000F91FE65DFC4E0681C02EDD24EE24FF241B
:10257000C501B401A70196010E94527E2B833C83C2
:102580004D835E83C501B401A70196010E94527E6E
:10259000C62E0093271310922813861A9108A108BB
:1025A000B10880925A1390925B13A0925C13B09280
:1025B0005D13C0DC10920D1310E0000F111F00938B
:1025C0000E1310920F131092101380E880931113C2
:1025D0008AE08093131388E280931413FE013396EC
:1025E0008381809316138281809317138181809356
:1025F00018138B818093191381E080931C1383DC63
:10260000882309F496C0CC20D1F1809127139091B2
:1026100028138C1991099093281380932713809184
:102620005A1390915B13A0915C13B0915D138C0DC4
:10263000911DA11DB11D80935A1390935B13A0931C
:102640005C13B0935D1300E012E05E010894A11CDE
:10265000B11C1A830983E091B007F0E084E0EE0F2B
:10266000FF1F8A95E1F7E65DFC4E8181B50140E0F0
:1026700050E00E94DA698823A9F5CA9451F7809145
:102680002713909128130197909328138093271371
:1026900080915A1390915B13A0915C13B0915D13DC
:1026A0000196A11DB11D80935A1390935B13A093C3
:1026B0005C13B0935D1380E092E09A838983E0918C
:1026C000B007F0E014E0EE0FFF1F1A95E1F7E65DAA
:1026D000FC4E8181BE016F5F7F4FA3010E94DA69CA
:1026E000882329F0803209F4DADBBFDC22C0809134
:1026F000271390912813892BB9F0E091B007F0E0EF
:10270000B4E0EE0FFF1FBA95E1F7E65DFC4E808165
:1027100080932513809126138093241381E0809366
:10272000B10720E030E007C01092B1079EDC9C01A9
:1027300002C021E030E0C90126960FB6F894DEBF52
:102740000FBECDBFCF91DF911F910F91FF90EF9002
:10275000DF90CF90BF90AF909F908F907F906F90C1
:102760000895CF92DF92EF92FF920F931F93DF9322
:10277000CF93CDB7DEB72A970FB6F894DEBF0FBE62
:10278000CDBF182F4F83588769877A87790128DB57
:10279000882309F4A4C02091261330E08091B0076B
:1027A00090E0F901EE0FFF1FE20FF31FA4E0880F86
:1027B000991FAA95E1F7E80FF91FE65DFC4E8681A7
:1027C0008230E0F420C04F81588569857A85812F59
:1027D000970159DE9C01009709F083C001508F8159
:1027E0009885A985BA850196A11DB11D8F8398870B
:1027F000A987BA8780E092E0E80EF91E002319F756
:1028000020E030E06EC08091B107882319F0A3DC8E
:10281000812FE6DA802F90E0A0E0B0E079E0880F29
:10282000991FAA1FBB1F7A95D1F78B839C83AD8319
:10283000BE8380DBFE0133968B8180930D138181F3
:1028400080930E13828180930F13838180931013E2
:1028500080E8809311138AE08093131388E28093B9
:102860001413FE013796838180931613828180931F
:1028700017138181809318138F818093191300930C
:102880001C1341DB882359F180E092E09A8389830D
:102890006E010894C11CD11C1BC0E091B007F0E090
:1028A00064E0EE0FFF1F6A95E1F7E65DFC4E818163
:1028B000B601A7010E94DA69882329F0803209F461
:1028C000EEDAD3DB0CC0015080E092E0E80EF91E96
:1028D000002319F71092B107C8DB9C0102C021E068
:1028E00030E0C9012A960FB6F894DEBF0FBECDBF07
:1028F000CF91DF911F910F91FF90EF90DF90CF90DC
:1029000008951F93DF93CF93CDB7DEB7A1970FB68E
:10291000F894DEBF0FBECDBF182F62DA882319F4FA
:1029200022E030E038C08091B107882319F013DC31
:10293000812F56DAFFDA94E290930D1380E88093AA
:10294000111386E08093131382E180931413909304
:102950001813D9DA882319F421E030E01CC08FE184
:1029600090E09A838983E091B007F0E014E0EE0FE5
:10297000FF1F1A95E1F7E65DFC4E8181BE016F5F96
:102980007F4FAE014D5F5F4F0E94DA69803209F4DC
:1029900086DA6BDB9C01C901A1960FB6F894DEBF05
:1029A0000FBECDBFCF91DF911F9108951F93DF938D
:1029B000CF93CDB7DEB72E970FB6F894DEBF0FBE1C
:1029C000CDBF182F0DDA882309F456C020912613A5
:1029D00030E08091B00790E0F901EE0FFF1FE20FA9
:1029E000F31F24E0880F991F2A95E1F7E80FF91FDC
:1029F000E65DFC4E8681823008F03EC08091B107D2
:102A0000882319F0A8DB812FEBD994DA80E8809332
:102A1000111386E0809313138AE1809314139CE0D2
:102A200090930D138FE380931613909318136BDA22
:102A3000882311F18CE090E09A838983E091B007BC
:102A4000F0E084E0EE0FFF1F8A95E1F7E65DFC4EB3
:102A50008181BE016F5F7F4FAE014D5F5F4F0E946E
:102A6000DA69882321F0803209F419DA1D82FDDA4F
:102A700090E08D81803809F491E0892F2E960FB671
:102A8000F894DEBF0FBECDBFCF91DF911F910895A7
:102A9000FF920F931F93DF93CF93CDB7DEB72A97A3
:102AA0000FB6F894DEBF0FBECDBF182F062FF72E3E
:102AB00097D9882319F422E030E05AC08091B107F9
:102AC000882319F048DB812F8BD934DA88E0809392
:102AD0000D1380E8809311138AE08093131385E22D
:102AE0008093141310DA8823E9F088E090E09A8349
:102AF0008983E091B007F0E074E0EE0FFF1F7A9554
:102B0000E1F7E65DFC4E8181BE016F5F7F4FAE0154
:102B10004D5F5F4F0E94DA69882339F0803209F4F3
:102B2000BED9A3DA21E030E023C0E02FFF2D8B8156
:102B300083838C8182838D8181838E8180832091A8
:102B4000261330E08091B00790E0F901EE0FFF1FEF
:102B5000E20FF31F54E0880F991F5A95E1F7E80F31
:102B6000F91FE65DFC4E8985869586837EDA9C0199
:102B7000C9012A960FB6F894DEBF0FBECDBFCF9124
:102B8000DF911F910F91FF900895AF92BF92CF9266
:102B9000DF92EF92FF920F931F93DF93CF9300D0BA
:102BA00000D0CDB7DEB77091B11650912913809146
:102BB000B510E2EBF6E1EE24FF240AE410E00FC1C9
:102BC00080818093A1006481E09ED001E19EB00DE0
:102BD000F09EB00D1124A154B94E20E030E0F6C0B3
:102BE00059018D919C9111972F5F3F4F55960897F2
:102BF00009F0ECC0552321F44093B51090E014C0C7
:102C0000AAE2B3E190E006C08C915096841709F4D3
:102C1000E0C09F5F9517C0F3951709F0DAC09330B5
:102C200009F4D7C04093B510892F90E0BC0154E05F
:102C3000660F771F5A95E1F7665D7C4EFB01408376
:102C400045E1C42ED12CAC9CA001AD9C500DBC9C88
:102C5000500D11242AE430E0E29E8001E39E100D25
:102C6000F29E100D1124400F511F4F54594EFA017E
:102C7000258975010894E11CF11CDC0133E0AA0FE1
:102C8000BB1F3A95E1F727FF15C0EC9CF001ED9CC6
:102C9000F00DFC9CF00D1124E00FF11FEF54F94EE4
:102CA0008181FB018183AA0FBB1FA45DBC4EFA0189
:102CB000828D14C0FA01828DFB018183AA0FBB1F94
:102CC000A45DBC4EEC9CF001ED9CF00DFC9CF00D65
:102CD0001124E00FF11FEF54F94E81818C9381EAAA
:102CE000809355198EEF80935619109258191092AF
:102CF000571910925A191092591981E090E0909347
:102D00005C1980935B1910925D1981EF97E10E9425
:102D1000C460882311F01092F11790912913E92FC4
:102D2000F0E08091F1178F5F14E0EE0FFF1F1A950E
:102D3000E1F7E65DFC4E8383853010F084E0838309
:102D4000EDE2F3E1FF24292F30E0B4E0220F331F3E
:102D5000BA95E1F72E0F3F1F03C08081F80E7096E1
:102D6000E217F307D1F79093B0079F5F9093291371
:102D700000E0EE24E3946E010894C11CD11C15C040
:102D8000802F90E0FC01EE0FFF1FE80FF91FE20F0C
:102D9000F31FE65DFC4E1482E582102F1F0D812F7C
:102DA000B0DD812FB60174DE0F5F8091B007282F50
:102DB00030E0E4E0220F331FEA95E1F7F901E65D28
:102DC000FC4E83810817E0F281E010C0261708F45A
:102DD00007CF0894E11CF11CE65BFF4F842F4E2DBA
:102DE000E71608F4EDCE8093B51080E00F900F90B9
:102DF0000F900F90CF91DF911F910F91FF90EF9067
:102E0000DF90CF90BF90AF900895DF92EF92FF9246
:102E10000F931F93DF93CF9300D000D0CDB7DEB7D1
:102E2000D82E0E94F00E882319F442E050E07CC0B6
:102E30008091B107882321F08ED98D2D0E94F00E4C
:102E400079D81092111386E0809313131092141303
:102E50005AD8882319F441E050E066C006D9AC0185
:102E6000209126138091B0074115510509F04BC000
:102E700030E090E0F901EE0FFF1FE20FF31F24E0B6
:102E8000880F991F2A95E1F7E80FF91FE65DFC4EC0
:102E90008481882309F048C08D2DBE016F5F7F4F6C
:102EA000F7DD892B69F5E090B007FF240091261328
:102EB00010E08D2D7BDDF801EE0FFF1FE00FF11FFD
:102EC00014E0EE0CFF1C1A95E1F7EE0DFF1DE65D18
:102ED000FC4E85832091261330E08091B00790E06E
:102EE000F901EE0FFF1FE20FF31FA4E0880F991FF7
:102EF000AA95E1F7E80FF91FE65DFC4E81E08483B7
:102F000043E050E011C030E090E0F901EE0FFF1F08
:102F1000E20FF31F64E0880F991F6A95E1F7E80F4D
:102F2000F91FE65DFC4E1482CA010F900F900F90BE
:102F30000F90CF91DF911F910F91FF90EF90DF9055
:102F400008951F93182F61DF812F0E94F00E8823B0
:102F500011F481E015C02091261330E08091B00774
:102F600090E0F901EE0FFF1FE20FF31F74E0880FEE
:102F7000991F7A95E1F7E80FF91FE65DFC4E86810F
:102F80001F910895FC01AEE5B3E184918D933196D4
:102F900083E1AC37B807C9F7CD014E970C94073BD6
:102FA0004F925F926F927F928F929F92AF92BF9259
:102FB000CF92DF92EF92FF920F931F93DF93CF9305
:102FC000CDB7DEB7C054D0400FB6F894DEBF0FBE09
:102FD000CDBF7C016B01142F442359F000D082E057
:102FE00091E0EDB7FEB7928381830E94007F0F903E
:102FF0000F900E94B4352AAF3BAF4CAF5DAF6EAFC0
:103000007FAFFE01E05CFF4F8083DE011196FE0181
:10301000FA9687E001900D928150E1F7112359F063
:1030200000D085E091E0EDB7FEB7928381830E94E6
:10303000007F0F900F9080E00E94F03BC70160E09E
:1030400040E0A0DF882309F4EBC00E944A37112337
:1030500059F000D08FE191E0EDB7FEB79283818304
:103060000E94007F0F900F9081E00E94F03BC6010C
:1030700060E041E087DF882309F4D2C00E944A372C
:1030800000E05EE3452E51E0552E48E0E42EF12CA1
:10309000EC0EFD1E3FE7632E31E0732E22E0C22EC0
:1030A00021E0D22E96E6892E91E0992E8DE4A82E6D
:1030B00081E0B82E01C0015080E00E94F03B80E02A
:1030C00090E061E00E9483368823D9F4002309F45C
:1030D000BDC0112349F000D0EDB7FEB75282418246
:1030E0000E94007F0F900F900E948A37882309F476
:1030F00097C081E00E94F03B0E948A378823D9F66E
:103100008FC00E94FE358823F1F1112349F000D0D1
:10311000EDB7FEB7B282A1820E94007F0F900F90A0
:10312000C7016EE141E020E00E940136882309F4E6
:1031300077C00E94B738882309F472C081E00E94EA
:10314000F03B112379F000D0EDB7FEB7F282E182B7
:103150000E94007FEDB7FEB7D282C1820E94007F3D
:103160000F900F90C7010E94FC39882329F48091A9
:1031700006168A3209F054C00E94B738882309F431
:103180004FC00F5F99CF112349F000D0EDB7FEB7C4
:10319000928281820E94007F0F900F90C7016EE1A2
:1031A00041E020E00E9401368823D1F1112379F01B
:1031B00000D0EDB7FEB7F282E1820E94007FEDB74A
:1031C000FEB7D282C1820E94007F0F900F900E94B2
:1031D000E33B882329F181E00E94F03B14C08091F9
:1031E00006168A32E9F4112349F000D0EDB7FEB794
:1031F000728261820E94007F0F900F9081E00E9496
:10320000DE38882369F0C7010E94213D882339F305
:1032100080E00E94073C8823D9F3823009F44CCF28
:1032200080E00E94F03BCE0101960E94D63A112325
:1032300011F480E022C000D084EA91E0EDB7FEB73F
:10324000928381830E94007F80E015C080E00E940D
:10325000F03BCE0101960E94D63A112311F481E091
:103260000CC000D083EB91E0EDB7FEB79283818371
:103270000E94007F81E00F900F90C05CDF4F0FB67F
:10328000F894DEBF0FBECDBFCF91DF911F910F919C
:10329000FF90EF90DF90CF90BF90AF909F908F9076
:1032A0007F906F905F904F90089580918213887106
:1032B00011F481E0089583E18093061680E008957B
:1032C00020916C1630916D1640916E1650916F16CC
:1032D000211531054105510509F436C080910316C9
:1032E000833079F4283F8FEF38078FEF48078FE05E
:1032F000580760F580E0275F3F4F4F4F5F4039F53B
:1033000023C0823079F4283F8FEF380780E04807E8
:1033100080E05807D8F480E0275F3F4F404050409E
:10332000B1F412C0813011F080E00895283F8FE0A1
:10333000380780E0480780E0580740F480E0275FC6
:103340003F404040504019F481E0089582E00895E4
:103350001092081681E0809392138FEF809394135C
:10336000809393131092A5138093A7138093A613B1
:103370000895482F20E080919213841321E0209338
:10338000081630E083E190E0289FF001299FF00DBE
:10339000389FF00D1124EE56FC4E40838FEF828350
:1033A0008091681690916916A0916A16B0916B167B
:1033B00083839483A583B683809174169091751648
:1033C000A0917616B091771687839087A187B287F0
:1033D000089580910816282F30E083E190E0289F1F
:1033E000F001299FF00D389FF00D1124EE56FC4E90
:1033F0009081418180919213891739F480919313C0
:10340000841718F48F5F809393138091A513891705
:1034100039F48091A613841718F48F5F8093A61354
:1034200083E190E0289FF001299FF00D389FF00D77
:103430001124EE56FC4E11820895CF92DF92EF9246
:10344000FF920F931F938091081690E023E130E0E4
:10345000829F6001839FD00C929FD00C112482E93F
:1034600093E1C80ED91E2091B91530E040E050E03C
:10347000F601E780F08401851285C801B7010E943A
:10348000527E2091B815F601228370E080E090E032
:10349000E61AF70A080B190BE782F08601871287F4
:1034A00020917016309171164091721650917316DA
:1034B000261B370B480B590B2387348745875687C4
:1034C00020917416309175164091761650917716AA
:1034D000620F731F841F951F6787708B818B928B80
:1034E00078DF1F910F91FF90EF90DF90CF900895BC
:1034F0006F927F928F929F92AF92BF92CF92DF9204
:10350000EF92FF920F931F93CF93DF93682F7091E9
:10351000B815A0906816B0906916C0906A16D09041
:103520006B16609074167090751680907616909059
:10353000771680919213861711F58091941387174F
:10354000F1F48091951390919613A0919713B091F7
:1035500098138A159B05AC05BD0589F42091991334
:1035600030919A1340919B1350919C1362167306ED
:103570008406950620F0E0E060E070E029C08091CC
:10358000A513861709F0CAC08091A713871709F001
:10359000C5C08091A8139091A913A091AA13B091CE
:1035A000AB138A159B05AC05BD0509F0B7C020918A
:1035B000AC133091AD134091AE135091AF1362161E
:1035C00073068406950608F4A9C0E1E061E070E0A6
:1035D00083E190E0689FE001699FD00D789FD00D56
:1035E0001124CE56DC4EAF84B888C988DA88D4015D
:1035F000C301821B930BA40BB50B9C01AD018A1573
:103600009B05AC05BD0508F58B859C85AD85BE8504
:10361000820F931FA41FB51F80937016909371168D
:10362000A0937216B0937316A21AB30AC40AD50AED
:10363000A0927416B0927516C0927616D092771634
:10364000E0930816C6DE81E06CC0E09308168FEFA9
:103650008A83E090B915FF2400E010E06B857C853B
:103660008D859E856A0D7B1D8C1D9D1D6150704052
:10367000804090402091C2153091C3154091C415EF
:103680005091C515621B730B840B950B2091C615C9
:103690003091C7154091C8155091C915621B730B25
:1036A000840B950BA80197010E94527E2E5F3F4F1D
:1036B0004F4F5F4F209368163093691640936A16F8
:1036C00050936B168F819885A985BA85A80EB91E6F
:1036D000CA1EDB1E0894A108B108C108D108C601A2
:1036E000B501A80197010E94527ECA01B901A80143
:1036F00097010E94137EA4019301261B370B480BF0
:10370000590B209374163093751640937616509388
:1037100077166F82788689869A8602C0862F29DE80
:1037200080E0DF91CF911F910F91FF90EF90DF909C
:10373000CF90BF90AF909F908F907F906F900895A3
:10374000282FE0910416F091051685E0EE0FFF1F7B
:103750008A95E1F7F170E854FC4E9081992329F4A1
:103760008AE08093061680E008958BE08093061629
:10377000953E81F09E3271F0838583FD0BC084FFFE
:1037800004C080E0222339F403C080E0213019F422
:1037900081E0089580E008951F93DC0140910416B4
:1037A0005091051695E0440F551F9A95E1F7517019
:1037B00048545C4E10E06C916A3219F1FA01E10F45
:1037C000F11D70856717B1F0262F30E0872F90E04C
:1037D00080962817390771F06C3211F0662339F49E
:1037E000703229F40EC0662351F011966C916C3240
:1037F000D1F71FEF1F5F133020F41196DCCF80E06C
:1038000001C081E01F910895E0910416F091051622
:1038100025E0EE0FFF1F2A95E1F7F170E854FC4E0A
:1038200022E833E1838580938213D901119684893C
:1038300012968C931297858913968C931397828D89
:1038400080938313838D11968C93DF015C962B5F9D
:103850003F4F848D8093871311968C911197F901B6
:10386000818312968C911297828313968C91838315
:1038700008958DE0809306168091821380710895DB
:103880008FEF9FEF90930516809304169093D515B4
:103890008093D4158091DB15882311F41092DA15EA
:1038A0001092821310928313109284131092851336
:1038B0001092861310928713109288131092891316
:1038C00010928A1310928013089581E080935E16FF
:1038D000E0910416F091051635E0EE0FFF1F3A95C2
:1038E000E1F7F170E854FC4E22E833E18091821355
:1038F0008387D901119612968C911297848B139617
:103900008C911397858B80918313828F11968C9164
:10391000838FDF015C962B5F3F4F80918713848FED
:10392000F901818111968C931197828112968C9363
:103930001297838113968C9308950F931F93CF93BF
:10394000DF93EC01042F86E180930616A091041604
:10395000B091051645E0AA0FBB1F4A95E1F7B1707B
:10396000A854BC4E11E040E050E070E0615070405F
:103970005B30A9F0FD01E50FF11DE081583011F435
:10398000112321F4E03261F4593048F418968C91F7
:103990001897803221F010E0EEE257E001C0E0E03D
:1039A000013089F480910716882309F5842F90E06F
:1039B000861797070CF0E0E08E2F81548A3108F4C7
:1039C000E05EE88314C028812A3229F1EE2321F435
:1039D0002C3579F02F3269F02E1749F030E08E2F18
:1039E00090E080962817390711F080E015C0EE238B
:1039F00051F480910716882371F0842F90E001968E
:103A00009983888308C080910716882309F421963A
:103A10004F5F5F5FADCF81E0DF91CF911F910F913D
:103A20000895DF92EF92FF920F931F93DF93CF934E
:103A300000D0CDB7DEB78C01D22EE0910416F09104
:103A4000051655E0EE0FFF1F5A95E1F7F170E854A7
:103A5000FC4E9081992329F0953E19F083858F3093
:103A600011F08BE06DC080910716882311F096FF4E
:103A700066C0DF01119650E07E010894E11CF11C44
:103A800070E0615070408C91F701808311968C91A9
:103A900011978183413081F4809107168823A1F525
:103AA000852F90E0861797071CF0F801108278C0E8
:103AB0008981F801808328C0F8018081E82FFF27E1
:103AC000E7FDF095EA32F10509F46AC029813A81EF
:103AD0002115310531F4EC35F105B1F0EF32F10586
:103AE00099F0C9018096E817F90711F4DD2061F01B
:103AF000C9018097E817F90711F4DD2029F0E217D2
:103B0000F30711F086E11CC089819A81892B49F461
:103B100080910716882309F443C0852F90E0019611
:103B20001BC0543011F4139632C05A3011F412965F
:103B30002EC05C3061F55E978C9186FD05C080E1FA
:103B40008093061680E02DC0413051F48091071615
:103B5000882331F08EE090E0F8019183808320C0CB
:103B6000413019F4F80111821BC0F80181819927B5
:103B700087FD9095009739F08C35910521F020E074
:103B800030E08F9711F421E030E0822F0AC080915D
:103B90000716882311F40F5F1F4F5F5F129673CFD4
:103BA00081E00F900F90CF91DF911F910F91FF90C7
:103BB000EF90DF900895009739F08C35910521F052
:103BC00020E030E08F9711F421E030E0822F08955B
:103BD000209104163091051665E0220F331F6A9577
:103BE000E1F7317028543C4EC90108958FEF80935E
:103BF000591610925E168FEF9FEFAFEFBFEF8093D5
:103C00005F1690936016A0936116B09362160895A4
:103C100081E080935E1608959091B8158091FD150E
:103C2000882341F080910B16981721F48091DF15BD
:103C3000882361F480910016882369F08091321600
:103C4000981749F48091EE15882329F088E2809333
:103C5000061680E0089581E00895F82FE091B815E8
:103C60002091D0153091D1154091D2155091D31596
:103C700060910416709105168091FD15882319F145
:103C800080910B16E817F9F4809123169091241671
:103C9000A0912516B0912616281739074A075B0709
:103CA00091F48091FE159091FF156817790759F4EA
:103CB000FF2329F48091DF1581FF05C02CC080917E
:103CC000DF15882311F580910016882349F1809132
:103CD0003216E81729F580914A1690914B16A0915B
:103CE0004C16B0914D16281739074A075B07C1F4E7
:103CF00080910116909102166817790789F4FF23C5
:103D000031F08091EE15882359F088E205C080914A
:103D1000EE1581FF05C089E28093061680E00895C4
:103D200081E00895882309F442C0482F4150242F90
:103D300030E087E290E0289FF001299FF00D389F46
:103D4000F00D1124E55FF94EA8EBB5E187E20D9087
:103D500001928150E1F7F901B4E0EE0FFF1FBA952F
:103D6000E1F7E21BF30BE152FA4EA0E8B3E18FE07A
:103D70000D9001928150E1F7F901EE0FFF1FE20F64
:103D8000F31FE350FA4EA3E0B6E183E00D900192F9
:103D90008150E1F7842F90E0FC0174E0EE0FFF1FEB
:103DA0007A95E1F7E81BF90BE152FA4E108208957B
:103DB000DF93CF93CDB7DEB7A7970FB6F894DEBFEA
:103DC0000FBECDBF882309F46AC0DE011196E8EB6F
:103DD000F5E197E201900D929150E1F78150482F63
:103DE00050E087E290E0489F9001499F300D589F36
:103DF000300D1124255F394EA8EBB5E1F90187E2BA
:103E000001900D928150E1F7D901FE01319687E2D0
:103E100001900D928150E1F7DE011196E0E8F3E1A7
:103E20008FE001900D928150E1F7CA0134E0880FD4
:103E3000991F3A95E1F7841B950B81529A4EA0E8A1
:103E4000B3E1FC012FE001900D922150E1F7DC017C
:103E5000FE0131968FE001900D928150E1F7DE0175
:103E60001196E3E0F6E183E001900D928150E1F7D5
:103E7000CA01880F991F840F951F83509A4EA3E0A3
:103E8000B6E1FC0123E001900D922150E1F7DC0145
:103E9000FE01319683E001900D928150E1F7A796E3
:103EA0000FB6F894DEBF0FBECDBFCF91DF9108955E
:103EB0001F9310915E16113001F510925E168091DD
:103EC00059160E942641882321F084E1809306162A
:103ED00012C040915A1650915B1660915C16709119
:103EE0005D168091591628EB33E10E94A940892B79
:103EF00021F01093061680E001C081E01F91089523
:103F000080E092E0E8EBF3E1DF019C011D9221509B
:103F10003040E1F708951F93182F90915916809122
:103F2000B8159817A9F420915A1630915B16409154
:103F30005C1650915D1680917C1390917D13A09139
:103F40007E13B0917F13281739074A075B07B9F131
:103F5000AFDF8823A9F18FEF8093591610925E1678
:103F60008FEF9FEFAFEFBFEF80935F1690936016D8
:103F7000A0936116B093621640917C1350917D130B
:103F800060917E1370917F1340935A1650935B1685
:103F900060935C1670935D16112369F08091B815DB
:103FA00028EB33E10E94B340892B29F081E0809314
:103FB000061680E005C08091B8158093591681E0FF
:103FC0001F9108958091031620918F1330919013C3
:103FD000833019F42C5F3F4F02C02E5F3F4F309368
:103FE000901320938F1380918F1390919013805092
:103FF0009240D9F41092901310928F1380917C13F9
:1040000090917D13A0917E13B0917F130196A11D15
:10401000B11D80937C1390937D13A0937E13B09376
:104020007F1381E078DF8823C9F0E0918F13F0914E
:104030009013E854FC4E808180936C1681818093AC
:104040006D1680910316833011F081E0089582810E
:1040500080936E16838180936F1681E00895CF92CE
:10406000DF92EF92FF920F931F93DF93CF9300D0D5
:10407000CDB7DEB7E82E409103164330D9F48091D6
:10408000681690916916A0916A16B0916B16E7E0D8
:10409000B695A79597958795EA95D1F79A838983E1
:1040A0008091681690E08F779070880F991F880F25
:1040B000991F0BC0423071F48091691689831A826E
:1040C0008091681690E0880F991F909390138093C9
:1040D0008F1318C04130B1F42091681630916916E1
:1040E000C90196958795820F931F909390138093A3
:1040F0008F1380919013982F969599831A828170CF
:1041000080939013EE2071F129813A8180910916F4
:1041100090910A162817390720F430930A16209335
:10412000091680917816909179168217930720F4DA
:1041300030937916209378164130A1F480918F1333
:10414000909190138F5F914069F42F5F3F4F809162
:104150007816909179168217930720F43093791688
:104160002093781689819A81A0E0B0E02091C21551
:104170003091C3154091C4155091C515820F931FFE
:10418000A41FB51F80937C1390937D13A0937E137F
:10419000B0937F1381E0BFDE882309F4C3C0209170
:1041A0008F1330919013890108541C4EF801F08050
:1041B00091816E010894C11CD11C82818983838105
:1041C000F6018183809103168130E9F42F5F31403D
:1041D000D1F480917C1390917D13A0917E13B091C6
:1041E0007F130196A11DB11D80937C1390937D13C5
:1041F000A0937E13B0937F1381E08DDE882309F4B2
:1042000091C09091B813EE2051F5F0926C169093F6
:104210006D1680910316833049F4F60180818093F6
:104220006E1681818F7080936F1661C010926E162A
:1042300010926F16813009F05AC08091681680FF85
:104240000AC0892F8295807FF2944FE0F4228F0D6F
:1042500080936C1692959F7090936D1648C08091D4
:104260000316813009F045C08091681680FF10C0A8
:10427000FFE0FF2290916C16892F8295807FF80EC7
:1042800020916D162295207F92959F70290F08C06E
:10429000F0906C16292F207F80916D168F70280F5B
:1042A00080918F13909190138F5F9140A1F520938F
:1042B000B81311E010935E1680917C1390917D13DA
:1042C000A0917E13B0917F130197A109B10980934A
:1042D0007C1390937D13A0937E13B0937F1381E0A2
:1042E0001ADE8823F9F0F092B71510935E1681E07C
:1042F0001AC0F0906C1620916D16833061F4809195
:104300006E16F8018283F6018181807F90916F168D
:10431000890FF8018383F801F082218381E0809383
:104320005E1601C080E00F900F90CF91DF911F913A
:104330000F91FF90EF90DF90CF9008952F923F92D2
:104340004F925F926F927F928F929F92AF92BF92A5
:10435000CF92DF92EF92FF920F931F93DF93CF9351
:1043600000D0CDB7DEB78A83162F88E0809306167B
:1043700080910316833061F42A81233049F46FEF72
:104380007FEF8FEF9FEF0E94182E882309F4DDC284
:104390008091701690917116A0917216B09173165B
:1043A0000097A105B10509F05EC08A81833009F448
:1043B000CCC290910316892F8150823008F040C002
:1043C000A0907416B0907516C0907616D09077169F
:1043D0008091CC159091CD157C0100E010E0AE14D9
:1043E000BF04C006D10608F0BCC12091C2153091AF
:1043F000C3154091C4155091C5152A0D3B1D4C1D88
:104400005D1D8091CA159091CB15A0E0B0E0280FFA
:10441000391F4A1F5B1F209370163093711640930B
:10442000721650937316EA18FB080C091D09E092E6
:104430007416F0927516009376161093771605C2CF
:104440009330E1F48091CA159091CB15A091CC15D1
:10445000B091CD158093681690936916A0936A1653
:10446000B0936B160BC08093681690936916A09357
:104470006A16B0936B169A81933029F0812F38D841
:10448000882321F0E2C10E94A81906D78FEF8093FC
:1044900073166090741670907516809076169090D2
:1044A0007716A091B915A983AA2EBB24CC24DD24AC
:1044B0006A147B048C049D0408F0C4C02090681624
:1044C0003090691640906A1650906B16E090C215B5
:1044D000F090C3150091C4151091C515E60CF71C9A
:1044E000081D191D8091C6159091C715A091C8157A
:1044F000B091C915E80EF91E0A1F1B1FC201B101B8
:104500006250704080409040A60195010E94137E49
:10451000E60EF71E081F191FE0927016F092711632
:104520000093721610937316BA81B230D9F4A6189C
:10453000B708C808D908A0927416B0927516C09230
:104540007616D09277160E941D1A81E090E0A0E0C6
:10455000B0E08093741690937516A0937616B0937E
:10456000771673C1E9818E2F90E020917416821B1B
:104570009109AA2797FDA095BA2F8093741690935E
:104580007516A0937616B0937716FA81F13009F07C
:1045900059C080910316813009F454C080E05FDD7A
:1045A000882309F4D2C1E0906816F0906916009152
:1045B0006A1610916B16A80197012F5F3F4F4F4F5E
:1045C0005F4F209368163093691640936A16509394
:1045D0006B1680916C1690916D16A0916E16B0912D
:1045E0006F16281739074A075B0751F1E0926816E2
:1045F000F092691600936A1610936B16E218F3088E
:10460000040915092091B91530E040E050E0C801D7
:10461000B7010E94137E2091741630917516409157
:10462000761650917716260F371F481F591F209373
:10463000741630937516409376165093771602C011
:10464000C1DCAECF80E00BDD882309F47EC10E947F
:104650006019182F813009F478C1809173168F3F4B
:1046600009F0D5C0123009F080C0609074167090C7
:10467000751680907616909077168091081690E0C7
:1046800023E130E0829FF001839FF00D929FF00DB7
:104690001124EE56FC4E87819085A185B28586193E
:1046A0009709A809B90987839087A187B287A09045
:1046B000B915BB24CC24DD24E090C615F090C715B5
:1046C0000091C8151091C9158091C2159091C3151C
:1046D000A091C415B091C515E80EF91E0A1F1B1F45
:1046E000209168163091691640916A1650916B16A8
:1046F0002250304040405040C601B5010E94137E18
:10470000E60EF71E081F191FE0927016F092711640
:104710000093721610937316A0927416B0927516C9
:10472000C0927616D09277162A81233011F00E941B
:104730001D1A8091681690916916A0916A16B09121
:104740006B168093701690937116A0937216B093A7
:104750007316609274167092751680927616909207
:1047600077168AE180930616F0C08091B9152091E2
:104770007416309175164091761650917716281B55
:1047800031094109510920937416309375164093ED
:104790007616509377168A81833009F0C5C02115AB
:1047A00031054105510509F0BFC080916C1690910B
:1047B0006D16A0916E16B0916F168093701690933F
:1047C0007116A0937216B09373168FEF9FEFAFEF31
:1047D000BFE080936C1690936D16A0936E16B09305
:1047E0006F1681E03CDC882309F4AFC0809170161D
:1047F00090917116A0917216B091731680936C16F9
:1048000090936D16A0936E16B0936F168DC09A811B
:104810009130E9F48091681690916916A0916A161A
:10482000B0916B160196A11DB11D20916C163091AF
:104830006D1640916E1650916F1682179307A4075C
:10484000B50709F453C00E941D1A81E07FC0AA81F8
:10485000A33009F04BC080916C1690916D16A09119
:104860006E16B0916F168093701690937116A09388
:104870007216B093731610926C1610926D161092F9
:104880006E1610926F168091B91590E0A0E0B0E01E
:1048900020917416309175164091761650917716C6
:1048A000281739074A075B0760F48FEF9FEFAFEFD8
:1048B000BFE080936C1690936D16A0936E16B09324
:1048C0006F1681E0CCDB882309F43FC0809170161D
:1048D00090917116A0917216B091731680936C1618
:1048E00090936D16A0936E16B0936F16123031F43C
:1048F0009A81933009F0A7CF2FD528C02091B91500
:104900008091741690917516A0917616B0917716D5
:10491000820F911DA11DB11D809374169093751681
:10492000A0937616B093771680916C1690916D16C1
:10493000A0916E16B0916F168093681690936916C9
:10494000A0936A16B0936B16A4CD80E00F900F90E1
:10495000CF91DF911F910F91FF90EF90DF90CF905B
:10496000BF90AF909F908F907F906F905F904F908F
:104970003F902F900895EF92FF920F931F93809195
:10498000041690910516F4E096958795FA95E1F74F
:104990007C0100E010E0909159168091B8159817AD
:1049A00019F520915F163091601640916116509173
:1049B00062168091D0159091D115A091D215B09129
:1049C000D315281739074A075B0771F480916316DE
:1049D00090916416A0916516B09166168E159F058C
:1049E000A007B10709F449C08091D0159091D11565
:1049F000A091D215B091D315809370169093711633
:104A0000A0937216B0937316E0927416F092751616
:104A1000009376161093771682E060E08FDC88238F
:104A200071F18091701690917116A0917216B091EB
:104A3000731680937C1390937D13A0937E13B09391
:104A40007F1381E068DA8823D1F08091D0159091AE
:104A5000D115A091D215B091D31580935F16909384
:104A60006016A0936116B0936216E0926316F092FE
:104A70006416009365161093661681E001C080E00D
:104A80001F910F91FF90EF900895DF92EF92FF92A8
:104A90000F931F93D82E20918B1330918C1340913C
:104AA0008D1350918E1379018A01A9E0169507950F
:104AB000F794E794AA95D1F782E0D81651F5909132
:104AC00059168091B815981709F040C020915F16CB
:104AD0003091601640916116509162168091831357
:104AE00090918413A0918513B091861328173907EC
:104AF0004A075B0759F58091631690916416A0915F
:104B00006516B09166168E159F05A007B107F1F4E2
:104B100078C083E0D816D1F48091831390918413E8
:104B2000A0918513B09186130097A105B10509F4F2
:104B300068C0317040705070211531054105510534
:104B400029F00894E11CF11C011D111D80918313B3
:104B500090918413A0918513B09186138093701661
:104B600090937116A0937216B0937316E092741618
:104B7000F0927516009376161093771682E0D81689
:104B800031F08D2D61E0DADB882399F13AC081E0C4
:104B900061E0D4DB8823B9F1809170169091711691
:104BA000A0917216B091731680937C1390937D132D
:104BB000A0937E13B0937F1381E0ADD9882319F1C0
:104BC0008091831390918413A0918513B0918613E3
:104BD00080935F1690936016A0936116B09362164F
:104BE000E0926316F09264160093651610936616B1
:104BF00008C083E0D81639F490E0809106168A3117
:104C000019F491E001C090E0892F1F910F91FF905E
:104C1000EF90DF900895DF92EF92FF920F931F9332
:104C2000D82E7A018B018091831390918413A091E7
:104C30008513B09186130097A105B10579F48FEF24
:104C40008093731610927416109275161092761641
:104C50001092771681E00E94B91929C08D2D15DFB9
:104C6000882311F081E0D7C0809106168A3109F0BF
:104C7000D1C08091081690E023E130E0829FF001DE
:104C8000839FF00D929FF00D1124EE56FC4E8FEF96
:104C900082832091B91587819085A185B285820F85
:104CA000911DA11DB11D87839087A187B28781E0E7
:104CB000D81649F4E0927416F092751600937616A1
:104CC000109377160CC081E090E0A0E0B0E08093F4
:104CD000741690937516A0937616B09377160E946B
:104CE0007B2E882309F496C08091831390918413BE
:104CF000A0918513B09186130097A105B10511F518
:104D000040917016509171166091721670917316E1
:104D10008091081690E023E130E0829FF001839FAC
:104D2000F00D929FF00D1124EE56FC4E43835483F8
:104D30006583768340938313509384136093851324
:104D40007093861381E0D816A9F48091741690911F
:104D50007516A0917616B0917716E81AF90A0A0B23
:104D60001B0BE0927416F092751600937616109352
:104D7000771618C081E090E0A0E0B0E020917416B2
:104D8000309175164091761650917716821B930BD1
:104D9000A40BB50B8093741690937516A09376169A
:104DA000B0937716E090C615F090C7150091C8151E
:104DB0001091C9158091C2159091C315A091C41589
:104DC000B091C515E80EF91E0A1F1B1F6091B91599
:104DD00070E080E090E02091701630917116409163
:104DE00072165091731622503040404050400E943D
:104DF000137EE60EF71E081F191FE0927016F09240
:104E0000711600937216109373160E941D1A8D2D41
:104E10003CDE01C080E01F910F91FF90EF90DF908A
:104E20000895BF92CF92DF92EF92FF920F931F935C
:104E3000CF93DF9380919113882309F04CC0809128
:104E4000B8158F3F11F481E03FC010E0BB24BA9445
:104E5000CC24CA94DC2C760101E08091B8150E9424
:104E60003C41EC010097B9F11092031610928013A7
:104E70009091B81580910B16981721F41092FD159A
:104E80001092DF1580913216981721F410920016B7
:104E90001092EE1580915916981761F4B092591638
:104EA00010925E16C0925F16D0926016E092611664
:104EB000F09262160E94A81900930616C330D1051D
:104EC00031F0229751F488E18093061606C01F5FE7
:104ED000143619F602C081E001C080E0DF91CF9165
:104EE0001F910F91FF90EF90DF90CF90BF900895AA
:104EF00098DF882369F080910316882349F0809118
:104F00008013882329F085E08093061680E00895B9
:104F100081E0089586DF882371F08091031688234D
:104F200049F40E94AF33882329F48EE0809306165B
:104F300080E0089581E00895EDDF882369F0809195
:104F40000416909105168F5F9F4F11F081E0089530
:104F50008FE08093061680E00895DCDF8823B1F0AF
:104F600080910416909105168F5F9F4F29F48FE072
:104F70008093061680E0089580918013882311F0B5
:104F800081E0089587E18093061680E00895C2DFEE
:104F9000882369F080910416909105168F5F9F4FCA
:104FA00029F48FE08093061680E00895A1CF08953C
:104FB000B1DF882309F09CCF08952F923F924F9242
:104FC0005F926F927F928F929F92AF92BF92CF9299
:104FD000DF92EF92FF920F931F93DF93CF9300D056
:104FE000CDB7DEB7982F8250823070F080917A165C
:104FF00090917B16A0917C16B0917D1681509040C7
:10500000A041B04018F02FC0923069F580917A1617
:1050100090917B16A0917C16B0917D16813030E185
:10502000930730E0A30730E0B30710F48CE283C0AD
:1050300081509847A040B04078F481E080930316F7
:10504000E1ECF1E024E1A0907A16B0907B16C090DC
:105050007C16D0907D160FC082E080930316E5ED9C
:10506000F1E028E2F0CF83E080930316EDEFF1E06A
:105070002EE1E9CF359680819181A281B3818A1595
:105080009B05AC05BD0520F084818093B91502C055
:10509000215081F72091B915222309F44BC06623D2
:1050A00069F081E090E0A0E0B0E08093C2159093B9
:1050B000C315A093C415B093C51508C01092C215AE
:1050C0001092C3151092C4151092C5156091031665
:1050D000613009F061C08091C2159091C315A09113
:1050E000C415B091C5150196A11DB11D8093C215BF
:1050F0009093C315A093C415B093C51551E0E52E48
:10510000F12C42E0642E712C812C34E0932E150199
:10511000260108942108310841085108A22EBB2419
:10512000CC24DD245DE0E516F10448F0F092BB15D7
:10513000E092BA1581E28093061680E081C0C30137
:10514000A0E0B0E0A2019101281B390B4A0B5B0BD8
:10515000CA01B901A60195010E94527E89019A01F6
:105160000E5F1F4FC40163E070E00E943E7E970116
:105170002F5F3F4F42E050E0640E751E40E054E068
:10518000840E951E6017710710F47901CBCFF09251
:10519000BB15E092BA1553C06330F9F48091C21583
:1051A0009091C315A091C415B091C5158096A11D0D
:1051B000B11D8093C2159093C315A093C415B093ED
:1051C000C515822F90E09695982F882797958795FB
:1051D00001969A838983E0E21AC0623011F0E0E020
:1051E00016C08091C2159091C315A091C415B091BD
:1051F000C5150196A11DB11D8093C2159093C315CD
:10520000A093C415B093C5152A836983E1E229816F
:105210003A8140E050E0CA01B901615070408040DD
:1052200090406A0D7B1D8C1D9D1D6E1B71098109AF
:1052300091090E94527E3093BB152093BA1581E0EC
:105240000F900F90CF91DF911F910F91FF90EF90F2
:10525000DF90CF90BF90AF909F908F907F906F9096
:105260005F904F903F902F900895982F81528E35E8
:1052700080F480548A3110F490520CC0E4E7F2E0DC
:105280008081981731F0319682E0EB37F807C1F74B
:1052900001C090E0892F08958FEF9FEF90930A1639
:1052A00080930916109279161092781608951F931C
:1052B0001092741610927516109276161092771638
:1052C00082E060E03BD8882309F443C08091B9159F
:1052D00090E00197AA2797FDA095BA2F209170160C
:1052E000309171164091721650917316820F931F70
:1052F000A41FB51F80937C1390937D13A0937E13FE
:10530000B0937F1310E01FC080E00E948B1F8823A2
:1053100001F1112311F40E94801F0E94081E809148
:105320007C1390917D13A0917E13B0917F13019710
:10533000A109B10980937C1390937D13A0937E13F0
:10534000B0937F131F5F8091B9158117E9F681E053
:1053500001C080E01F91089551C0C901A0E0B0E0F4
:105360002091C2153091C3154091C4155091C515B7
:10537000820F931FA41FB51F80937C1390937D13FE
:10538000A0937E13B0937F1381E00E948B1F88232C
:1053900009F442C08091091690910A16A0E0B0E08D
:1053A0002091BA153091BB1540E050E0820F931F59
:1053B000A41FB51F2091C2153091C3154091C4158B
:1053C0005091C515820F931FA41FB51F80937C13A6
:1053D00090937D13A0937E13B0937F1380E00E947F
:1053E0008B1F8823C9F00E94081E80910916909196
:1053F0000A16019690930A168093091620910916B1
:1054000030910A1680917816909179168217930739
:1054100008F0A3CF81E0089580E0089548DF882355
:10542000A1F10E94081E8EE28093B813E9EBF3E12C
:1054300080E2819393E1E33CF907D9F780E180832F
:1054400080918313878780918413808B809185134B
:1054500081878091861382878EE2858B868B7796F3
:1054600080E2819393E1E33EF907D9F780E18083FD
:105470008091D01587878091D115808B8091D2152E
:1054800081878091D315828781E0089510927C13E3
:1054900010927D1310927E1310927F1380E00E9471
:1054A0008B1F882309F455C00E94081E0E94801F8C
:1054B00085E58093B6158AEA8093B7151092761524
:1054C00082E08093781580910316833009F442C0FE
:1054D000823089F480917A1690917B16A0917C1687
:1054E000B0917D1680509040A140B04010F494E0FF
:1054F00006C096E004C090E0813009F491E09093FA
:105500007A1530917B1620917A16832F880F880F99
:10551000922F9295969596959370890F80937B150F
:10552000832F807C922F9F73890F80937C1590919D
:105530007C1690937D1581E080937E1520938215D3
:10554000309383159093841580917D1680938515F3
:1055500081E008959BE0D3CFEF92FF920F931F93CA
:10556000DF93CF9300D0CDB7DEB77C01062F142F89
:105570000E94081E0E94E81DFC01119321E030E00A
:105580005FEFBE016F5F7F4F4FE02B3011F4408320
:105590002CC02C3051F12A3141F12B3131F12D3019
:1055A00011F4008322C03323F9F4D7018C91992799
:1055B00087FD90959A8389838C35910511F08F979B
:1055C00011F41A82198230E089819A81892B09F4B9
:1055D00031E0DB018C91819311968C9180832F5F58
:1055E0000894E11CF11C01C050832F5F203210F49D
:1055F0003196CBCF0F900F90CF91DF911F910F91EC
:10560000FF90EF900895EF92FF920F931F93CF9327
:10561000DF93F82E10E065EEE62EADD9882311F465
:1056200090E030C00E94E81DEC0108818B858F302E
:1056300011F0112399F4E8820E94081E8B858F30A7
:1056400011F406FD0BC08091041690910516019788
:10565000909305168093041611E0DFCFFF2011F41C
:1056600091E010C010928B1310928C1310928D1336
:1056700010928E1383E009DA90E0882309F491E018
:1056800081E09827892FDF91CF911F910F91FF9093
:10569000EF900895CF92DF92EF92FF920F931F93B6
:1056A000DF93CF93CDB7DEB7A0970FB6F894DEBFE8
:1056B0000FBECDBFEE24FF2400E010E06E01089481
:1056C000C11CD11CF0920516E092041654D988230F
:1056D00031F4809106168A3109F04FC006C00E944D
:1056E000E81DFC018081882329F51093051600939D
:1056F000041610E216C03FD9882309F43EC00E9468
:10570000E81DDC01812F1D928A95E9F70E94081E91
:10571000809104169091051601969093051680933A
:10572000041680910416909105168E159F0519F7A1
:1057300081E024C0853EE9F0E016F106C1F0D60113
:1057400080E201900D928150E1F7109305160093CD
:10575000041611D9882389F00E94E81DDC01F601A6
:1057600080E201900D928150E1F70E94081E0F5FC8
:105770001F4F0894E11CF11CA5CF80E0A0960FB646
:10578000F894DEBF0FBECDBFCF91DF911F910F9177
:10579000FF90EF90DF90CF900895EF92FF920F93DC
:1057A0001F93CF93DF93EC0112E00DE08881E82E88
:1057B000FF24E7FCF094C7010E94DB1D8823A9F4B5
:1057C000EDE6F2E0808190E0E816F90611F48CE154
:1057D0000FC0319682E0E437F807A1F7002311F4F7
:1057E0001F5F0DE001502196E1CF153120F08BE2D3
:1057F0008093061610E0812FDF91CF911F910F91BA
:10580000FF90EF9008953F924F925F926F927F9238
:105810008F929F92AF92BF92CF92DF92EF92FF92C0
:105820000F931F93CF93DF936C013B01142F822EB4
:10583000222319F0AA24BB2405C00E94081E0E943E
:10584000E81D5C011A3010F421E005C0143610F098
:1058500023E001C022E0812F6AE00E94327EF0E363
:105860003F2E390E812F64E60E94327E892F6AE036
:105870000E94327EE0E34E2E480E812F64E60E94A5
:10588000327E70E3572E580EEE2401E0FF24C22F23
:10589000D0E0C095D0952896922E919486E0980EEF
:1058A00001C007E0F6011081013079F48E2D90E0FF
:1058B000C817D90741F01E3231F0812F90E00E94C5
:1058C000DB1D882379F002E0EDCF083099F4FBE08E
:1058D000EF1631F0812F90E00E94DB1D882311F03C
:1058E00009E0E0CF812FC1DC182F0894C11CD11C26
:1058F0008823C1F2073071F41E3231F0812F90E01D
:105900000E94DB1D882311F008E0CCCF0894C11C55
:10591000D11CC8CF063021F488E0E816D9F4C1CFF5
:10592000093021F4EBE0EE16A9F427C0053019F494
:10593000132D06E010C0043019F4142D05E00BC03F
:10594000033019F4152D04E006C0023021F4092DAE
:105950001EE701C010E2882021F0F30111933F01FE
:1059600003C0F50111935F01E3948F2D879588277C
:105970008795F694F80EF10E95CF8F2DDF91CF918C
:105980001F910F91FF90EF90DF90CF90BF90AF905D
:105990009F908F907F906F905F904F903F90089571
:1059A000CF93DF93EC010E94E81DFC0180818823E6
:1059B00011F48AE006C0853E19F083858F3029F402
:1059C0008BE08093061680E00EC08BE08093061675
:1059D000CF01BE014BE050E00E947C7E9C0180E044
:1059E000232B09F481E0DF91CF910895CF92DF92CC
:1059F000EF92FF921F93DF93CF93CDB7DEB72B9734
:105A00000FB6F894DEBF0FBECDBF7C0110E06E0173
:105A10000894C11CD11C02C01F3F29F11F5FC701A0
:105A2000B601412F21E0EFDE109205161092041608
:105A30000E94BB24882329F4809106168A3199F4A8
:105A400013C0C601ADDF882339F7809106168A306E
:105A500059F08091041690910516019690930516C1
:105A600080930416E5CF10E0812F2B960FB6F894A3
:105A7000DEBF0FBECDBFCF91DF911F91FF90EF90A2
:105A8000DF90CF9008951F93CF93DF93182F0E943C
:105A9000581F882309F469C00E94801F112329F030
:105AA00082E090E0A0E0B0E004C081E090E0A0E0FF
:105AB000B0E080937C1390937D13A0937E13B093FA
:105AC0007F1380910316833019F080E290E017C0B5
:105AD00080917C1390917D13A0917E13B0917F13E0
:105AE0000196A11DB11D80937C1390937D13A0930B
:105AF0007E13B0937F138091B91590E04E96C091BC
:105B0000BA15D091BB15CC0FDD1FC80FD91F29C006
:105B100081E00E948B1F882341F1E8EBF3E1808153
:105B2000882329F00E94801F0E94081E06C085E17C
:105B3000E73BF80711F03196F2CF80917C139091FA
:105B40007D13A0917E13B0917F130196A11DB11D0D
:105B500080937C1390937D13A0937E13B0937F1357
:105B600021972097A9F681E001C080E0DF91CF91D5
:105B70001F9108958091C2159091C315A091C415ED
:105B8000B091C51580937C1390937D13A0937E13E1
:105B9000B0937F1380E00E948B1F882309F446C0D6
:105BA0000E94081E80910316833039F481E692E04A
:105BB00068EB73E14CE00E94C707809103168230C6
:105BC00039F48DE592E068EB73E144E00E94C70789
:105BD00080910316813039F48AE592E068EB73E135
:105BE00043E00E94C7078091BA159091BB15A0E0D1
:105BF000B0E02091C2153091C3154091C415509169
:105C0000C515820F931FA41FB51F80937C1390931B
:105C10007D13A0937E13B0937F1380E00E948B1FAF
:105C2000882321F00E94081E81E0089580E00895F5
:105C3000DF93CF9300D000D0CDB7DEB769837A83EE
:105C40008B839C832091BC153091BD1540E050E0C2
:105C50008091C2159091C315A091C415B091C5153E
:105C6000821B930BA40BB50B80937C1390937D1335
:105C7000A0937E13B0937F1380E00E948B1F882334
:105C800099F10E94081E0E94801F82E592E068EB55
:105C900073E144E00E94C70786E592E06CE975E194
:105CA00044E00E94C707FE01319689818093A015C8
:105CB00081818093A11582818093A2158381809335
:105CC000A3158FEF9FEFAFEFBFEF8093A4159093D5
:105CD000A515A093A615B093A71585E58093B615D5
:105CE0008AEA8093B71581E00F900F900F900F9084
:105CF000CF91DF910895CF92DF92EF92FF920F93B1
:105D00001F9380910316833041F46FEF7FEF8FEF85
:105D10009FEF8EDF882309F441C1809173168F3F76
:105D200079F421E082E090E0A0E0B0E08093681692
:105D300090936916A0936A16B0936B16022F14C045
:105D40008091701690917116A0917216B091731691
:105D50000196A11DB11D8093681690936916A093BA
:105D60006A16B0936B1601E08FEF9FEF90930A16BF
:105D700080930916109279161092781610E0BFEFF2
:105D8000CB2EBFEFDB2EBFEFEB2EBFE0FB2EE4C030
:105D900080E00E942F20882309F400C180916C16B6
:105DA00090916D16A0916E16B0916F160097A10597
:105DB000B10509F0A5C08091681690916916A0916F
:105DC0006A16B0916B1680936C1690936D16A09323
:105DD0006E16B0936F16113089F40197A109B109BD
:105DE0008093681690936916A0936A16B0936B1609
:105DF00081E00E942F208823E1F5D0C080917316A6
:105E00008F3F39F18091701690917116A0917216A2
:105E1000B09173160097A105B10569F4809103163E
:105E2000833009F0B5C08091CA159091CB15A0912F
:105E3000CC15B091CD158093681690936916A093F8
:105E40006A16B0936B1681E00E942F20882309F414
:105E5000A5C080916C1690916D16A0916E16B091B0
:105E60006F168093701690937116A0937216B0936C
:105E7000731680916C1690916D16A0916E16B0916C
:105E80006F168093681690936916A0936A16B09364
:105E90006B16C0926C16D0926D16E0926E16F09250
:105EA0006F1681E00E942F20882309F477C020918B
:105EB0007416309175164091761650917716809130
:105EC000B91590E0A0E0B0E082179307A407B507EA
:105ED00048F0109274161092751610927616109261
:105EE00077165AC0281B390B4A0B5B0B209374168C
:105EF00030937516409376165093771611E019C0BB
:105F0000113009F449C00023A1F0809168169091E6
:105F10006916A0916A16B0916B168C509E4FAF4FC8
:105F2000BF4F8093681690936916A0936A16B0933A
:105F30006B168091681690916916A0916A16B091BF
:105F40006B160196A11DB11D80936816909369167A
:105F5000A0936A16B0936B1620916816309169165B
:105F600040916A1650916B168091BE159091BF15A5
:105F7000A091C015B091C115281739074A075B07D2
:105F800008F406CF112341F420E0002309F0CACE23
:105F90008BE18093061602C0DFD901C080E01F911B
:105FA0000F91FF90EF90DF90CF900895AF92BF9246
:105FB000CF92DF92FF920F931F93F82E1092051647
:105FC00010920416182F00E081E0A82EB12CC12CED
:105FD000D12C0E94BB248823B1F4809106168A310B
:105FE000B9F5A0927416B0927516C0927616D0923A
:105FF000771681DE882319F4002301F129C057D9CF
:10600000882339F725C00E94E81DFC018081882380
:1060100021F4115011F481E01CC08091041690917C
:10602000051601969093051680930416892B89F620
:10603000002321F08BE1809306160AC02BDB882316
:1060400039F010920516109204161F2D01E0C1CFF1
:1060500080E01F910F91FF90DF90CF90BF90AF90A5
:106060000895FF920F931F93CF93DF93EC0195DB7D
:10607000182F882309F43CC0CE01B8DC082F8823F0
:1060800021F48AE28093061633C0812F8FDF8823A4
:1060900079F1CE0160E070E0402F20E0B4DBF82E13
:1060A000012F015011E016C0809104169091051641
:1060B000019790930516809304160E94BB248823B1
:1060C000B9F0101709F4105CCE016F2D412F44DA9E
:1060D0002D961F5F011740F78091041690910516C9
:1060E000800F911D909305168093041681E001C0E6
:1060F00080E0DF91CF911F910F91FF900895DF9382
:10610000CF9300D0CDB7DEB7882369F081E090E06F
:10611000A0E0B0E080937C1390937D13A0937E1356
:10612000B0937F1308C010927C1310927D131092CD
:106130007E1310927F1380E00E948B1F882311F43E
:1061400090E0A5C00E94081E0E94801F8BE192E093
:1061500068EB73E14DE10E94C70785E58093B615B2
:106160008AEA8093B7158091B9158093C5139091F1
:106170007B16990F990F80917A1682958695869550
:106180008370980F9093D21380910316833029F473
:1061900088E392E068EF73E104C088E392E06CED7D
:1061A00073E14AE10E94C7078091BA159091BB152F
:1061B0009A83898320910316FE0131962330E1F4FE
:1061C00080E28093C61389818093DC138181809360
:1061D000DD1382E08093E41381E08093E81383E38E
:1061E00080930D1482E380930E148FE190E09093DE
:1061F000BD158093BC1523C081E08093C61382E057
:106200008093CA1389818093CE1381818093CF13A9
:1062100081E38093F113213011F482E301C086E31E
:106220008093F21380917A1690917B16A0917C1640
:10623000B0917D168F5F9F4FA040B04098F0809145
:106240007A168093D81380917B168093D91380910E
:106250007C168093DA1380917D168093DB132330B4
:1062600049F40AC080917A168093CB1380917B16F3
:106270008093CC1391E00BC06FEF7FEF8FEF9FEF18
:10628000D7DC90E0882309F491E081E09827892FFA
:106290000F900F90CF91DF910895DF93CF9300D0AF
:1062A00000D0CDB7DEB72091BC153091BD1540E0D0
:1062B00050E08091C2159091C315A091C415B09182
:1062C000C515821B930BA40BB50B80937C13909385
:1062D0007D13A0937E13B0937F1381E00E948B1FE8
:1062E000882379F18091B615853559F58091B715D8
:1062F0008A3A39F588EB93E162E572E044E050E0D8
:106300000E94CE07892BE9F48CE995E166E572E0FD
:1063100044E050E00E94CE07892B99F4FE013196AB
:106320008091A01589838091A11581838091A21508
:1063300082838091A315838329813A814B815C817B
:1063400004C02FEF3FEF4FEF5FEFB901CA010F908D
:106350000F900F900F90CF91DF910895EF92FF92E1
:106360000F931F9382E090E0A0E0B0E08093681666
:1063700090936916A0936A16B0936B1680910316DA
:10638000813009F044C0EE24FF2487012AC080E058
:106390000E942F20882309F4A3C080916C1690914D
:1063A0006D16A0916E16B0916F160097A105B105FC
:1063B00029F40894E11CF11C011D111D809168163F
:1063C00090916916A0916A16B0916B160196A11D65
:1063D000B11D8093681690936916A0936A16B093C6
:1063E0006B16209168163091691640916A1650918B
:1063F0006B168091BE159091BF15A091C015B091FC
:10640000C115281739074A075B0708F25DC08330BA
:1064100069F443DF7B018C018FEFE8168FEFF806FC
:106420008FEF08078FEF180709F04EC080E00E9439
:106430002F20882309F454C0EE24FF24870128C0AC
:1064400080916C1690916D16A0916E16B0916F169A
:106450000097A105B10529F40894E11CF11C011D68
:10646000111D0E94E21F8823D9F180916816909136
:106470006916A0916A16B0916B160196A11DB11D07
:106480008093681690936916A0936A16B0936B1662
:10649000209168163091691640916A1650916B16DA
:1064A0008091BE159091BF15A091C015B091C115F6
:1064B000281739074A075B0718F2809103168330C3
:1064C00019F4B701C801B4DB2091B91530E040E000
:1064D00050E0C801B7010E94137E9B01AC0104C0CB
:1064E00020E030E040E050E0B901CA011F910F9177
:1064F000FF90EF900895EF92FF920F931F93CF9329
:10650000DF9380910316813059F428DF2091B9156B
:1065100030E040E050E00E94527ECA01B901C5C09F
:1065200082E090E0A0E0B0E0809368169093691656
:10653000A0936A16B0936B1680E00E942F208823E8
:1065400009F4C4C080910316833009F04BC0A5DE66
:106550007B018C018FEFE8168FEFF8068FEF0807AD
:106560008FEF180709F09FC0C091BA15D091BB15E5
:10657000EE24FF24870128E030E02EC080818823AC
:1065800041F482E090E0A0E0B0E0E80EF91E0A1FBE
:106590001B1F285F3F4F389692E02030390770F379
:1065A00080917C1390917D13A0917E13B0917F1305
:1065B0000196A11DB11D80937C1390937D13A09330
:1065C0007E13B0937F1381E00E948B1F882309F410
:1065D0007DC0219720E030E0209739F0F901E854A0
:1065E000FC4ECCCFEE24FF2487018091031682302D
:1065F000D1F5C091BA15D091BB1524E030E02DC083
:106600008081882341F482E090E0A0E0B0E0E80ED1
:10661000F91E0A1F1B1F2C5F3F4F349692E020305B
:10662000390770F380917C1390917D13A0917E13B4
:10663000B0917F130196A11DB11D80937C1390939F
:106640007D13A0937E13B0937F1381E00E948B1F74
:106650008823E1F1219720E030E0209721F0F90133
:10666000E854FC4ECDCF8091BE159091BF15A091FE
:10667000C015B091C1158E159F05A007B10710F484
:1066800024E625C08E199F09A00BB10B892F9A2FE4
:10669000AB2FBB278E159F05A007B10720F4E81A82
:1066A000F90A0A0B1B0BC801B70124E630E040E0F1
:1066B00050E00E94137E2091BE153091BF1540918D
:1066C000C0155091C1150E94527E01C020E0822F5A
:1066D000DF91CF911F910F91FF90EF9008950F934D
:1066E0001F93082F8091B8156AE776E10E94344124
:1066F00007FD02C011E015C00F7780917A169091C6
:106700007B16A0917C16B0917D160196A11DB11D3E
:1067100080937A1690937B16A0937C16B0937D1687
:1067200010E0802F612F0E94DD278823A1F0112324
:1067300021F00E94462A882371F0812FE0DC882313
:1067400051F0812FA0D9882331F014DA882319F071
:106750000E94581F01C080E01F910F9108952F9251
:106760003F924F925F926F927F928F929F92AF92E1
:10677000BF92CF92DF92EF92FF920F931F93DF931E
:10678000CF93CDB7DEB72A970FB6F894DEBF0FBE12
:10679000CDBF1092D0151092D1151092D215109233
:1067A000D3150E94401C1092031610927C13109275
:1067B0007D1310927E1310927F130E94112788235D
:1067C00009F4B5C1BCE7CB2EB3E1DB2E81E00E941A
:1067D0008B1F882309F4ABC18091B615853531F044
:1067E0008091B7158A3A11F082E06FC060907C13F7
:1067F00070907D1380907E1390907F1361147104CC
:106800008104910409F053C0A6E7B5E1E0E08C9162
:10681000803811F0882379F414968C911497813084
:1068200079F0843069F0863059F08E3049F08B3041
:1068300039F08C3029F0EF5F5096E43041F737C0E3
:10684000F0E0A4E0EE0FFF1FAA95E1F7E854FC4E3C
:10685000EA53FE4F819180937C138191D60111966A
:106860008C931197819112968C9312978081139635
:106870008C93E0907C13F0907D1300917E13109127
:106880007F138091B8150E942D4190E0A0E0B0E008
:10689000BC01CD01A80197010E94137E60937C1377
:1068A00070937D1380937E1390937F138FCF80918D
:1068B000B8138B3E49F48091BA13803929F4809142
:1068C000CD13807F803F21F083E0809306162FC197
:1068D00084E0809306163090C41336948091C513DB
:1068E000389E202C11242092B9157E010894E11CB9
:1068F000F11C8091CE1389838091CF13F70181839E
:1069000089819A81892B81F48091DC13898380911C
:10691000DD1381838091DE13882309F008C1809103
:10692000DF13882309F003C1032D10E089819A81C8
:10693000089F2001099F500C189F500C1124509261
:10694000BB154092BA159091CB13992399F480917D
:10695000CC13882379F4FE0133968091D8138B836E
:106960008091D91381838091DA1382838091DB1324
:10697000838308C0FE0133969B838091CC1381836F
:10698000128213826B817C818D819E816F837887D7
:1069900089879A87C201880F991F9093CB1580939E
:1069A000CA158091C913D7018C938091CA1311968F
:1069B0008C93432D50E0CA0164E0880F991F6A95BB
:1069C000E1F729813A81820F931F55E0880F991FC3
:1069D0005A95E1F7440F019760E0742F0E943E7EC4
:1069E000609FA001619F500D709F500D1124509326
:1069F000CD154093CC158091C613F701808380910B
:106A0000C713818329813A818091E813B901681BFA
:106A10007109609FC001619F900D709F900D1124BE
:106A20009093BD158093BC15029FC001039F900DEC
:106A3000129F900D11245C01CC24DD246A0C7B1C78
:106A40008C1C9D1C6092C2157092C3158092C41557
:106A50009092C5157A0100E010E0C201A0E0B0E01C
:106A6000880F991FAA1FBB1FE80EF91E0A1F1B1FC4
:106A7000E092C615F092C7150093C8151093C9157A
:106A8000222009F454C0632D70E080E090E02F8153
:106A9000388549855A850E94137E6A197B098C09BD
:106AA0009D096E197F09800B910B05C096958795FE
:106AB000779567952694A1E02A16C1F76E5F7F4F00
:106AC0008F4F9F4F6093BE157093BF158093C01575
:106AD0009093C1156250704080409040653FBFE088
:106AE0007B07B0E08B07B0E09B0718F420920316F9
:106AF00008C0655F7F4F8040904028F482E080931B
:106B0000031681E015C083E0809303168091E4139F
:106B10008093CA158091E5138093CB158091E6137D
:106B20008093CC158091E7138093CD15EACF80E058
:106B30002A960FB6F894DEBF0FBECDBFCF91DF917E
:106B40001F910F91FF90EF90DF90CF90BF90AF908B
:106B50009F908F907F906F905F904F903F902F907D
:106B600008958091B8150895DF93CF93CDB7DEB720
:106B700027970FB6F894DEBF0FBECDBF2091B81592
:106B80003091D0159091D1154091D2155091D315D7
:106B900070910416809105167E838F833A839B83C0
:106BA0004C835D83492F5C816D8190E027960FB601
:106BB000F894DEBF0FBECDBFCF91DF9108956091F5
:106BC0008713709188138091891390918A13089587
:106BD000CF93DF93EC010E949C27882359F00E94F9
:106BE000BB24882339F0CE010E94CC1B882319F0E6
:106BF00081E001C080E0DF91CF9108950C94391CB1
:106C00000895AF92BF92CF92DF92EF92FF920F93CF
:106C10001F93CF93DF938C01C62EB42EA22E0E9419
:106C20009C27882309F463C081E0B81619F4CC20AE
:106C300009F45EC0C0910416D0910516209719F48E
:106C4000DD24D39407C02197D0930516C093041672
:106C50002196DD24EE24FF2402C0DD24D3940E947B
:106C6000BB24882309F443C0DD2031F0C8016C2D1A
:106C70004B2D0E949D1C3CC0C8016C2D4B2D2A2D14
:106C80000E94111D882389F080910716882339F00E
:106C9000F801808191818E0D9F1D91838083D09317
:106CA0000516C093041681E023C08091061680313A
:106CB00039F0D0930516C09304168B3071F217C0CB
:106CC00080910716882329F08DE090E0E80EF91EE8
:106CD00004C0035F1F4F93EFC90E8091041690917B
:106CE000051601979093051680930416B8CF80E09F
:106CF000DF91CF911F910F91FF90EF90DF90CF9098
:106D0000BF90AF9008958F929F92AF92BF92CF9213
:106D1000DF92EF92FF920F931F93CF93DF93EC01DB
:106D2000062F0E94D827882309F490C0C09004162B
:106D3000D0900516E090D415F090D5159090DA1506
:106D400010E088248394AA24AA94BA2C013011F06C
:106D5000112361F080910416909105162FEF8E3F5C
:106D6000920711F488E00BC0019619C080910416B7
:106D7000909105162FEF8F3F920721F489E08093C1
:106D8000061659C0009751F48091DA158823B1F3A3
:106D90008091DB15882391F711E005C0019790934E
:106DA0000516809304160E94BB24882329F4809141
:106DB00006168A3111F13FC08091DA150E94A01B9E
:106DC0008823D9F0112311F6013031F48091D415C4
:106DD0009091D515019605C08091D4159091D51547
:106DE00001979093D5158093D415209721F40E9494
:106DF000041C81E02BC02197A9CF809106168A3010
:106E000019F08A3109F0A2CF112321F01092DA157E
:106E100010E09CCF8091DA15813009F4AFCF8091DA
:106E2000DB15882309F0AACFB0920516A0920416AC
:106E30008092DA158BCF9092DA15D0920516C09217
:106E40000416F092D515E092D41580E0DF91CF9131
:106E50001F910F91FF90EF90DF90CF90BF90AF9078
:106E60009F908F9008951F93CF93DF93EC01162F7F
:106E700080E090E061E047DF882341F0CE0160E0F0
:106E800040E0212FBEDE882399F381E0DF91CF918E
:106E90001F9108950E94D827882319F00E94401C52
:106EA00081E00895CF93DF93EC01F4DF882371F143
:106EB000CE0160E0D8DF882321F08AE280930616B5
:106EC00025C0CE01CED8882309F1109283131092E9
:106ED00084131092851310928613109287131092C8
:106EE00088131092891310928A1310928213809142
:106EF000D4159091D51501969093D5158093D415FE
:106F000081E08093DA150E94581F01C080E0DF9174
:106F1000CF910895EF92FF920F931F930E94D8276D
:106F2000882309F454C08091D0159091D115A09177
:106F3000D215B091D3150097A105B10511F489E1DF
:106F400044C081E090E090930516809304160E945F
:106F5000BB248823E1F10E94041CE090D015F0903E
:106F6000D1150091D2151091D31580918313909172
:106F70008413A0918513B09186138093D0159093BC
:106F8000D115A093D215B093D31584DF8823F9F0DF
:106F90008091DB15882391F08091DA15882371F0B8
:106FA00018C08091831390918413A0918513B091A0
:106FB00086138E159F05A007B10759F080E090E079
:106FC00061E0A1DE882369F788E08093061680E0FF
:106FD00001C081E01F910F91FF90EF9008952F92D3
:106FE0003F924F925F926F927F928F929F92AF9259
:106FF000BF92CF92DF92EF92FF920F931F93DF9396
:10700000CF9300D000D0CDB7DEB79C838B836A834B
:107010000E94D827882309F492C0E090D015F09000
:10702000D1150091D2151091D315E114F104010589
:10703000110509F45AC020900416309005162091CD
:10704000821329836090831370908413809085133A
:1070500090908613A0908713B0908813C0908913E6
:10706000D0908A135090DB154090DA1581E0809320
:10707000DB158093DA154EDF882329F45092DB1557
:107080004092DA155DC05092DB154092DA1580917E
:10709000CE159091CF1590930516809304168B8191
:1070A0009C816A8141E020E0ACDD3092051620929F
:1070B0000416E092D015F092D1150093D2151093DA
:1070C000D3153981309382136092831370928413A5
:1070D0008092851390928613A0928713B0928813A2
:1070E000C0928913D0928A132BC0809107168823EF
:1070F00039F083E090E0EB81FC819183808316C0BE
:1071000090E0992331F0913011F080E009C08AE3DA
:1071100007C08091B8158F3F11F488E501C08F5BDF
:10712000EB81FC8180839F5F933011F481E008C084
:107130002B813C812F5F3F4F3C832B83E2CF80E04C
:107140000F900F900F900F90CF91DF911F910F91A3
:10715000FF90EF90DF90CF90BF90AF909F908F9077
:107160007F906F905F904F903F902F9008950E9476
:10717000C727882309F10E94391C8823E9F08091F0
:107180000416909105169093CF158093CE1580919B
:10719000831390918413A0918513B09186138093EB
:1071A000D0159093D115A093D215B093D31572DE5C
:1071B000882319F081E0089580E008950F931F93CC
:1071C000082F0E94C7278823D9F434C080E090E0BC
:1071D00061E099DD882331F0002399F08DE18093FF
:1071E000061628C097DE882329F181E00E94032B30
:1071F000882301F1112311F481E01DC01150E6CF65
:107200001FEF0E94391C882329F0B1DF882391F0F9
:107210001F5FDCCF81E00E942D1E882359F081E0A2
:107220000E94032B882331F01F3F81F633DE0E943A
:10723000581F01C080E01F910F9108951F93182FD0
:1072400029DE882339F410C08091DA15181711F45B
:1072500081E00AC080E090E061E055DD8823A1F77D
:1072600089E08093061680E01F910895DF92EF92E7
:10727000FF920F931F93CF93DF93D82EE090D415F6
:10728000F090D51507DE882319F4C0E0D0E01FC0C8
:1072900000E010E0C0E0D0E008C08091DA15813055
:1072A00011F4219602C00F5F1F4F80E090E061E073
:1072B0002ADD882391F7EEDD8FEFE8168FEFF806D1
:1072C00019F0C70161E01FDD81E0D812E801CE01AD
:1072D000DF91CF911F910F91FF90EF90DF90089574
:1072E0001F93CF93DF93182FC1DFEC01009729F490
:1072F00089E08093061680E00DC0812F9FDF8823F0
:1073000049F0C130D10511F481E004C0CE010297EB
:1073100061E0F9DCDF91CF911F9108956F927F9228
:107320008F929F92AF92BF92CF92DF92EF92FF9295
:107330000F931F93CF93DF93EC010E94C7278823FD
:1073400009F44AC081E00E942D1E882309F444C03C
:1073500080900416909005166090DA157090821354
:10736000A0908313B0908413C0908513D09086139F
:10737000E0908713F09088130091891310918A137D
:10738000CE0190DD882341F10E94BB24882321F1A6
:1073900070928213A0928313B0928413C0928513CB
:1073A000D0928613E0928713F0928813009389138A
:1073B00010938A130E94651C909205168092041601
:1073C00080E00E94032B882339F00E94581F8823F5
:1073D00019F0862D85DF01C080E0DF91CF911F91EC
:1073E0000F91FF90EF90DF90CF90BF90AF909F9064
:1073F0008F907F906F900895CF93DF93EC010E9460
:10740000D827882309F449C0CE014CDD882309F42C
:1074100044C08FEF8093731681E090E0A0E0B0E06D
:107420008093741690937516A0937616B093771682
:107430000E947B2E882329F40E94032B0E94581F50
:107440002CC08091701690917116A0917216B09117
:1074500073168093831390938413A0938513B09332
:10746000861310928713109288131092891310922A
:107470008A1380E1809382130E940E2A882369F088
:107480000E94BB24882349F00E94651C0E94581F5B
:10749000882319F080E024DF01C080E0DF91CF91E4
:1074A00008950E94112780910316882329F420E073
:1074B00030E040E050E011C06091B91570E080E02C
:1074C00090E02091BE153091BF154091C0155091AC
:1074D000C1150E94137E9B01AC01B901CA01089538
:1074E0000E94112780910316882309F004C808958B
:1074F0000E94112780910316882329F420E030E0B0
:1075000040E050E004C00E94AE319B01AC01B901E3
:10751000CA0108950E947827882389F08091031674
:10752000882361F01092D0151092D1151092D215C7
:107530001092D3150E94401C81E0089510C908954F
:107540000E94112780910316882309F4E3DF8091BC
:10755000031608951F93182F0E947827882351F04F
:107560000E940C1E882331F0812FB9D8882311F096
:10757000F6D801C080E01F9108951F93182F0E9434
:107580007827882389F07FD6181728F086E0809323
:10759000061680E009C08091B815811721F010937C
:1075A000B8151092031681E01F910895CF93DF93D1
:1075B000EC018881E2DF882331F1ACDF882319F107
:1075C00089819A81AB81BC818093D0159093D1152C
:1075D000A093D215B093D3155DDC882349F413C072
:1075E00080E090E061E08FDB882311F453DC0BC076
:1075F00020910416309105168D819E812817390738
:1076000079F781E001C080E0DF91CF910895BF92CA
:10761000CF92DF92EF92FF920F931F93DF93CF935E
:10762000CDB7DEB727970FB6F894DEBF0FBECDBF3C
:107630008C01B62EC42E0E947827882309F4A2C09C
:107640006091B8152091D0153091D1154091D21587
:107650005091D31580910416909105169F838E83C7
:107660002A833B834C835D836983F80180818C3559
:1076700011F08F3239F44EDF882309F47FC00F5F99
:107680001F4F42C0F80191819A33B1F422812C3509
:1076900011F02F3289F4992787FD90950E94747E0E
:1076A00081546BDF882309F469C034DF882309F42F
:1076B00065C00D5F1F4F28C08E3299F49C3511F0C4
:1076C0009F3279F40E5F1F4F1FC024DC882309F41A
:1076D00055C0F7018081882319F00894E11CF11C42
:1076E0008701F80180818E3279F481818E3261F4D4
:1076F00062E0E62EF12CE00EF11E82818C3529F33A
:107700008F3219F3882309F3C5DB8823B9F1EE24FE
:10771000FF24DD2402C0DD24D394F8018081882376
:1077200011F481E02FC0C8016B2D9DDB882329F463
:10773000CC2021F17801DD24D3940F5F1F4FF80195
:107740008081882339F4DD2041F3C701ABDB882336
:1077500011F714C08C3511F08F3279F7DD2021F04C
:10776000C7014ADE882351F00E94391C882331F07A
:10777000FEDC882319F00F5F1F4FCFCFCE0101969B
:1077800015DF80E027960FB6F894DEBF0FBECDBFA1
:10779000CF91DF911F910F91FF90EF90DF90CF90ED
:1077A000BF90089570C5089590918C16981749F070
:1077B000882319F4992329F0892F0E94921E81E0D1
:1077C000089580E008950E94391C882329F084E2FE
:1077D0008093061680E0089582E0E6DF81E0089558
:1077E0001F93182F833028F087E28093061680E0DD
:1077F0000CC080918C16811739F00E94D81E812F01
:107800000E94D81E10938C1681E01F910895BF929C
:10781000CF92DF92EF92FF920F931F93CF93DF935C
:10782000982FB0908C1680917B028F3F19F4DD2445
:10783000D394F7C0992309F001C18E3F39F083D466
:10784000009721F0039709F0F9C0F6C080917B0200
:107850007DD480918A1690918B16892B09F05DC09A
:1078600082E0BEDF44D1882319F0F2E0DF2E0FC0A2
:107870008FEF9FEF90938B1680938A1685E896E1A1
:107880002FD3882319F4DD24D39401C0DD248B2D5C
:10789000A7DFDD2009F09FC080918A1690918B169A
:1078A00090938416809383168EE796E1D6D1882331
:1078B00009F4C4C020918A1630918B1680918316EA
:1078C000909184168217930740F582E089DF6091DA
:1078D0008A1670918B162091831630918416621B44
:1078E000730B80E090E0E9E0660F771F881F991F17
:1078F000EA95D1F742E01AD1882311F4DD24D3941C
:107900008B2D6EDF809183169091841690938B1649
:1079100080938A16DD2009F05EC0C0918A16D0914E
:107920008B1688E0C030D80710F0C0E0D8E0409156
:107930008616509187166091881670918916E0908E
:107940007F16F0908016009181161091821680911A
:10795000851620917E166E0110D480937B02DD2463
:107960008F3F11F4DD24D3949E0140E050E08091DC
:10797000861690918716A0918816B0918916820F6D
:10798000931FA41FB51F8093861690938716A0930C
:107990008816B093891680917F1690918016A091D9
:1079A0008116B0918216280F391F4A1F5B1F209342
:1079B0007F163093801640938116509382168091E3
:1079C0008A1690918B168C1B9D0B90938B1680932F
:1079D0008A16DD2031F180917B02B8D38FEF80933E
:1079E0007B0282E0FDDEE0908713F0908813009127
:1079F000891310918A131ED18B2DF2DE82E0D816E6
:107A000059F4C801B70140E091D0882319F0FDD1A5
:107A1000882311F4DD24D3940DD181E0D81609F424
:107A2000CDDB8D2DDF91CF911F910F91FF90EF90C6
:107A3000DF90CF90BF900895DD24F3CFDD24D39461
:107A4000CACF0F931F939C0180917B028F3F21F03F
:107A500085E2809306161EC0C90124DA8823D1F07E
:107A60008FE010D38823B1F000918C1682E0B8DE4D
:107A700089E008D3182F802FB3DE112311F4DAD058
:107A800009C08EEF80937B0210928B1610928A169B
:107A900081E001C080E01F910F91089580E0A0DE99
:107AA000C9D081E09DDEC6D082E09ADEC3D00C94BE
:107AB000581F0F931F9310920716109291130E9454
:107AC000F61D0E94A81910E00FEF812F89DE109299
:107AD00003160093B815109280131092DB151F5FE8
:107AE000133099F710928C161F910F9108950E94F0
:107AF000AD27882311F46FEF17C060E02091871342
:107B0000309188134091891350918A1380918B137F
:107B100090918C13A0918D13B0918E1382179307BF
:107B2000A407B50708F061E0862F0895EF92FF9251
:107B30000F931F93DF93CF930F92CDB7DEB77B01E7
:107B40008C0149830E94AD279981882309F46AC07A
:107B5000913039F1913078F0923021F0933009F082
:107B600060C039C080918B1390918C13A0918D13BC
:107B7000B0918E131EC08091871390918813A091AD
:107B80008913B0918A138E159F05A007B107E0F104
:107B9000E0928B13F0928C1300938D1310938E133D
:107BA00040C08091871390918813A0918913B09160
:107BB0008A138E159F05A007B10730F18E199F0912
:107BC000A00BB10B80938B1390938C13A0938D1308
:107BD000B0938E1326C020918B1330918C1340915B
:107BE0008D1350918E132E0D3F1D401F511F8091FC
:107BF000871390918813A0918913B0918A138217EB
:107C00009307A407B50728F487E08093061680E061
:107C100009C020938B1330938C1340938D13509392
:107C20008E1381E00F90CF91DF911F910F91FF9004
:107C3000EF9008950E94AD27882371F08091801302
:107C400081FF08C00E94BB24882331F00E94651C7C
:107C50000E94581F109280130895CF93DF93EC0178
:107C60000E94AD27882309F47DC08091801381FD97
:107C700004C085E18093061675C04D815E8160E089
:107C800070E081E00E940B26882309F46BC08D818F
:107C90009E810097C1F09C0140E050E080917416F5
:107CA00090917516A0917616B0917716281739071E
:107CB0004A075B0740F4209374163093751640937F
:107CC0007616509377162091741630917516409160
:107CD00076165091771689E0220F331F441F551FE7
:107CE0008A95D1F780918B1390918C13A0918D136D
:107CF000B0918E13280F391F4A1F5B1F20938B13DF
:107D000030938C1340938D1350938E13809187136F
:107D100090918813A0918913B0918A1382179307C9
:107D2000A407B50740F4209387133093881340933A
:107D3000891350938A138091B815888380917016A7
:107D400090917116A0917216B091731689839A83DF
:107D5000AB83BC8380917416909175169E838D833E
:107D600081E001C080E0DF91CF9108951F93182F2B
:107D70000E94AD27882309F445C08091801381FDBE
:107D800004C085E1809306163DC082E041E050E0EA
:107D900060E070E00E940B268823A1F10E94081E7B
:107DA00080918B1390918C13A0918D13B0918E13B1
:107DB000FC01F170E854FC4E10839C01AD012F5F73
:107DC0003F4F4F4F5F4F20938B1330938C13409353
:107DD0008D1350938E138091871390918813A091E7
:107DE0008913B0918A1382179307A407B50740F44B
:107DF00020938713309388134093891350938A13E9
:107E000081E001C080E01F9108950E94AD27882382
:107E100001F18091801381FD05C085E180930616F4
:107E200080E0089580918B1390918C13A0918D1315
:107E3000B0918E138093871390938813A093891326
:107E4000B0938A1383E00E944525882311F00C9497
:107E5000581F80E008958091801380FD02C08EE15C
:107E60001FC020918713309188134091891350913E
:107E70008A1380918B1390918C13A0918D13B091E4
:107E80008E1382179307A407B50748F482E00E9477
:107E90004525882351F4809106168A3119F480E231
:107EA000809306162FEF3FEF19C080918B139091AE
:107EB0008C13A0918D13B0918E13FC01F170E854D6
:107EC000FC4E208130E00196A11DB11D80938B13E3
:107ED00090938C13A0938D13B0938E13C9010895C2
:107EE000AF92BF92CF92DF92EF92FF920F931F93C8
:107EF000CF93DF93EC010E94AD27882309F4B6C02D
:107F00008091801380FD02C08EE10EC0F0DD8823D9
:107F100051F481E00E944525882349F4809106169A
:107F20008A3109F0A3C080E2809306169FC06D815C
:107F30007E8161157105D9F09B0140E050E0809190
:107F4000741690917516A0917616B0917716281731
:107F500039074A075B0758F4E82FE61B209374168D
:107F600030937516409376165093771601C0E0E073
:107F7000A0907416B0907516C0907616D0907716B3
:107F80008601750149E0EE0CFF1C001F111F4A9588
:107F9000D1F780918B1390918C13A0918D13B09198
:107FA0008E13E80EF91E0A1F1B1FE0928B13F0922E
:107FB0008C1300938D1310938E132091871330919F
:107FC00088134091891350918A132E153F0540075D
:107FD0005107A8F5809188138695317040705070D4
:107FE000211531054105510509F08F5F2091B91523
:107FF000622F0E94327E822F891B821709F480E053
:10800000282F2E1BA21AB108C108D108A0927416FD
:10801000B0927516C0927616D0927716922F990F5D
:1080200080E0A0E0B0E0E81AF90A0A0B1B0BE0922E
:108030008B13F0928C1300938D1310938E138091F9
:10804000B81588838091701690917116A091721660
:10805000B091731689839A83AB83BC838091741625
:10806000909175169E838D8381E001C080E0DF9141
:10807000CF911F910F91FF90EF90DF90CF90BF9025
:10808000AF9008950F931F93082F0E94C72788234E
:1080900009F44AC00E945519882309F445C0102FDD
:1080A00001FF14C081E00E942D1E8823E9F1809118
:1080B000821380FF02C085E106C08091B815C6D04A
:1080C000882349F084E1809306162EC080E00E9448
:1080D0002D1E882349F112FF08C0109287131092B9
:1080E00088131092891310928A1313FF09C01092FB
:1080F0008B1310928C1310928D1310928E1310C04C
:108100008091871390918813A0918913B0918A135D
:1081100080938B1390938C13A0938D13B0938E1335
:108120000093801381E001C080E01F910F910895BA
:1081300080E00895882319F02EEE30E002C028ED8B
:1081400030E0C901089580E090E0089580E090E07B
:108150000895882329F4CB01BA01A9010C94DF0802
:1081600081500C94B511882329F4CB01BA01A901DF
:108170000C94EB0881500C9443126F927F928F9273
:108180009F92AF92BF92CF92DF92EF92FF920F93A6
:108190001F93CF93DF93682E4A015B01722E0E94DA
:1081A000581FC1E0D0E01FC0862DB501A40128EB07
:1081B00033E1D9DFEC010097C9F4872DB801A7019D
:1081C00028EB33E1C6DFEC01009781F40894811CB1
:1081D000911CA11CB11C0894E11CF11C011D111D76
:1081E0000894C108D108C114D104F1F60E94F61D0B
:1081F000CD2B11F480E001C08FEFDF91CF911F9163
:108200000F91FF90EF90DF90CF90BF90AF909F9035
:108210008F907F906F900895882319F021E030E0CF
:1082200006C0CB01BA01A9010E942A099C01C9011B
:108230000895882319F021E030E006C0CB01BA018F
:10824000A9010E94F7089C01C9010895882311F42F
:108250000C94DC0881500C94340F882311F481E0D5
:10826000089581500C94A117882319F4CB010C9424
:108270001E0981500C944815882311F40C940909A7
:1082800081500C9405170E94CD0E8F5F0895809148
:10829000B3072091B4078217B9F0222331F4843058
:1082A00099F08F5F8093B30706C090E0019630E0AD
:1082B0008217930749F08091B3078F5F8093B307CC
:1082C000853011F41092B30708954091B3072091BF
:1082D000B407442331F4243009F184E08093B307D8
:1082E0000AC0842F90E0019730E082179307B1F025
:1082F00041504093B3078091B30790E0FC0135E013
:10830000EE0FFF1F3A95E1F7880F991FE81BF90B55
:10831000E954F84F8081882309F4B9CF0895AC015E
:10832000FC0120E08081882321F02F5F31962E31DF
:10833000C9F7FA01E20FF11D829131968C3519F0DF
:108340008CE5808311820895CF93DF93FC01EC01CB
:10835000849107C0992787FD90950E949307FE019D
:10836000849121968823B1F7DF91CF910895809170
:108370006B19882329F08091F0178850823018F407
:1083800088E69BE0E1CF00D08CE792E0EDB7FEB746
:10839000928381830E94007F0F900F9008958091B7
:1083A0006B19882329F08091F0178850823018F4D7
:1083B00088E69BE0C9DF81E080936C1908951F93E4
:1083C0008091C910882321F488E69BE0BDDF3BC083
:1083D00084E08093F11713E01093F2171092F317D3
:1083E00081E28093551981E08093561910925819B3
:1083F0001092571910925A191092591983E090E06F
:1084000090935C1980935B1910925D1981EF97E14D
:108410000E94C46081EA80935519109356191092F6
:1084200058191092571910925A191092591986E03A
:1084300090E090935C1980935B1910925D1981EF25
:1084400097E10E94C4601F9108958091C91088230C
:1084500019F488E69BE035C08BE698E061E040E0E7
:10846000D6D8882319F48FED92E02BC084E0809356
:10847000F1171092F2178FEF8093F31781E2809338
:10848000551981E080935619109258191092571976
:1084900010925A191092591983E090E090935C1948
:1084A00080935B1910925D1981EF97E10E94C4607F
:1084B0000E94CA79882319F480EB9BE002C08BEA02
:1084C0009BE042CF8091C910882319F488E69BE095
:1084D0003BCF84E08093F1171092F2178FEF8093D7
:1084E000F31781E28093551981E080935619109219
:1084F00058191092571910925A191092591983E06D
:1085000090E090935C1980935B1910925D1981EF54
:1085100097E10C94C4608091F017863019F088E6DA
:108520009BE012DF81E08093B8108093F0170C94E9
:1085300098638091F0178850823018F088E69BE0AD
:1085400003DF81E08093B71008958091F0178630A3
:1085500019F088E69BE0F8DE88E08093F017089534
:1085600083E593E0F1CE80916B08882369F08BE678
:1085700098E0D5DE8BE698E061E040E048D88823BB
:1085800019F48FED92E0E0CE0895EF92FF920F93F1
:108590001F93CF93DF938091B207882309F4F7C329
:1085A00020E00AC0A35BB74FEC938E2F81548A3131
:1085B00010F4E05EEC932F5FA22FB0E08091B4073F
:1085C00090E0FC0105E0EE0FFF1F0A95E1F7880F30
:1085D000991FE81BF90BEA0FFB1FE954F84FE081E4
:1085E000E03221F08091B2078217E0F6422FA35BC0
:1085F000B74F1C92122F115020E030E0F42EF3946C
:10860000EE248091B40790E0FC01B5E0EE0FFF1F6F
:10861000BA95E1F7880F991FE81BF90BEF0DF11DD3
:10862000E954F84F8081823219F4EE24E394F394F4
:1086300000E0C901880F991FE90175E0CC0FDD1F2B
:108640007A95E1F7C81BD90B19C0DE01A00FB11D47
:10865000A559B74F8091B40790E0FC0165E0EE0F9B
:10866000FF1F6A95E1F7880F991FE81BF90BE40FCC
:10867000F11DE954F84F80818C930F5F402F4F0D0F
:108680005091B407642F70E0EE20A1F4852F90E0A4
:10869000FC01A5E0EE0FFF1FAA95E1F7880F991FD7
:1086A000E81BF90BE60FF71FE954F84F8081803281
:1086B000A1F41AC0852F90E0FC01B5E0EE0FFF1F7A
:1086C000BA95E1F7880F991FE81BF90BE60FF71F22
:1086D000E954F84F8081823231F08091B2078417DB
:1086E00008F0B3CFE1104F5FC901880F991FF9015E
:1086F00055E0EE0FFF1F5A95E1F7E81BF90BE00F6D
:10870000F11DE559F74F10822F5F3F4F22303105A1
:1087100009F074CF1092B2078091B4078F5F8093F5
:10872000B407853011F41092B4078091B407809398
:10873000B307ADE4B8E040E050E0FA01E65BFE4F7D
:10874000E4918C91992787FD90952E2F30E0821728
:10875000930741F44F5F5F4F141710F481E01BC380
:108760001196EBCFADE4B8E040E050E0FA01E45EF2
:10877000FE4FE4918C91992787FD90952E2F30E044
:108780008217930741F44F5F5F4F141710F482E094
:1087900002C31196EBCFADE4B8E040E050E0FA013F
:1087A000EF59FE4FE4918C91992787FD90952E2FDC
:1087B00030E08217930741F44F5F5F4F141710F4B6
:1087C00083E0E9C21196EBCFADE4B8E040E050E0C1
:1087D000FA01EB5FFE4FE4918C91992787FD90950C
:1087E0002E2F30E08217930731F44F5F5F4F14173D
:1087F00068F01196EDCF80914E088A3349F480914C
:108800004D0880936B0880E380936C0884E0C3C2BA
:10881000ADE4B8E040E050E0FA01E15EFE4FE491E3
:108820008C91992787FD90952E2F30E08217930722
:1088300041F44F5F5F4F141710F485E0ACC21196FE
:10884000EBCFADE4B8E040E050E0FA01E25FFE4F6C
:10885000E4918C91992787FD90952E2F30E0821717
:10886000930741F44F5F5F4F141710F486E093C2F3
:108870001196EBCFADE4B8E040E050E0FA01EF5ED6
:10888000FE4FE4918C91992787FD90952E2F30E033
:108890008217930741F44F5F5F4F141710F487E07E
:1088A0007AC21196EBCFADE4B8E040E050E0FA01B7
:1088B000EE5FFE4FE4918C91992787FD90952E2FC6
:1088C00030E08217930741F44F5F5F4F141710F4A5
:1088D00088E061C21196EBCFADE4B8E040E050E033
:1088E000FA01EB5BFE4FE4918C91992787FD9095FF
:1088F0002E2F30E08217930741F44F5F5F4F14171C
:1089000010F489E048C21196EBCFADE4B8E040E046
:1089100050E0FA01E85CFE4FE4918C91992787FDC5
:1089200090952E2F30E08217930741F44F5F5F4FF1
:10893000141710F48AE02FC21196EBCFADE4B8E023
:1089400040E050E0FA01E45CFE4FE4918C919927FD
:1089500087FD90952E2F30E08217930741F44F5FEB
:108960005F4F141710F48BE016C21196EBCFADE4F5
:10897000B8E040E050E0FA01E45AFE4FE4918C91F7
:10898000992787FD90952E2F30E08217930741F4A9
:108990004F5F5F4F141710F48CE0FDC11196EBCFC1
:1089A000ADE4B8E040E050E0FA01EB5DFE4FE49149
:1089B0008C91992787FD90952E2F30E08217930791
:1089C00041F44F5F5F4F141710F48DE0E4C111962E
:1089D000EBCFADE4B8E040E050E0FA01E55DFE4FDA
:1089E000E4918C91992787FD90952E2F30E0821786
:1089F000930741F44F5F5F4F141710F48EE0CBC123
:108A00001196EBCFADE4B8E040E050E0FA01E75E4C
:108A1000FE4FE4918C91992787FD90952E2F30E0A1
:108A20008217930741F44F5F5F4F141710F48FE0E4
:108A3000B2C11196EBCFADE4B8E040E050E0FA01EE
:108A4000EF5CFE4FE4918C91992787FD90952E2F36
:108A500030E08217930741F44F5F5F4F141710F413
:108A600080E199C11196EBCFADE4B8E040E050E071
:108A7000FA01E15BFE4FE4918C91992787FD909577
:108A80002E2F30E08217930741F44F5F5F4F14178A
:108A900010F481E180C11196EBCFADE4B8E040E085
:108AA00050E0FA01EC5AFE4FE4918C91992787FD32
:108AB00090952E2F30E08217930741F44F5F5F4F60
:108AC000141710F482E167C11196EBCFADE4B8E062
:108AD00040E050E0FA01E55FFE4FE4918C91992768
:108AE00087FD90952E2F30E08217930741F44F5F5A
:108AF0005F4F141710F483E14EC11196EBCFADE434
:108B0000B8E040E050E0FA01E75AFE4FE4918C9162
:108B1000992787FD90952E2F30E08217930741F417
:108B20004F5F5F4F141710F484E135C11196EBCFFE
:108B3000ADE4B8E040E050E0FA01E859FE4FE491BE
:108B40008C91992787FD90952E2F30E082179307FF
:108B500041F44F5F5F4F141710F485E11CC111966B
:108B6000EBCFADE4B8E040E050E0FA01E359FE4F4E
:108B7000E4918C91992787FD90952E2F30E08217F4
:108B8000930741F44F5F5F4F141710F486E103C160
:108B90001196EBCFADE4B8E040E050E0FA01EE58BA
:108BA000FE4FE4918C91992787FD90952E2F30E010
:108BB0008217930741F44F5F5F4F141710F487E15A
:108BC000EAC01196EBCFADE4B8E040E050E0FA0126
:108BD000E758FE4FE4918C91992787FD90952E2FB1
:108BE00030E08217930741F44F5F5F4F141710F482
:108BF00088E1D1C01196EBCFADE4B8E040E050E0A1
:108C0000FA01E158FE4FE4918C91992787FD9095E8
:108C10002E2F30E08217930741F44F5F5F4F1417F8
:108C200010F489E1B8C01196EBCFADE4B8E040E0B4
:108C300050E0FA01E957FE4FE4918C91992787FDA6
:108C400090952E2F30E08217930741F44F5F5F4FCE
:108C5000141710F48AE19FC01196EBCFADE4B8E091
:108C600040E050E0FA01E257FE4FE4918C919927E1
:108C700087FD90952E2F30E08217930741F44F5FC8
:108C80005F4F141710F48BE186C01196EBCFADE463
:108C9000B8E040E050E0FA01E856FE4FE4918C91D4
:108CA000992787FD90952E2F30E08217930741F486
:108CB0004F5F5F4F141710F48CE16DC01196EBCF2E
:108CC000ADE4B8E040E050E0FA01EE55FE4FE4912B
:108CD0008C91992787FD90952E2F30E0821793076E
:108CE00041F44F5F5F4F141710F48DE154C011969B
:108CF000EBCFADE4B8E040E050E0FA01E555FE4FBF
:108D0000E4918C91992787FD90952E2F30E0821762
:108D1000930741F44F5F5F4F141710F48EE13BC08F
:108D20001196EBCFADE4B8E040E050E0FA01EB542F
:108D3000FE4FE4918C91992787FD90952E2F30E07E
:108D40008217930741F44F5F5F4F141710F48FE1C0
:108D500022C01196EBCFADE4B8E040E050E0FA015C
:108D6000E354FE4FE4918C91992787FD90952E2F27
:108D700030E08217930741F44F5F5F4F141710F4F0
:108D800080E209C01196EBCF8EEE92E0DDDA82ED43
:108D900091E0DADA80E0DF91CF911F910F91FF909F
:108DA000EF9008952F923F924F925F926F927F9231
:108DB0008F929F92AF92BF92CF92DF92EF92FF92EB
:108DC0000F931F93CF93DF939091F017963041F05C
:108DD000892F8850823020F088E69BE0B5DA3DC2CA
:108DE0009850923018F482E39CE0AEDAA090B5106F
:108DF000BB24EAE4EE2EF12C75E1472E512C66E9F6
:108E0000662E63E0762E50E9852E53E0952E4BE9D1
:108E1000242E43E0342E1AC2B092B5108B2D90E070
:108E20008E9DF0018F9DF00D9E9DF00D1124EF544D
:108E3000F94E21812093A10000D000D000D0EDB7E1
:108E4000FEB7319645EB52E0ADB7BEB712965C93D4
:108E50004E931197019693838283248315820E94F7
:108E6000007F8091B51090E0ADB7BEB711962CECA5
:108E700032E0EDB7FEB7328321838E9DF0018F9DE6
:108E8000F00D9E9DF00D1124EF54F94E80859185D3
:108E900013969C938E9312978681978115969C9337
:108EA0008E9314970E94007F0F900F90E1EEF2E0F6
:108EB000ADB7BEB71296FC93EE9311978091B510A3
:108EC00090E08E9DF0018F9DF00D9E9DF00D112480
:108ED000EF54F94E838590E0880F991F14969C9368
:108EE0008E9313970E94007F8091B51090E08E9D25
:108EF000F0018F9DF00D9E9DF00D1124EF54F94E61
:108F000082850F900F900F900F9086FF03C081E035
:108F10009CE002C08AE19CE017DA00D000D0ADB737
:108F2000BEB7119624EF32E0EDB7FEB7328321834E
:108F30008091B51090E025E230E0829FF001839FA0
:108F4000F00D929FF00D1124EE0FFF1FED54F94E1E
:108F5000808112968C93129713961C920E94007F28
:108F60008091D9000F900F900F900F9083FF03C056
:108F700086E49CE002C08DE59CE0E6D98091B510C6
:108F800090E08E9DF0018F9DF00D9E9DF00D1124BF
:108F9000EF54F94E828585FF03C087EB9BE002C04A
:108FA00088ED9BE0D1D900D000D0ADB7BEB7119607
:108FB00023E133E0EDB7FEB7328321838091B51012
:108FC00090E08E9DF0018F9DF00D9E9DF00D11247F
:108FD000EF54F94E858112968C93129713961C923A
:108FE0000E94007F00E00F900F900F900F901CC127
:108FF000C02EDD244DB75EB74C5050400FB6F894EC
:109000005EBF0FBE4DBFADB7BEB7119641E353E093
:10901000EDB7FEB752834183C49CE001C59CD00DDF
:10902000D49CD00D1124F901EC0FFD1FEF54F94E23
:10903000848512968C93129713961C9213978585AC
:1090400014968C93149715961C9215978685978580
:1090500017969C938E9316978089918919969C9365
:109060008E931897828993891B969C938E931A9757
:109070000E94007F8DB79EB70A960FB6F8949EBFE8
:109080000FBE8DBFEDE7F3E0ADB7BEB71296FC9310
:10909000EE9311970E94007F8091B51090E08E9D15
:1090A000F0018F9DF00D9E9DF00D1124EC0FFD1F22
:1090B000EF54F94E0F900F9084898823B9F110E096
:1090C00022C000D000D0EDB7FEB73196ADB7BEB725
:1090D00012969C928E921197A12FB0E0AA0FBB1FFF
:1090E000AA0FBB1FAC0FBD1FA20FB31FAF54B94EC9
:1090F00055968C91828313820E94007F1F5F0F9090
:109100000F900F900F908091B51090E08E9D900180
:109110008F9D300D9E9D300D1124FE01E20FF31F37
:10912000EF54F94E8489181760F209C000D0EDB7EA
:10913000FEB7728261820E94007F0F900F908DE0D7
:1091400090E00E9493078AE090E00E94930700D08D
:10915000ADB7BEB712963C922E9211970E94007F37
:109160008091B51090E0C49C9001C59C300DD49CBA
:10917000300D11248E9DF0018F9DF00D9E9DF00D00
:109180001124E20FF31FEF54F94E0F900F908489D2
:109190008823C1F110E0E90122C000D000D0EDB772
:1091A000FEB73196ADB7BEB712969C928E921197CC
:1091B000A12FB0E0AA0FBB1FAA0FBB1FAC0FBD1F92
:1091C000A20FB31FAF54B94E56968C91828313826F
:1091D0000E94007F1F5F0F900F900F900F90809163
:1091E000B51090E08E9D90018F9D300D9E9D300DAD
:1091F0001124FE01E20FF31FEF54F94E8489181772
:1092000060F209C000D0EDB7FEB7728261820E94A1
:10921000007F0F900F908DE090E00E9493078AE00E
:1092200090E00E9493070F5F8091B51090E08E9DB3
:1092300090018F9D300D9E9D300D1124F901EF544A
:10924000F94E8581081708F4D3CEB3948091B116F6
:10925000B81608F4E1CDA092B510DF91CF911F911F
:109260000F91FF90EF90DF90CF90BF90AF909F90C5
:109270008F907F906F905F904F903F902F900895C8
:10928000EF92FF921F93DF93CF93CDB7DEB72E9768
:109290000FB6F894DEBF0FBECDBF80916B08882358
:1092A00009F442C00E94B435288739874A875B8712
:1092B0006C877D878E87DE011196FE01389687E0E8
:1092C00001900D928150E1F710E07E010894E11CBD
:1092D000F11CC7010E94D63A8BE698E061E040E0BD
:1092E0000E94073B882359F080E00E94DE388823E3
:1092F00021F480EB9BE028D802C01F5FEACF00D0AA
:1093000000D0EDB7FEB731968EEA93E0ADB7BEB7A9
:1093100012969C938E931197128313820E94007F62
:109320000F900F900F900F902E960FB6F894DEBF0F
:109330000FBECDBFCF91DF911F91FF90EF900895A9
:109340003F924F925F926F927F928F929F92AF92D5
:10935000BF92CF92DF92EF92FF920F931F93DF9312
:10936000CF93CDB7DEB727970FB6F894DEBF0FBE09
:10937000CDBF382E802F0983C12E1A83D22E2B8386
:10938000E32E3C83F42E4D83052F5E83162F6F83CF
:10939000582E0E94581F0E94F61D809180008C7FDD
:1093A0008093800080918100877E809381008091EE
:1093B0008100887F856080938100B09A109285003B
:1093C00010928400980159019601A701C901DA01A0
:1093D0006C017D018824992466247724A4E04A2E18
:1093E0005A943FC0D701C60183709070A070B070CE
:1093F0000097A105B10511F414E004C08C2D837011
:10940000142D181B812F90E0A816B90608F41A2D08
:10941000332049F0852DB701A6012EEA38E0012F4F
:109420000E94151108C0852DB701A6012EEA38E06B
:10943000012F0E94B113892B29F083EC93E00E9445
:10944000117F59C0B09911C00E9416083C01812FAC
:1094500090E0A81AB90A880E991EC10ED11CE11C11
:10946000F11CA114B10409F0BDCFB40180E090E07B
:1094700028EE33E040E050E00E94137E7B018C0137
:10948000B30180E090E0FBE0660F771F881F991F13
:10949000FA95D1F720E43FE140E050E00E94527E8F
:1094A000C801B7010E94527E332049F000D000D09D
:1094B00000D0EDB7FEB7319684ED93E008C000D040
:1094C00000D000D0EDB7FEB7319686EF93E0ADB790
:1094D000BEB712969C938E93119722833383448355
:1094E00055830E94007F8DB79EB706960FB6F894FD
:1094F0009EBF0FBE8DBF27960FB6F894DEBF0FBE7E
:10950000CDBFCF91DF911F910F91FF90EF90DF9032
:10951000CF90BF90AF909F908F907F906F905F9013
:109520004F903F9008956F927F928F929F92AF924B
:10953000BF92CF92DF92EF92FF920F931F93DF9330
:10954000CF93CDB7DEB727970FB6F894DEBF0FBE27
:10955000CDBF682E09831A832B833C834D835E83A2
:109560006F83702EEA80FB800C811D818E809F802E
:109570000E94581F0E94F61D809180008C7F80936E
:10958000800080918100877E80938100809181009E
:10959000887F856080938100B09A10928500109238
:1095A0008400CC24DD24AA24BB2425C0662041F0FD
:1095B000872DB801A70128EB33E10E94A94007C01D
:1095C000872DB801A70128EB33E10E94B340892B16
:1095D00029F083EC93E00E94117F56C00894E11CAF
:1095E000F11C011D111DB09909C00E9416085C01F3
:1095F0000894C11CD11CC814D904C0F2B60180E083
:1096000090E028EE33E040E050E00E94137E7B01C2
:109610008C01B50180E090E0BBE0660F771F881FEA
:10962000991FBA95D1F720E43FE140E050E00E9455
:10963000527EC801B7010E94527E662049F000D0D8
:1096400000D000D0EDB7FEB7319684ED93E008C0AE
:1096500000D000D000D0EDB7FEB7319686EF93E092
:10966000ADB7BEB712969C938E9311972283338326
:10967000448355830E94007F8DB79EB706960FB630
:10968000F8949EBF0FBE8DBF27960FB6F894DEBF2D
:109690000FBECDBFCF91DF911F910F91FF90EF9043
:1096A000DF90CF90BF90AF909F908F907F906F9002
:1096B00008952F923F924F925F926F927F928F9276
:1096C0009F92AF92BF92CF92DF92EF92FF920F9351
:1096D0001F93DF93CF93CDB7DEB764970FB6F8949F
:1096E000DEBF0FBECDBF29833A834B835C836D837E
:1096F0007E838F83A886B986CA86DB86EC86FD8644
:109700000E872C8B2A813B814C815D81288B398B84
:109710004A8B5B8BAF8629843A844B845C8480912E
:1097200080008C7F8093800080918100877E809371
:10973000810080918100887F8560809381008D8584
:109740009E856E807F808615970508F43C0142E077
:10975000A42EB12C81C0B09A109285001092840082
:109760008C89488959896A897B892F858201710191
:1097700065010E94BD40182F8F3F51F0812F0E943C
:10978000A34083309105D1F3009729F00197B1F7F9
:1097900083EC93E00CC00E9416084C01B09B0AC0F9
:1097A00031E0A316B10409F05BC087E194E00E94A8
:1097B000117F56C04DB75EB7485050400FB6F89471
:1097C0005EBF0FBE4DBFCDB6DEB60894C11CD11C26
:1097D0002BE234E0EDB7FEB732832183B50180E0A0
:1097E00090E028EE33E040E050E00E94137E7B01E1
:1097F0008C01B40180E090E03BE0660F771F881F8A
:10980000991F3A95D1F720E43FE140E050E00E94F3
:10981000527EC801B7010E94527EF6012283338333
:1098200044835583C50196958795978386830E94C7
:10983000007FC501880F991F13E0AA0CBB1C1A9565
:10984000E1F7A80EB91E2DB73EB7285F3F4F0FB600
:10985000F8943EBF0FBE2DBF6A147B0408F07BCF87
:1098600064960FB6F894DEBF0FBECDBFCF91DF91E7
:109870001F910F91FF90EF90DF90CF90BF90AF902E
:109880009F908F907F906F905F904F903F902F9020
:10989000089580916B08882321F08BE698E00C9462
:1098A00052370895EF92FF920F931F93DF93CF9358
:1098B000CDB7DEB72E970FB6F894DEBF0FBECDBF83
:1098C0007B011F821E820E94BD3A882351F4DE0173
:1098D0001896FE01319687E001900D928150E1F7D4
:1098E0005FC00E948A3A882351F4DE011896FE0177
:1098F000319687E001900D928150E1F751C089E5E2
:1099000094E00E945237882309F5809106168A3226
:1099100051F0DE011896FE01319687E001900D921C
:109920008150E1F73DC080E00E94DE3889E594E097
:109930000E945237882351F4DE011896FE013196B9
:1099400087E001900D928150E1F72AC08EE00E94DD
:1099500042408E010F5F1F4F882359F40E94DE386A
:10996000DE011896F80187E001900D928150E1F731
:1099700017C0FF82EE82C8010E942D3E882339F471
:109980001F821E820E941A3E80E00E94DE38DE01A5
:109990001896FE01319687E001900D928150E1F713
:1099A000288539854A855B856C857D858E8590E027
:1099B0002E960FB6F894DEBF0FBECDBFCF91DF91CC
:1099C0001F910F91FF90EF900895AF92BF92CF92A9
:1099D000DF92EF92FF920F931F93DF93CF93CDB758
:1099E000DEB7A3970FB6F894DEBF0FBECDBF809150
:1099F0006B08882309F4E7C00E94B4352E8B3F8B97
:109A0000488F598F6A8F7B8F8C8FDE011196FE01F4
:109A1000769687E001900D928150E1F700D081E6C3
:109A200094E0EDB7FEB7928381830E94007F0F9090
:109A30000F9080916B08815660E078E033DF2D8FC6
:109A40003E8F4F8F58A369A37AA38BA3DE0118968C
:109A5000FE017D9687E001900D928150E1F78D85A2
:109A60009E85892B21F400D080E894E02DC0809160
:109A70008908882309F467C082E00E94F03B809146
:109A80008908815660E078E00DDF2D8F3E8F4F8F83
:109A900058A369A37AA38BA3DE011F96FE017D96CE
:109AA00087E001900D928150E1F78C899D89892B87
:109AB000C1F480E00E94F03B0E941A3E80E00E94C8
:109AC000DE3800D082EA94E0EDB7FEB7928381835E
:109AD0000E94007F0F900F90CE0101960E94D63A0F
:109AE00072C084EC94E00E94117F288539854A85F4
:109AF0005B856C857D858E85AF84B888C988DA885A
:109B0000EB88FC880D89D5DD8EEE94E00E94117FF4
:109B10002F85388949895A896B897C898D89A884E0
:109B2000B984CA84DB84EC84FD840E85C2DD82E0C6
:109B30000E94F03B0E941A3E80E00E94DE3880E0E6
:109B40000E94F03B2CC080E0088519852A853B8562
:109B50004C855D856E85E7DC81E0088519852A8561
:109B60003B854C855D856E85DEDC0E94B1358823A2
:109B7000B1F088E195E00E94117F80E008851985A9
:109B80002A853B854C855D856E85DADB81E008851D
:109B900019852A853B854C855D856E85D1DB0E94C4
:109BA0001A3E80E00E94DE38CE0101960E94D63A2D
:109BB00000D087E395E0EDB7FEB7928381830E94E2
:109BC000007F0F900F90A3960FB6F894DEBF0FBEE4
:109BD000CDBFCF91DF911F910F91FF90EF90DF905C
:109BE000CF90BF90AF90089580916B08882351F07B
:109BF0008BE698E00E94FC39882321F480EB9BE0FF
:109C00000C94A44108954F925F926F927F928F922D
:109C10009F92AF92BF92CF92DF92EF92FF921F93EB
:109C2000DF93CF93CDB7DEB72E970FB6F894DEBF94
:109C30000FBECDBF80916B08882309F447C1809186
:109C40008908882309F442C1ABE6EA2EA8E0FA2E7F
:109C5000C7010E948F41C7014E960E948F4100D0DC
:109C600085E495E0EDB7FEB7928381830E94007F83
:109C70000F900F900E94B435288739874A875B87F9
:109C80006C877D878E87DE011196FE01389687E00E
:109C900001900D928150E1F782E00E94F03B00D0EC
:109CA0008CE595E0EDB7FEB7928381830E94007F3B
:109CB0000F900F908BE698E061E040E00E94073B38
:109CC000882309F4DDC00E944A3780E00E94F03BFF
:109CD00000D086E795E0EDB7FEB7928381830E94BE
:109CE000007F0F900F9089E898E061E041E00E94CA
:109CF000073B882309F4C4C00E944A3710E0F5E905
:109D00004F2EF5E05F2EE0EC6E2EE5E07E2E7DEB33
:109D1000C72E75E0D72E69ED862E65E0962E54EAA3
:109D2000A52E55E0B52E01C0115082E00E94F03BF7
:109D300080E090E061E00E9483368823C9F411231B
:109D400009F4B0C000D0EDB7FEB7528241820E9444
:109D5000007F0F900F900E948A37882309F490C0EB
:109D600080E00E94F03B0E948A378823E9F688C091
:109D70000E94FE358823D9F100D0EDB7FEB7B2823C
:109D8000A1820E94007F0F900F908BE698E06EE119
:109D900041E020E00E940136882309F471C00E944E
:109DA000B738882309F46CC080E00E94F03B00D0F3
:109DB000EDB7FEB7F282E1820E94007FEDB7FEB7F9
:109DC000D282C1820E94007F0F900F90C7010E9433
:109DD000FC39882329F4809106168A3209F050C094
:109DE0000E94B738882309F44BC01F5F9ECF00D074
:109DF000EDB7FEB7728261820E94007F0F900F90D4
:109E00008BE698E06EE141E020E00E940136882375
:109E1000B9F100D0EDB7FEB7F282E1820E94007F77
:109E2000EDB7FEB7D282C1820E94007F0F900F90E3
:109E30000E94E33B882321F180E00E94F03B12C0A6
:109E4000809106168A32E1F400D0EDB7FEB7928217
:109E500081820E94007F0F900F9081E00E94DE3887
:109E6000882371F08BE698E00E94213D882341F31E
:109E700080E00E94073C8823D9F3823009F455CF53
:109E800080E00E94F03BCE0101960E94D63A00D0BD
:109E90008EEF95E0EDB7FEB7928381830E94007F3D
:109EA00080E011C080E00E94F03BCE0101960E944C
:109EB000D63A00D08DE096E0EDB7FEB7928381836D
:109EC0000E94007F81E00F900F9001C080E02E96ED
:109ED0000FB6F894DEBF0FBECDBFCF91DF911F91BB
:109EE000FF90EF90DF90CF90BF90AF909F908F90BA
:109EF0007F906F905F904F900895DF93CF93CDB791
:109F0000DEB72E970FB6F894DEBF0FBECDBF80919F
:109F10006B08882309F458C00E94B4352887398714
:109F20004A875B876C877D878E87DE011196FE01ED
:109F3000389687E001900D928150E1F78BE698E02A
:109F400061E040E00E94073B882329F48FED92E016
:109F50000E94A44139C08BE698E06EE141E021E027
:109F60000E9401360E94E33B882319F480EB9BE0BA
:109F700025C080918908882339F487EA98E00E94F7
:109F8000D63A8823E9F00BC089E898E061E040E028
:109F90000E94073B882319F48FED92E00FC08BE6F7
:109FA00098E00E94213D882339F080E00E94073C20
:109FB0008823D9F3813021F485EC91E00E94A441FB
:109FC000CE0101960E94D63A2E960FB6F894DEBFC7
:109FD0000FBECDBFCF91DF91089580916B0888238C
:109FE000D1F0809189088823B1F08BE698E061E098
:109FF00040E00E94073B882321F48FED92E00C940F
:10A00000A44189E898E00E948E39882321F480EBEE
:10A010009BE00C94A44108951F9300D08BE196E03F
:10A02000EDB7FEB7928381830E94007F0F900F905F
:10A030000E949C07182F813711F08032C9F700D099
:10A0400081E396E0EDB7FEB7928381830E94007FA3
:10A0500080E00F900F90103209F481E01F91089575
:10A060001F9380916B088823D1F18BE698E061E023
:10A0700040E00E94073B882319F48FED92E007C06F
:10A0800082E00E944240882329F480EB9BE00E94FA
:10A09000A44125C081E193E00E94A4410E949C0755
:10A0A000182F813191F0992787FD90950E94930791
:10A0B000812F0E94B63E1D3089F78AE090E00E9411
:10A0C00093078AE00E94B63EE9CF0E941A3E8DE0D7
:10A0D00090E00E9493078AE090E00E9493071F910E
:10A0E0000895FF920F931F93F82E80916B08882399
:10A0F00099F18BE698E061E040E00E94073B8823FD
:10A1000029F48FED92E00E94A44126C089E00E94CC
:10A11000424000E013C0FF2031F0043120F07CDF2A
:10A12000882381F000E00E942B3F182F992787FD9C
:10A1300090950E9493071A3009F40F5F0E94773DB3
:10A14000882349F30E941A3E8DE090E00E94930715
:10A150008AE090E00E9493071F910F91FF9008956D
:10A160002F923F924F925F926F927F928F929F9227
:10A17000AF92BF92CF92DF92EF92FF920F931F9315
:10A18000DF93CF93CDB7DEB76E970FB6F894DEBFEF
:10A190000FBECDBF882E0E94B13500D000D025E47F
:10A1A00036E0ADB7BEB712963C932E93119790E070
:10A1B0008F599F4F14969C938E9313970E94007F04
:10A1C0000F900F900F900F900E94B1350E949A400F
:10A1D0000E94A44100D084E596E0EDB7FEB79283DB
:10A1E00081830E94007F0F900F900E94A03A8230DE
:10A1F00041F0833071F0813021F500D082E696E0A5
:10A200000BC000D08AE696E0EDB7FEB7928381835B
:10A2100009C000D082E796E0ADB7BEB712969C9316
:10A220008E9311970E94007F0F900F905E0108940B
:10A23000A11CB11CC5016EE10E94EF37882391F487
:10A2400005C08AE796E00E94117FE9C000D085E949
:10A2500096E0EDB7FEB7928381830E94007F0F9056
:10A260000F9014C000D000D086EA96E0ADB7BEB71C
:10A2700012969C938E9311971496BC92AE9213975C
:10A280000E94007F0F900F900F900F9080916B08AD
:10A29000882389F08A3279F480916C088E3259F4DF
:10A2A000EBE6F8E082818193B8E0E738FB07D1F76D
:10A2B0009924939401C0992400D087EB96E0EDB7E0
:10A2C000FEB7928381830E94007F0F900F900E94BF
:10A2D0004A3700E010E0EE24FF24CC24DD241E01E8
:10A2E0000894211C311C83ED482E86E0582EBEECCC
:10A2F0006B2EB6E07B2E6BC09920D9F40E94FE3500
:10A30000882369F000D0ADB7BEB712967C926E92EA
:10A3100011970E94007F0894E11CF11C07C000D037
:10A32000EDB7FEB7528241820E94007F0F900F90DE
:10A330000CC00E94FE35882309F049C08BE698E0E6
:10A340000E94E835882309F442C00F5F1F4F882020
:10A3500091F0C80164E170E00E943E7E892B59F4BF
:10A360000115110541F0C016D10629F055DE8823EC
:10A3700009F455C06801C5016EE141E021E00E9489
:10A3800001360E94DF352DB73EB7285030400FB65A
:10A39000F8943EBF0FBE2DBFEDB7FEB7319628ED46
:10A3A00036E0ADB7BEB712963C932E9311976283F9
:10A3B000738384839583378226820E94007F8DB7C2
:10A3C0009EB708960FB6F8949EBF0FBE8DBF80E073
:10A3D00090E061E00E948336882309F08DCF00D0A1
:10A3E00000D084EE96E0ADB7BEB712969C938E93E4
:10A3F00011970E191F0914961C930E9313970E9420
:10A40000007F81EF96E0EDB7FEB792838183F482FF
:10A41000E3820E94007F0F900F900F900F906E9636
:10A420000FB6F894DEBF0FBECDBFCF91DF911F9165
:10A430000F91FF90EF90DF90CF90BF90AF909F90E3
:10A440008F907F906F905F904F903F902F900895E6
:10A450000E94B1350E949A400E94A44180E290E09F
:10A460000E9493070E94B13590E08F599F4F0E9440
:10A4700093070E94513A9B01AC01EBE0569547953A
:10A4800037952795EA95D1F7777080709070605076
:10A4900074408040904020F02F5F3F4F4F4F5F4F00
:10A4A00000D000D000D08CEF96E0EDB7FEB79283DD
:10A4B000818323833483458356830E94007F8DB735
:10A4C0009EB706960FB6F8949EBF0FBE8DBF089537
:10A4D0001F93DF93CF93CDB7DEB72E970FB6F894C7
:10A4E000DEBF0FBECDBF80916B08882371F1182F9E
:10A4F00011560E94D23B181728F089E892E00E947A
:10A50000A44123C00E94B435288739874A875B87D6
:10A510006C877D878E87DE011196FE01389687E075
:10A5200001900D928150E1F7812F0E94BD3A88235E
:10A5300021F00E948A3A882341F481E792E00E9448
:10A54000A441CE0101960E94D63A2E960FB6F894F9
:10A55000DEBF0FBECDBFCF91DF911F9108951F9336
:10A560008EE097E00E94117F10E01CC0812F90E0E8
:10A570008F599F4F0E9493078AE390E00E949307B0
:10A5800080E290E00E949307812F0E949A400E94EF
:10A59000A4418DE090E00E9493078AE090E00E9441
:10A5A00093071F5F0E94D23B181700F31F91089575
:10A5B00080916B08882361F081560E94BD3A81E04A
:10A5C0000E94AA3A882321F482E093E00C94A441EB
:10A5D00008956F927F928F929F92AF92BF92DF9277
:10A5E000EF92FF920F931F93DF93CF93CDB7DEB718
:10A5F0002E970FB6F894DEBF0FBECDBF0E94B435C4
:10A60000288739874A875B876C877D878E87DE013D
:10A610001196FE01389687E001900D928150E1F786
:10A62000DD248DEB682E85E0782E01E5802E07E095
:10A63000902E1BE2A12E17E0B12E70C08D2D0E942E
:10A64000BD3A0E948A3A882309F467C08D2D90E0B4
:10A650008F599F4F0E9493078AE390E00E949307CF
:10A6600080E290E00E9493078D2D0E949A400E9404
:10A67000A44100D0ADB7BEB712967C926E921197EE
:10A680000E94007F0F900F9080916B088C3681F5AF
:10A690000E94783A7B018C010E94513AEDB7FEB7D7
:10A6A0003A970FB6F894FEBF0FBEEDBF3196ADB727
:10A6B000BEB71296BC92AE92119716950795F79475
:10A6C000E794E282F38204831583969587957795C4
:10A6D000679566837783808791870E94007FEDB7B7
:10A6E000FEB73A960FB6F894FEBF0FBEEDBF15C089
:10A6F0000E94703A00D000D0EDB7FEB73196ADB7EA
:10A70000BEB712969C928E921197828313820E94FA
:10A71000007F0F900F900F900F90D3940E94D23B28
:10A72000D81608F48BCFCE0101960E94D63A2E9609
:10A730000FB6F894DEBF0FBECDBFCF91DF911F9152
:10A740000F91FF90EF90DF90BF90AF909F908F9010
:10A750007F906F9008951092B20734C060918F1966
:10A7600070919019992787FD90950E94D47E209131
:10A77000B207422F50E08091B40790E0DC01E5E0A1
:10A78000AA0FBB1FEA95E1F7880F991FA81BB90B09
:10A79000A40FB51FA954B84F8091B30790E0FC01F6
:10A7A00065E0EE0FFF1F6A95E1F7880F991FE81B20
:10A7B000F90BE40FF51FE954F84F80818C932F5F5C
:10A7C0002093B2078091B207282F30E08091B30721
:10A7D00090E0FC0175E0EE0FFF1F7A95E1F7880F1E
:10A7E000991FE81BF90BE20FF31FE954F84F808122
:10A7F000882309F0B3CF8091B40790E0FC0155E0C5
:10A80000EE0FFF1F5A95E1F7880F991FE81BF90B10
:10A81000E20FF31FE954F84F108208951DC06091B4
:10A820008F197091901988E090E00E94D47E609119
:10A830008F197091901980E290E00E94D47E60910F
:10A840008F197091901988E090E00E94D47E8091D9
:10A85000B20781508093B2078091B2078823F9F63E
:10A8600008951F930E947A07882309F485C00E94E7
:10A870009C07182F8091B507882349F0813021F477
:10A880001B3511F482E032C01092B50775C01B3140
:10A8900061F11C3134F4183061F11D3009F047C00A
:10A8A00006C01132D9F1143209F041C03BC08DE02D
:10A8B00090E00E9493078AE090E00E9493078091C5
:10A8C000B2072091B40730E0F90195E0EE0FFF1FC9
:10A8D0009A95E1F7220F331FE21BF30BE80FF11DEE
:10A8E000E954F84F108281E048C081E08093B507B9
:10A8F00043C08091B207882309F43EC088E090E00D
:10A900000E94930780E290E00E94930788E090E025
:10A910000E9493078091B20781502CC07FDF0E9474
:10A92000654103C07BDF0E94474115DF25C0812FB1
:10A9300080528F3508F58091B2078E31E9F0812F72
:10A94000992787FD90950E9493078091B2072091E7
:10A95000B40730E0F901B5E0EE0FFF1FBA95E1F75B
:10A96000220F331FE21BF30BE80FF11DE954F84FE0
:10A9700010838F5F8093B20780E01F910895DF936B
:10A98000CF93CDB7DEB727970FB6F894DEBF0FBED3
:10A99000CDBF8091B6078823B1F48091D90081FDA5
:10A9A000A3C081E08093B60785ED91E00E94A441A9
:10A9B000D6DD82ED91E00E94A4410E94593D80E0E5
:10A9C0000E94F03B0DC08091D90081FF09C0109218
:10A9D000B60785E292E00E94A4410E944E3D84C0E9
:10A9E00040DF882309F480C00E94C54290E0FC014A
:10A9F0003197E032F10508F06FC0E45BFF4FEE0FD6
:10AA0000FF1F0590F491E02D0994A9DD69C0E1DDF7
:10AA100067C0CEDD65C05CDD63C01ADD61C080E06B
:10AA200001C081E09DDB5CC00E94B34259C00E941E
:10AA30008A3756C080E001C081E053DB51C00E94DC
:10AA4000B0424EC0D1D84CC00E94494C49C00E946F
:10AA5000404946C005DB44C00E94B43529833A838F
:10AA60004B835C836D837E838F83A7EAB8E0FE010E
:10AA7000319687E001900D928150E1F731C087EA6D
:10AA800098E00E94D63A2CC038DA2AC0A6DA28C04C
:10AA9000BAD826C00E94E54C23C080E00E94390746
:10AAA000FFCF0E94D2461CC00E94A54219C00E943E
:10AAB000994216C00E948B4213C00E94624210C08D
:10AAC0000E9425420DC00E94DF410AC00E94CF4172
:10AAD00007C00E94B74104C08EEE92E00E94A441DC
:10AAE00082ED91E00E94A44127960FB6F894DEBF54
:10AAF0000FBECDBFCF91DF9108950E947E0783E9FD
:10AB000097E06CE977E00E94897E1092B607109278
:10AB1000B7071092D5071092F30710921108109200
:10AB20002F080895DF93CF93CDB7DEB762970FB6A6
:10AB3000F894DEBF0FBECDBF40919516433108F0AB
:10AB400042E180E789831A828091A2168B831C825E
:10AB50001D821E821F828AE0888719861A861B86BC
:10AB60001C868091A3168D878091A4168E871F86E0
:10AB7000188A198A1A8A9E012F5F3F4FF90103C074
:10AB800081918093F1008E2F821B8417C8F38091EE
:10AB9000E8008F778093E80080918D1690918E1653
:10ABA000A0918F16B0919016841B9109A109B1094B
:10ABB00080938D1690938E16A0938F16B093901657
:10ABC0001092A1161092A2161092A3161092A4161B
:10ABD00081E062960FB6F894DEBF0FBECDBFCF9175
:10ABE000DF9108958091921690E083709070892B88
:10ABF00021F480919316882369F081E08093A11657
:10AC000085E08093A21684E28093A3161092A41686
:10AC100080E0089590919516913608F090E620E036
:10AC2000EFE8FCE015C0283019F4E3E7FCE009C0C8
:10AC3000203119F4EBE7FCE004C0203211F4EBE81A
:10AC4000FCE084918093F1002F5F243219F031965B
:10AC5000291748F38091E8008F778093E80080916E
:10AC60008D1690918E16A0918F16B0919016821B22
:10AC70009109A109B10980938D1690938E16A09326
:10AC80008F16B09390161092A1161092A2161092E1
:10AC9000A3161092A41681E00895E1EFF0E08CE194
:10ACA00080838AE08083108285E080831082108216
:10ACB0001082108210821082108281E080830895B9
:10ACC00091E09093F1009AE09093F10020E82093B6
:10ACD000F10093E09093F1001092F1001092F100D6
:10ACE0001092F1001092F1008D3040F02093F100AD
:10ACF0001092F1001092F1001092F10008951F934C
:10AD0000182F882311F01092F1006093F100109237
:10AD1000F100809160190E942641882321F080E88B
:10AD20008093F10002C01092F100112331F01092D3
:10AD3000F1001092F1001092F1001092F1001F91B9
:10AD400008951F93282F882319F01091991602C097
:10AD5000109195168091931690E08F7390708C31BE
:10AD6000910539F08F33910581F1019709F08FC07A
:10AD700005C0822F6FE0C3DF90DF05C0822F6FE038
:10AD8000BEDF812F9DDF8091E8008F778093E80000
:10AD900080918D1690918E16A0918F16B09190167D
:10ADA0004097A109B10980938D1690938E16A093B8
:10ADB0008F16B09390161092A1161092A2161092B0
:10ADC000A3161092A41681E06EC0222359F01D3103
:10ADD00010F06BE102C0612F6250822F90DF1830BB
:10ADE00071F50BC01C3110F06BE102C0612F615096
:10ADF00080E085DF143019F511C08091E8008F776D
:10AE00008093E80080918D1690918E16A0918F16F8
:10AE1000B09190160897A109B109C5CF8091E800BB
:10AE20008F778093E80080918D1690918E16A09177
:10AE30008F16B09190160497A109B109B4CF812F54
:10AE40003FDF1D3090F029DF8091E8008F778093FD
:10AE5000E80080918D1690918E16A0918F16B0917A
:10AE600090164C97A109B1099ECF8091E8008F7789
:10AE70008093E80080918D1690918E16A0918F1688
:10AE8000B0919016811B9109A109B1098CCF81E085
:10AE90008093A11685E08093A21684E28093A31686
:10AEA0001092A41680E01F9108950F931F93DF93D3
:10AEB000CF9300D000D000D0CDB7DEB7FE013396DF
:10AEC0008091931683838091941682838091951646
:10AED0008183809196168B83809198168A838091C6
:10AEE0009916898380916119813039F48093A11674
:10AEF00085E08093A21684E294C080918D16909193
:10AF00008E16A0918F16B09190160097A105B105ED
:10AF1000C1F489819A81892B39F41092A11610927B
:10AF2000A2161092A31609C081E08093A11685E0B5
:10AF30008093A21684E28093A3161092A41681E057
:10AF40007EC0809160190E942641813039F480933F
:10AF5000A11687E08093A21687E263C04B815C81D3
:10AF60006D817E8100918D1610918E1620918F1625
:10AF700030919016E9E03695279517950795EA9553
:10AF8000D1F78091601998010E940C41823091059F
:10AF9000C9F183309105F1F1892B09F045C0298170
:10AFA0003A8140E050E080918D1690918E16A091EC
:10AFB0008F16B091901669E0B695A79597958795ED
:10AFC0006A95D1F7281739074A075B0739F41092B9
:10AFD000A1161092A2161092A31609C081E08093C8
:10AFE000A11685E08093A21684E28093A3161092A6
:10AFF000A41610928D1610928E1610928F16109223
:10B0000090169DCF81E08093A11682E08093A216D6
:10B010008AE307C081E08093A11686E08093A216A0
:10B0200088E28093A31608C081E08093A11684E093
:10B030008093A2161092A3161092A41680E0269672
:10B040000FB6F894DEBF0FBECDBFCF91DF911F9139
:10B050000F9108950F931F93DF93CF9300D000D0EB
:10B0600000D0CDB7DEB7FE0133968091931683836F
:10B070008091941682838091951681838091961693
:10B080008B83809198168A83809199168983809109
:10B090006119882341F481E08093A11685E08093B3
:10B0A000A21684E281C000918D1610918E16209117
:10B0B0008F16309190160115110521053105B9F44F
:10B0C00089819A81892B39F41092A1161092A216C7
:10B0D0001092A31609C081E08093A11685E08093A9
:10B0E000A21684E28093A3161092A4164CC04B8142
:10B0F0005C816D817E81A9E036952795179507952E
:10B10000AA95D1F78091601998010E941941823067
:10B110009105D9F18330910509F43FC0892B09F0DD
:10B1200046C029813A8140E050E080918D1690918F
:10B130008E16A0918F16B0919016F9E0B695A7954E
:10B1400097958795FA95D1F7281739074A075B072E
:10B1500039F41092A1161092A2161092A31609C0EB
:10B1600081E08093A11685E08093A21684E280930B
:10B17000A3161092A41610928D1610928E1610928D
:10B180008F161092901681E01DC081E08093A11669
:10B1900082E08093A2168AE307C081E08093A11623
:10B1A00086E08093A21688E28093A31608C081E00F
:10B1B0008093A11684E08093A2161092A316109299
:10B1C000A41680E026960FB6F894DEBF0FBECDBF62
:10B1D000CF91DF911F910F9108950F931F93DF93EC
:10B1E000CF9300D000D0CDB7DEB7809160198E012B
:10B1F0000F5F1F4FB8010E9434418230910509F45E
:10B200003FC08330910509F443C0892B09F04AC03F
:10B21000F80183818093F10082818093F100818124
:10B220008093F10080818093F1001092F1001092E0
:10B23000F10082E08093F1001092F1008091E8002B
:10B240008F778093E80080918D1690918E16A09153
:10B250008F16B09190160897A109B10980938D16A9
:10B2600090938E16A0938F16B09390161092A116FD
:10B270001092A2161092A3161092A41681E01DC07F
:10B2800081E08093A11682E08093A2168AE307C032
:10B2900081E08093A11686E08093A21688E28093D5
:10B2A000A31608C081E08093A11684E08093A216C3
:10B2B0001092A3161092A41680E00F900F900F909A
:10B2C0000F90CF91DF911F910F9108958091601998
:10B2D0000E943C418230910551F08330910579F014
:10B2E000892BB9F41092A1161092A21618C081E011
:10B2F0008093A11682E08093A2168AE307C081E0C2
:10B300008093A11686E08093A21688E28093A3160C
:10B3100008C081E08093A11684E08093A216109269
:10B32000A3161092A41681E00895809191168A3296
:10B3300021F45F9ABADD5F980895883221F45E9A0D
:10B3400089DE5E9808958B3111F18C3160F4833081
:10B35000B1F0843018F48823A1F023C0823181F049
:10B360008A31F9F410C0853269F0863218F48E31D2
:10B37000C1F40DC08F3259F08A3599F406C0D2CB92
:10B3800031CCA4CF2ACF80E001C081E0DACC10928A
:10B39000A1161092A2161092A3161092A41681E084
:10B3A000089581E08093A11685E08093A21680E243
:10B3B0008093A3161092A41680E008951F920F9216
:10B3C0000FB60F920BB60F921124EF92FF920F93CC
:10B3D0001F932F933F934F935F936F937F938F931D
:10B3E0009F93AF93BF93CF93DF93EF93FF9380919E
:10B3F000E10082FF09C08091E20082FF05C08BEF6F
:10B400008093E1000E947B778091E10080FF40C043
:10B410008091E20080FF3CC08091B2108130D9F46D
:10B420008091AD168823B9F08091E2008E7F8093E1
:10B43000E2008FEE8093E1008091E20080618093D2
:10B44000E20089B58D7F89BD19BC8091D8008062EA
:10B450008093D8001DC08FEE8093E1008091AE10E4
:10B460009091AF1080629093AF108093AE108EEFEA
:10B470008093E1008091E20080618093E2008091FE
:10B48000D80080628093D80089B58D7F89BD19BCB2
:10B490008091E10084FF27C08091E20084FF23C0F7
:10B4A00009B400FC05C08EE089BD09B400FEFDCFE3
:10B4B0008091D8008F7D8093D8008FEE8093E1003B
:10B4C0008091E2008F7E8093E2008091AE10909197
:10B4D000AF1080649093AF108093AE108091E20023
:10B4E00081608093E2008091E10085FF1AC0809125
:10B4F000E20085FF16C08091E2008F7E8093E2001B
:10B500008FED8093E1008091E2008F7D8093E200D7
:10B510008091AE109091AF1080689093AF1080939F
:10B52000AE108091E10083FF12C08091E20083FFA2
:10B530000EC087EF8093E1000E9439088091AE1021
:10B540009091AF1091609093AF108093AE10809166
:10B55000DA0081FF29C08091D80081FF25C0809149
:10B56000D90081FF02C082E001C081E08093B11068
:10B570008DEF8093DA009091B1108091A516981705
:10B5800099F08091D90081FF06C08091AE10909112
:10B59000AF10886005C08091AE109091AF108061AF
:10B5A0009093AF108093AE1080919F0081FF17C0E1
:10B5B0008091A00081FF13C00E9486088DEF8093C8
:10B5C0009F008AE08093F0178091AE109091AF10A9
:10B5D00098609093AF108093AE100E949863809112
:10B5E0009F0080FF09C08091A00080FF05C08EEF02
:10B5F00080939F000E94860880919F0085FF98C0DD
:10B600008091A00085FF94C080919F008F7D8093E2
:10B610009F008091AE109091AF1092609093AF1008
:10B620008093AE108091B0108F5F8093B0108091A6
:10B63000BA108F5F8093BA108091B0108A3F08F4DF
:10B6400075C01092B010C0E0D0E000E821E0E22E1A
:10B65000F12CFE0194E0EE0FFF1F9A95E1F7EC1B31
:10B66000FD0BE451F74E8081813009F05AC01091F2
:10B67000A700C093A70084858F5F848784858B3063
:10B6800008F44DC08091AA008295869586958370B6
:10B69000833009F444C0108203878091AE008B7F11
:10B6A0008093AE008091AE008E7F8093AE0080913B
:10B6B000AE008D7F8093AE008091AE008F7E809330
:10B6C000AE008091AE008F7B8093AE00C7010C2E40
:10B6D00002C0880F991F0A94E2F78093A800109285
:10B6E000A8000E94166B882349F480915F19882373
:10B6F00029F48091A0008F7D8093A000FE0184E05A
:10B70000EE0FFF1F8A95E1F7EC1BFD0BE451F74E9E
:10B71000218532856381748180E8F9010995109350
:10B72000A7002196C730D10509F093CF0E94A27DD2
:10B7300080919F0086FF21C08091A00086FF1DC0E0
:10B740008091A0008F7B8093A0008EE089BD09B41A
:10B7500000FEFDCF8091D8008F7D8093D80080912E
:10B760009F008F7B80939F008091AE109091AF10CF
:10B7700094609093AF108093AE10FF91EF91DF91A2
:10B78000CF91BF91AF919F918F917F916F915F9179
:10B790004F913F912F911F910F91FF90EF900F903C
:10B7A0000BBE0F900FBE0F901F9018958091D70081
:10B7B00081608093D7008091D70080648093D70008
:10B7C00082B11092B1108091D90081FF05C082E052
:10B7D0008093B110D3D209C081E08093B1108DEF76
:10B7E0008093DA0078940E945E728091B110809309
:10B7F000A51608958091D90081FF02C082E001C0A2
:10B8000081E08093B1109091A5168091B1109817A6
:10B8100009F44EC08DEF8093DA008091D90081FD4C
:10B8200021C08091E2008F7D8093E2008091E20050
:10B830008F7E8093E2008091E2008E7F8093E20011
:10B840008091E200877F8093E2008091E000816038
:10B850008093E0008091D8008F768093D8000E947A
:10B860005E7226C08091A0008D7F8093A0008091A1
:10B87000A0008F7D8093A00080919E008E7F80939A
:10B880009E008091DD0081608093DD0077986F9A43
:10B890008091D70080618093D7008091D80080622A
:10B8A0008093D8008091D8008F768093D80066D29C
:10B8B0008091B1108093A516813019F0823019F46F
:10B8C00089C20C94616D08950F931F93DF93CF93FA
:10B8D00000D0CDB7DEB78091E8008B7F8093E80081
:10B8E0001091F1000091F1000630F9F0073068F492
:10B8F000013009F434C1013008F4A1C1033009F466
:10B9000062C1053009F020C2EDC0093009F40FC151
:10B910000A3020F4083009F017C2BAC00A3009F41E
:10B92000C1C10B3009F010C2E7C1103809F00CC2D8
:10B930006091F1008091F100813019F0823089F43A
:10B9400006C082E18093AE1687E99CE005C089E5D8
:10B950008093AE1689EA9CE09093B0168093AF1660
:10B9600005C00E940374882309F4EEC18091F100A0
:10B970008091F1008091F10089838091F1008A83A8
:10B980008091E800877F8093E80029813A81809147
:10B99000AE1690E08217930730F48F739070892B66
:10B9A00021F461E003C02093AE1660E08091E800CE
:10B9B0008F7E8093E8003091AF164091B0162091B1
:10B9C000AE162DC08091E80084FF05C0832F942F10
:10B9D000FC0190E013C08091D90080FFF7CF8091E7
:10B9E000E80080FFEFCFF2CF522F5150903451F04A
:10B9F0009F5F84918093F1003196252F3E2F4F2F2A
:10BA0000222391F78091E80084FD16C08091D9002F
:10BA100080FF12C08091E8008E7F8093E80022238F
:10BA200039F43093AF164093B0161092AE160AC098
:10BA30008091E80084FFD3CF3093AF164093B016C7
:10BA40002093AE166130B9F48091E80084FF05C000
:10BA500012C08091D90080FF04C08091E80080FF6F
:10BA6000F8CF8091E8008E7F8093E80004C0809139
:10BA7000D90080FF04C08091E80084FFF8CF809156
:10BA8000E8008F7E8093E8008091E8008B7F27C0DC
:10BA9000103809F059C18091E800877F8093E80051
:10BAA0008091AD168093F1008091E8008E7F8093A5
:10BAB000E8008091E8008F778093E80004C08091CF
:10BAC000D90080FF04C08091E80082FFF8CF809108
:10BAD000E8008B7F8093E8008091E8008F77809367
:10BAE000E80045C1112309F02FC19091F100809128
:10BAF000E3009F778078982B9093E3008091E80093
:10BB0000877F8093E8008091E8008E7F8093E80033
:10BB100004C08091D90080FF04C08091E80080FFBC
:10BB2000F8CF8091E30080688093E30020C1112367
:10BB300009F00AC19091F100923008F005C180919E
:10BB4000E800877F8093E8009093AD168091E8002D
:10BB50008E7F8093E800892F0E94E67508C111232B
:10BB6000C1F1123009F0F0C08091F1009091F10024
:10BB7000882309F0E9C0E091F100EF77E093E90054
:10BB80008091EB0080FF43C0EE23B1F08091EB0089
:10BB900080618093EB0081E090E00E2E02C0880F60
:10BBA000991F0A94E2F78093EA001092EA008091CC
:10BBB000EB0088608093EB001092E900F0E0EA551A
:10BBC000F94E108233C0112321F0123009F0BCC0AD
:10BBD00003C08091F100B8C08091F1009091F10014
:10BBE000882309F0B1C0E091F100EF7751F4809122
:10BBF000EB0080628093EB008091E800877F809368
:10BC0000E800E093E9008091EB0080FD03C0109212
:10BC1000E9009AC08091EB0080628093EB00109263
:10BC2000E900F0E0EA55F94E81E080838091E80078
:10BC3000877F8093E8008091E8008E7F50CF8091CD
:10BC4000F1008091F100E091F100113829F01238F3
:10BC500059F0103809F078C08091E800877F809310
:10BC6000E8001092F1000DC08091E800877F80937A
:10BC7000E800F0E0EF77F070EA55F94E80818093AC
:10BC8000F1001092F1008091E8008E7F8093E8002F
:10BC900004C08091D90080FF1ACF8091E80082FF14
:10BCA000F8CF15CF113809F04FC08091F100809185
:10BCB000F1009091F10099839091F1009A8388238B
:10BCC00009F042C08091E800877F8093E800898175
:10BCD0009A810E94A6738093F1008091E8008E7F84
:10BCE0008093E80004C08091D90080FFF0CE80915D
:10BCF000E80082FFF8CFEBCE113031F56091F10012
:10BD00008091F1009091F10099839091F1009A83D4
:10BD10008823D1F48091E800877F8093E8008981AF
:10BD20009A810E94A8731092E9008091E8008E7FAA
:10BD30008093E80004C08091D90080FF18C08091F2
:10BD4000E80080FFF8CF13C0812F602F0E9410768B
:10BD5000882369F48091EB0080628093EB008091EE
:10BD6000E800877F8093E80081E08093A6160F901B
:10BD70000F90CF91DF911F910F9108957894E8ED86
:10BD8000F0E080818F7680838081806980838081EC
:10BD90008F7B8083789408958EE089BD09B400FE7E
:10BDA000FDCFF8948091D8008F7D8093D8000E94B9
:10BDB00039088091E0008E7F8093E0007894809134
:10BDC000E20081608093E2008091E20088608093CD
:10BDD000E20008958091D90080FF13C08091B310D4
:10BDE000882379F481E08093B3101092B21080918F
:10BDF000AE109091AF1082609093AF108093AE1010
:10BE0000CBDF8091D90080FD18C034C01092B310F0
:10BE10001092AD168091AE109091AF108460909307
:10BE2000AF108093AE108091E00081608093E000BD
:10BE30008091D80080628093D8008091AE1090915C
:10BE4000AF1090FF10C08091AE109091AF109E7F08
:10BE50009093AF108093AE1081E08093EA0010922F
:10BE6000EA001092AD161092E9008091E80083FF7D
:10BE700006C02ACD8091B3108130F9F6C7CF08955E
:10BE80000F931F93CF93DF938091B51090E02AE436
:10BE900030E0829FF001839FF00D929FF00D1124FE
:10BEA000DF01A754B94E8091F9178C938091FA174E
:10BEB00011968C93DF01A954B94E8091FB178C9396
:10BEC0008091FC1711968C93EF54F94E00851185E3
:10BED00050E0EF012696A52FB0E0FD01EE0FFF1F09
:10BEE000EB59F84F8081918180179107E9F4BD01EA
:10BEF0006F5F7F4FFB01EE0FFF1FEB59F84F408143
:10BF000011C0FB01E40FF11DEE0FFF1FEB59F84FBD
:10BF100020813181888199812817390711F481E0C6
:10BF20000DC04150442369F7AA0FBB1FA959B84F50
:10BF30008C918E5F580F593070F280E0DF91CF9175
:10BF40001F910F9108952F923F924F925F927F928F
:10BF50008F929F92AF92BF92CF92DF92EF92FF9219
:10BF60000F931F93DF93CF9300D0CDB7DEB78091AF
:10BF7000F217823011F080E086C04091F3174983B8
:10BF80008091F4178A838091B51090E02AE430E024
:10BF9000B901869F9001879F300D969F300D112427
:10BFA000F901EF54F94E8091F81782878091F917C3
:10BFB0008387742E50E040E015E1412E512C490159
:10BFC000B5E0CB2ED12CCE0EDF1E57C08081580F8E
:10BFD00054C0652F70E0FB01EF50F84E8181843032
:10BFE000A9F7A580B680378120E0A2E0EA2EF12CE7
:10BFF000EE0EFF1E8F010D5F1F4F1F0184E090E0CA
:10C00000280E391EE22FF0E0E958F84F80818A159A
:10C0100051F581818B1539F58281831721F5842FA4
:10C0200090E0849DF001859DF00D949DF00D11240C
:10C03000E80DF91DEF54F94ED7018C918487D80192
:10C040008C918587A6861786B08A118A328B138ACF
:10C05000D1018C91848B4F5FF60180818F5F80834B
:10C06000433080F42D5F2D5F283160F26F50784EA1
:10C07000DB018C91580F5B3F18F4571508F4A9CFDA
:10C08000842F411181E00F900F90CF91DF911F918C
:10C090000F91FF90EF90DF90CF90BF90AF909F9067
:10C0A0008F907F905F904F903F902F900895282F12
:10C0B0009091F11718C08081980F9B3F10F090E08D
:10C0C00014C0A92FB0E0FD01EF50F84E81818430FB
:10C0D00091F78281821719F48381861731F0AF506E
:10C0E000B84E8C91980F9A3F60F3892F0895482F8E
:10C0F0008091B510682F70E08AE490E0689FF001AD
:10C10000699FF00D789FF00D1124EA53F94E20E05D
:10C1100030E028C0E2E0F0E0EE0FFF1FEE0FFF1F5F
:10C1200085E190E0AC01249FC001259F900D349FD4
:10C13000900D1124E80FF91F8AE490E09C01629FA2
:10C14000C001639F900D729F900D1124E80FF91F9D
:10C15000EF54F94E868908952F5F3F4F759623302F
:10C16000310581F08081841719F4E0E0F0E0D4CF4C
:10C170008481841719F4E1E0F0E0CECF8085841744
:10C1800059F7C8CF80E008951F93DC012091B510C6
:10C1900030E085E290E0289FF001299FF00D389F64
:10C1A000F00D1124EE0FFF1FED54F94E10818AE4BB
:10C1B00090E0289FF001299FF00D389FF00D112489
:10C1C000EF54F94E81818093A1008091AE1090913F
:10C1D000AF109D7F9093AF108093AE102091A00080
:10C1E0008091A00080628093A0003091F01707C07A
:10C1F0008091D90081FD70C13A3009F46DC1809100
:10C20000AE109091AF1091FFF3CF25FD05C0809146
:10C21000A0008F7D8093A0001092A7008091AA00BB
:10C220008F7C8093AA008091A600877F8093A600D0
:10C230008091A9008F7B8093A9006091551960932C
:10C24000AF00809156198093AF0080915719809369
:10C25000AF00809158198093AF0080915919809355
:10C26000AF0080915A198093AF0080915B19809341
:10C27000AF0080915C198093AF008091A6008F770A
:10C280008093A6000BC08091D90081FD25C13A3072
:10C2900009F422C18091A60084FD2EC18091A600E0
:10C2A00083FFF1CF8091AE109091AF109D7F90935E
:10C2B000AF108093AE102091A0008091A00080620A
:10C2C0008093A0008091A90080648093A900409190
:10C2D0005B1950915C1907C08091D90081FDFCC0A9
:10C2E0003A3009F4F9C08091AE109091AF1091FFEF
:10C2F000F3CF25FD05C08091A0008F7D8093A00025
:10C3000067FF86C08091A9008F7D8093A9008091EE
:10C31000AA008F7C80618093AA008091A6008E7F06
:10C320008093A600612F70E040C08091A9008F7BB0
:10C330008093A9000FC08091D90081FDCDC09A30B3
:10C3400009F4CAC08091A60084FDD6C08091A600E1
:10C3500081FDDCC08091A60080FFEDCF2091F6002A
:10C36000211739F480915D19813019F0461B570B64
:10C3700002C040E050E0FD01922F04C08091AF0068
:10C38000819391509923D1F7A20FB11D8091A900FB
:10C3900080648093A9008091A6008E7F8093A60080
:10C3A0008091A6008F778093A6009091F017411599
:10C3B000510509F0BACF8091AA008F7C80628093EA
:10C3C000AA008091A6008B7F8093A6008091A9008F
:10C3D0008F7B8093A9008091A6008F778093A60021
:10C3E0000FC08091D90081FD77C09A3009F474C0E4
:10C3F0008091A60084FD80C08091A60081FD86C04A
:10C400008091A60082FFEDCF8091A6008B7F96C021
:10C410008091AA008F7C80628093AA008091A60000
:10C420008B7F8093A600612F70E037C08091A900B8
:10C430008F7B8093A9004617570730F4242F40E0E4
:10C4400050E0FD01922F08C0461B570B212FF9CF5A
:10C4500081918093AF0091509923D1F7A20FB11D24
:10C460008091A6008F778093A6000EC08091D9009E
:10C4700081FD32C03A3081F18091A60084FD3CC03C
:10C480008091A60081FD42C08091A60082FFEECF80
:10C490008091A6008B7F8093A6004115510531F64F
:10C4A0008091A90080648093A9008091AA008F7C6C
:10C4B00080618093AA008091A6008E7F8093A60061
:10C4C0008091A9008F7B8093A90027C08091D9001B
:10C4D00081FD02C03A3061F48091A90080648093AC
:10C4E000A90081E08093A8001092A80088E029C0EC
:10C4F0008091A60084FF06C08091F5008F71109294
:10C50000F5001FC08091A60081FF07C08091A600A2
:10C510008D7F8093A60080E214C08091A60080FFEA
:10C52000D5CF8091A6008E7F8093A6008091A90030
:10C5300080648093A9008091A6008F778093A600E5
:10C5400080E01F910895AF92BF92CF92DF92FF9249
:10C550000F931F93CF93DF93A82EBB248AE490E020
:10C56000A89EF001A99EF00DB89EF00D1124EF5485
:10C57000F94E86859785099709F043C08091EA179F
:10C5800081508093EA179181C0E0D0E0FE01E5512F
:10C59000F84E8081891789F5FE01EE0FFF1FEE0F1F
:10C5A000FF1FE652F84E82E080838183DE01AA0FEE
:10C5B000BB1FAA0FBB1FA452B84E8C93838305EBFD
:10C5C00016E1FF246E010894C11CD11CF801808182
:10C5D00090E08C159D0539F48091B11681508093BF
:10C5E000B1168F2DB0DFF394065B1F4FF4E0FF16FA
:10C5F00069F7C551D84E188204C02196C430D105C0
:10C6000029F68091B11690E095012F5F3F4F821778
:10C610009307B1F520E030E0A5E1B0E08AE490E0D6
:10C62000A89EB001A99E700DB89E700D112417C070
:10C630008081882359F09091A7008093A700809172
:10C64000AB008D7F8093AB009093A7004F5F349633
:10C65000433071F72F5F3F4F2330310589F02F5F53
:10C660003F4F2A9FF0012B9FF00D3A9FF00D1124B0
:10C6700021503040E60FF71FEE54F94E40E0D8CF7E
:10C680008AE490E0A89E9001A99E300DB89E300DDE
:10C690001124D901AF54B94E11961C92119785E21D
:10C6A00090E0A89EF001A99EF00DB89EF00D112417
:10C6B000EE0FFF1FED54F94E1082118214961C925A
:10C6C000149715961C92159717961C921E92169702
:10C6D00019961C921E9218971A961C921A971B96DE
:10C6E0001C92F901E354F94E80E01082118213820A
:10C6F0001282158214821782168210861186128683
:10C7000013861486158616861786108A118A128A51
:10C71000138A148A8F5F7596833039F7DF91CF9132
:10C720001F910F91FF90DF90CF90BF90AF90089531
:10C730001F9310E0812F07DF1F5F1430D9F710928D
:10C74000B5108091B2168093A10080E07FD181E086
:10C750007DD182E07BD183E079D11092EB171092EA
:10C76000EC171092ED171092EE171092B1161F9160
:10C7700008952F923F924F925F926F927F928F9285
:10C780009F92AF92BF92CF92DF92EF92FF920F9360
:10C790001F93DF93CF9300D000D0CDB7DEB7809149
:10C7A000B1168150282F30E08AE490E0289FF001F4
:10C7B000299FF00D389FF00D1124EF54F94E45815B
:10C7C00049839091A700DD24D394D092A700809153
:10C7D000AB0081FF04C0D39456E0D516B1F7909317
:10C7E000A7008AE490E0DC012A9FC0012B9F900DF6
:10C7F0003A9F900D11240DEBE02E06E1F02EE80E8D
:10C80000F91E662477241C01FEC0F7018081618136
:10C810004EDCE82FF0E0EF50F84EB080B80ED701B4
:10C820001896AC90AA941A82E5E1F0E06E9E200181
:10C830006F9E500C7E9E500C1124DAC08081B80E81
:10C84000FAEFFB1508F4EAC04B2D50E05C834B83F4
:10C85000FA01EF50F84E8181853081F713E0812E87
:10C86000912C840E951EF401EF50F84E0081033098
:10C8700071F4D70112968D919C911397089739F412
:10C8800018968C911897815018968C93B0C0D092BE
:10C89000A7008091A9008E7F8093A9008091AB00B2
:10C8A0008D7F8093AB008091A90081608093A90067
:10C8B000033061F4F70182819381099739F4D092B2
:10C8C000A7001092AD0081E960E04AC08091EA17AC
:10C8D000882331F5D092A700EB81FC81EF50F84E10
:10C8E00086818093AD00128117FD03C0B0E2CB2E8C
:10C8F00002C0A0E1CA2EEB81FC81EF50F84E84818A
:10C9000090E00E9460080295000F000F007C1F77E6
:10C91000012B682F6295607F6460802F8C2920C076
:10C92000023001F5D092A700EB81FC81EF50F84E68
:10C9300086818093AD00128117FD02C000E201C024
:10C9400000E1EB81FC81EF50F84E848190E00E9481
:10C9500060081068682F6295607F6460812F802B6B
:10C960000E944F08FA81AF2FB0E0AD01440F551F70
:10C97000440F551F440D551D420D531D4F54594E24
:10C980002B813C812F50384EF9018281FA01858B31
:10C99000D68AAD01440F551F440F551F4E5F5F4FA0
:10C9A000440D551D420D531D4F54594EF9018481BC
:10C9B000FA01858B1396AA0FBB1FAA0FBB1FA40DEC
:10C9C000B51DA20DB31DAF54B94E41EF57E1840E12
:10C9D000951EF40180811C968C93D9012C91B6E0B0
:10C9E000BD15E0F0B20ED394EA81EF5FEA83AA941A
:10C9F000FFEFAF1609F028CF0894611C711C45E1C8
:10CA000050E0E40EF51E5981651608F4FECE8091C3
:10CA1000EF1784608093EF1781E001C080E00F90F2
:10CA20000F900F900F90CF91DF911F910F91FF907A
:10CA3000EF90DF90CF90BF90AF909F908F907F90BE
:10CA40006F905F904F903F902F90089590E0EAEDA7
:10CA5000F7E1880F991F880F991FDF01A80FB91FF1
:10CA600022E02C9311962C931197E80FF91F228343
:10CA700013962C930895DF93CF9300D000D0CDB7B9
:10CA8000DEB793EA909355191092561910925819DF
:10CA9000109257198093591910925A1984E090E016
:10CAA00090935C1980935B1910925D1981EF97E167
:10CAB0006BDB6091F1177091F2178091F3179091F1
:10CAC000F4170F900F900F900F90CF91DF91089572
:10CAD0008F929F92AF92BF92CF92DF92EF92FF928E
:10CAE0000F931F93CF93DF93882EC62EE42EFF243F
:10CAF0000894E108F108F701E551F84EE081A2EB56
:10CB0000B6E1992490E08C918E1709F4992E9F5FDD
:10CB1000A65BBF4F9430B9F7E4EBF6E120E08081EB
:10CB2000881529F48181841711F4D22E06C02F5F55
:10CB3000E65BFF4F243099F7DD24C82DD0E0870154
:10CB4000000F111F000F111F82E0C81681F48D2DF8
:10CB5000FADC8091B11681508093B116C00FD11FBD
:10CB6000C752D84EC88281E08093B61064C25E017D
:10CB70000894A108B108E801CA0DDB1DC652D84EC1
:10CB80008881843009F456C0853009F4F9C08230B8
:10CB900009F051C2CC2009F04EC28091B1168F5FCE
:10CBA0008093B116815090E025E230E0829FF00141
:10CBB000839FF00D929FF00D1124EE0FFF1FED5497
:10CBC000F94E81822AE430E0829FF001839FF00DCC
:10CBD000929FF00D1124EF54F94E44839092B510BA
:10CBE000892D90E0829FF001839FF00D929FF00DC0
:10CBF0001124EF54F94E81818093A10083E2809348
:10CC0000551983E08093561984E090E09093581969
:10CC1000809357198092591910925A1910925C19E1
:10CC200010925B1910925D1981EF97E1ADDA84E003
:10CC3000888301C291E0C91609F0FDC13091F01757
:10CC400020E08091AE109091AF1091FF0AC08091CA
:10CC5000AE109091AF109D7F9093AF108093AE1067
:10CC60002F5F8091D90081FD06C03A3021F080917C
:10CC7000DF0082FF0BC0EE0CFF1CEE0CFF1CEA0C69
:10CC8000FB1CEAEDF7E1EE0EFF1EA5C02A3FC8F23D
:10CC9000D092B5102D2D30E00AE410E0209FF00175
:10CCA000219FF00D309FF00D1124EF54F94E81813A
:10CCB0008093A10085E290E0289FE001299FD00D9C
:10CCC000389FD00D1124CC0FDD1FCD54D94E88E0F4
:10CCD000888380E88093551986E08093561980E018
:10CCE00091E0909358198093571910925A19109205
:10CCF000591980E490E090935C1980935B1981E06E
:10CD000080935D1981EF97E13FDA882309F093C1A1
:10CD10009092B510892D90E0809FF001819FF00DD9
:10CD2000909FF00D1124EF54F94E81818093A10062
:10CD30008091F817888383E28093551983E080936C
:10CD4000561984E090E09093581980935719809277
:10CD5000591910925A1910925C1910925B1910927D
:10CD60005D1981EF97E110DAEE0CFF1CEE0CFF1C51
:10CD7000EA0CFB1C8AED97E1E80EF91E85E02CC059
:10CD8000F1E0CF1609F057C13091F01720E0809103
:10CD9000AE109091AF1091FF0AC08091AE109091AB
:10CDA000AF109D7F9093AF108093AE102F5F809156
:10CDB000D90081FD06C03A3021F08091DF0082FF6A
:10CDC0000EC0EE0CFF1CEE0CFF1CEA0CFB1C8AEDE7
:10CDD00097E1E80EF91E82E0F70180832CC12A3F1B
:10CDE000B0F2D092B510CD2DD0E08AE490E0C89F8B
:10CDF0008001C99F100DD89F100D11240F54194E9A
:10CE0000F80181818093A1001092551985E08093EB
:10CE100056192596D0935819C093571925971092F3
:10CE20005A191092591910925C1910925B191092AC
:10CE30005D1981EF97E1A8D98D2D8B5FF801818372
:10CE4000D092B5108093A10080E88093551986E0B8
:10CE50008093561980E091E0909358198093571968
:10CE600010925A191092591982E190E090935C192E
:10CE700080935B1910925D1981EF97E185D9882322
:10CE800009F0D9C00E94405F813029F48091EF17EA
:10CE900081608093EF1780E88093551916E0109316
:10CEA000561980E092E09093581980935719109288
:10CEB0005A19109259190FEFC02ED12CD0925C192B
:10CEC000C0925B1910925D1981EF97E15DD98823BB
:10CED00009F0B1C038D8882309F4ADC04ADC8823F2
:10CEE00009F4A9C01092551989E08093561981E080
:10CEF00090E0909358198093571910925A191092F4
:10CF0000591910925C1910925B1910925D1981EFFA
:10CF100097E13AD9882309F08EC0EE0CFF1CEE0C85
:10CF2000FF1CEA0CFB1C8AED97E1E80EF91EF701E5
:10CF300010838091B51090E02AE430E0829FF001E8
:10CF4000839FF00D929FF00D1124EF54F94E8685CA
:10CF50009785099709F06CC080EA80935519109362
:10CF6000561980E099E290935819809357191092BE
:10CF70005A1910925919D0925C19C0925B191092EB
:10CF80005D1981EF97E100D9882309F054C0009121
:10CF9000F31711E0A3E2AA2EF3E0BF2EE8E0CE2EB5
:10CFA000D12C79E5E72E79E1F72E16C0A09255191C
:10CFB000B0925619D0925819C09257191093591916
:10CFC000F701118210925C1910925B1910925D1991
:10CFD00081EF97E1D9D81F5F011740F7E091EA1779
:10CFE0009E2F9F5F9093EA17F0E0EE0FFF1FEE0F6A
:10CFF000FF1FDF01A652B84E82E08C9311968C93EE
:10D000001197E452F84E808313968C93A92FB0E0C9
:10D01000A651B84E8AE490E0C89FF001C99FF00D78
:10D02000D89FF00D1124EF54F94E81818C9303C0E9
:10D0300081E08093B910DF91CF911F910F91FF9004
:10D04000EF90DF90CF90BF90AF909F908F9008951A
:10D050002F923F924F925F927F928F929F92AF92C8
:10D06000BF92CF92DF92EF92FF920F931F93CF93D5
:10D07000DF93A62E992420E030E070E061507040EC
:10D0800014C04081423041F0463031F02617370756
:10D0900009F0A6C0952E04C05F5F3196553089F720
:10D0A0002F5F3F4F2430310549F0F901EE0FFF1F8C
:10D0B000EE0FFF1FE652F84E51E0E3CFCA2CDD24FD
:10D0C000CC0CDD1CCC0CDD1C26ED37E1C20ED31ED2
:10D0D000C1E0D0E0482E5524E3E27E2E88248394DC
:10D0E00070E1272E312CBC2E992019F0C91509F0BA
:10D0F0006FC0C2010C2E02C0959587950A94E2F785
:10D1000080FF60C08B2DB7DC7B018C0180FF22C0CB
:10D1100070925519809256193092581920925719C9
:10D12000D0935A19C093591910925C1910925B1937
:10D1300010925D1981EF97E127D8C7018170907037
:10D14000892B29F0F1FC3EC08B2D60E039C08B2D7E
:10D1500062E036C082FF18C070925519809256194D
:10D1600082E190E09093581980935719D0935A19FF
:10D17000C093591910925C1910925B1910925D19A5
:10D1800081EF97E101D81EC084FF1CC07092551931
:10D1900080925619E4E1F0E0F0935819E0935719A2
:10D1A000D0935A19C093591910925C1910925B19B7
:10D1B00010925D1981EF97E10E94C4608B2D61E0B0
:10D1C0004A2D86DCF6018081823011F0863041F4F0
:10D1D0000894C11CD11C2196C530D10509F083CF1C
:10D1E000DF91CF911F910F91FF90EF90DF90CF9043
:10D1F000BF90AF909F908F907F905F904F903F90A7
:10D200002F900895EF92FF920F931F93CF93DF9388
:10D21000182FE090A0008091A00080628093A00071
:10D220001093A7008091AA008F7C80628093AA004F
:10D230008091A6008B7F8093A6008091A9008F7BB0
:10D240008093A900F090F017B0E0C8E0D0E092C061
:10D250008091AB0090E08077907024E09595879561
:10D260002A95E1F79E0102C0220F331F8A95E2F74B
:10D27000A22F822F90E06817790710F0022F02C0CA
:10D28000062FA62FFA019A2F04C081918093AF0038
:10D2900091509923D1F74A0F511D1092B0108091EF
:10D2A000A6008B7F8093A6008091A6008F77809345
:10D2B000A60030E054C08091D90081FD0DC08AE005
:10D2C000F81651F08091B0108A3F98F01092B0108B
:10D2D0003A3010F43F5F0DC081E090E002C0880F4B
:10D2E000991F1A95E2F78093A8001092A80090E881
:10D2F0004DC08091A60084FF27C09091F5009F71DA
:10D300001092F500983001F5B53608F03FC020E0E6
:10D310008091AE109091AF1091FF0AC08091AE1035
:10D320009091AF109D7F9093AF108093AE102F5FC0
:10D330008091D90081FD02C0223050F3BF5F8091FF
:10D34000A9008F7B8093A9008091A60081FF07C070
:10D350008091A6008D7F8093A60090E217C08091F7
:10D36000A60082FFA8CF601B71098091A6008B7F69
:10D370008093A6006115710509F06ACF8091AC0019
:10D3800090E083709070892BC9F790E08091A9009C
:10D3900080648093A900E5FC05C08091A0008F7D8A
:10D3A0008093A000892FDF91CF911F910F91FF9063
:10D3B000EF9008952F923F924F925F926F927F92DB
:10D3C0008F929F92AF92BF92CF92DF92EF92FF9295
:10D3D0000F931F93CF93DF93582E8B01EA01FB012C
:10D3E000A081B181118210824090A0008091A000A4
:10D3F00080628093A0005092A7008091A900806273
:10D400008093A9008091AA008F7C80618093AA00FC
:10D410008091A6008E7F8093A60058E0252E312CA7
:10D42000E1C08091A9008F7B8093A9008091A60024
:10D430008F778093A6001092B0102091F01790E0A3
:10D4400041C08091D90081FD0CC02A3051F08091FB
:10D45000B0108A3F98F01092B0109A3010F49F5F8D
:10D460000DC081E090E002C0880F991F5A94E2F746
:10D470008093A8001092A80090E8BDC08091A600FB
:10D4800084FF06C09091F5009F711092F500B3C023
:10D490008091A60081FF16C08091A60080FD16C075
:10D4A00081E090E002C0880F991F5A94E2F78093C0
:10D4B000A8001092A8008091A6008D7F8093A600FE
:10D4C00090E299C08091A60080FFBBCF8091A90017
:10D4D00080648093A9002091F7008091F600F22EDD
:10D4E000EE2490E08E299F29A817B90708F460C0A0
:10D4F0002091F7008091F600D22ECC2490E08C2968
:10D500009D298A179B07F8F44091F7002091F600B7
:10D510008091AB00542F40E030E0242B352B90E07D
:10D520008077907044E0959587954A95E1F7B10131
:10D5300002C0660F771F8A95E2F72617370718F49F
:10D54000A0E0B0E00BC02091F7008091F600B22E71
:10D55000AA2490E08A299B29A81BB90B8091F70087
:10D560002091F600982E882430E028293929F801E6
:10D5700080819181820F931F91838083209769F12D
:10D580008091F7009091F600782E6624692F70E064
:10D5900066297729FE019B0105C08091AF00819328
:10D5A0002150304021153105C1F7C60FD71F15C0D6
:10D5B000F801808191818A0F9B1F9183808320973E
:10D5C00051F0FE019D018091AF00819321503040C8
:10D5D000D1F7CA0FDB1FA0E0B0E08091A6008E7FDC
:10D5E0008093A600109709F01CCF8091A900806459
:10D5F0008093A90090E045FC05C08091A0008F7D3C
:10D600008093A000892FDF91CF911F910F91FF9000
:10D61000EF90DF90CF90BF90AF909F908F907F90D2
:10D620006F905F904F903F902F90089520E030E0F2
:10D63000F90174E0EE0FFF1F7A95E1F7E21BF30B9F
:10D64000E451F74E8081813031F02F5F3F4F27301A
:10D65000310571F780E008951F920F920FB60F9277
:10D660000BB60F921124EF92FF920F931F932F93FB
:10D670003F934F935F936F937F938F939F93AF935A
:10D68000BF93CF93DF93EF93FF938091A700809395
:10D690005E190E94A7088093A700C82FD0E0FE0162
:10D6A00024E0EE0FFF1F2A95E1F7EC1BFD0BE45180
:10D6B000F74EE184F2848091A60084FF2DC0809112
:10D6C000F5008F71838710828091AE008B7F8093ED
:10D6D000AE008091AE008E7F8093AE008091AE0050
:10D6E0008D7F8093AE008091AE008F7E8093AE00E0
:10D6F0008091AE008F7B8093AE0081E090E00C2E95
:10D7000002C0880F991F0A94E2F78093A800109234
:10D71000A8001092F50086C18091A60081FF04C088
:10D7200080E28387108259C18091A60080FFB0C03B
:10D730000781108583819481080F191FA181B2810F
:10D7400083819481A81BB90B8091A9008064809388
:10D75000A9004091F7002091F600942F80E030E07E
:10D76000822B932BA817B90708F45EC04091F700ED
:10D770002091F600942F80E030E0822B932B8A17C3
:10D780009B0700F56091F7008091F6002091AB00B7
:10D79000562F40E090E0482B592B30E02077307036
:10D7A00094E0359527959A95E1F788E090E002C0DE
:10D7B000880F991F2A95E2F74817590718F4A0E037
:10D7C000B0E00BC04091F7002091F600942F80E06C
:10D7D00030E0822B932BA81BB90BFE0184E0EE0FE7
:10D7E000FF1F8A95E1F7EC1BFD0BE451F74E6381B7
:10D7F00074814091F7002091F600942F80E030E092
:10D80000822B932B860F971F948383838091F7003D
:10D810009091F60006C08091AF00F80181938F01CE
:10D8200091509923C1F712C0838194818A0F9B1F65
:10D83000948383839A2F06C08091AF00F80181936F
:10D840008F0191509923C1F7A0E0B0E08091A6002C
:10D850008E7F8093A600FE0114E0EE0FFF1F1A9545
:10D86000E1F7AB2BB9F08091A9008F7B8093A900E1
:10D870008091A6008F778093A6001092B010EC1BC9
:10D88000FD0BE451F74E14868FEF9FE09687858756
:10D8900010E02CC0EC1BFD0BE451F74E10821386F8
:10D8A0008091AE008B7F8093AE008091AE008E7F22
:10D8B0008093AE008091AE008D7F8093AE0080910A
:10D8C000AE008F7E8093AE008091AE008F7B809300
:10D8D000AE0081E090E00C2E02C0880F991F0A94E0
:10D8E000E2F78093A8001092A80011E08091A600B2
:10D8F00082FF99C08091A6008B7F8093A600FE01D5
:10D90000A4E0EE0FFF1FAA95E1F7EC1BFD0BE4511D
:10D91000F74E2381348185819681820F931F9483F2
:10D92000838316821582A781B085638174814181CA
:10D93000528183819481481B590B09F44CC080911A
:10D94000A9008F7B8093A9008091AB0090E0807745
:10D950009070E4E095958795EA95E1F728E030E04E
:10D9600002C0220F331F8A95E2F7822F90E04817FA
:10D97000590708F4242FA60FB71FFE0164E0EE0F2D
:10D98000FF1F6A95E1F7EC1BFD0BE451F74E858113
:10D990009681820F911D9683858304C08D9180931B
:10D9A000AF0021502223D1F71092B010FE0154E0B5
:10D9B000EE0FFF1F5A95E1F7EC1BFD0BE451F74EFC
:10D9C00014868FEF9FE0968785878091A6008F77DA
:10D9D0008093A60028C0108213868091AE008B7FB2
:10D9E0008093AE008091AE008E7F8093AE008091D8
:10D9F000AE008D7F8093AE008091AE008F7E8093CD
:10DA0000AE008091AE008F7B8093AE0081E090E00D
:10DA10000C2E02C0880F991F0A94E2F78093A80089
:10DA20001092A80011E080915E198093A70020E079
:10DA300030E0F90144E0EE0FFF1F4A95E1F7E21BE9
:10DA4000F30BE451F74E8081813059F02F5F3F4F47
:10DA50002730310571F717C08091A0008F7D80932A
:10DA6000A0001123A9F0FE0124E0EE0FFF1F2A956C
:10DA7000E1F7EC1BFD0BE451F74E83856381748164
:10DA8000F701099505C080915F19882329F3E9CF33
:10DA9000FF91EF91DF91CF91BF91AF919F918F91C6
:10DAA0007F916F915F914F913F912F911F910F91B6
:10DAB000FF90EF900F900BBE0F900FBE0F901F9036
:10DAC0001895EF92FF920F931F93CF93DF9380915E
:10DAD000F017853009F4ABC2863090F4823009F437
:10DAE0006EC1833030F48823D9F0813009F0DDC471
:10DAF0005EC0833009F482C1843009F0D6C46DC29F
:10DB0000883009F41FC4893020F4863009F0CDC470
:10DB100067C38A3009F4C5C48A3008F46FC4C5C429
:10DB20008091EF17887F8093EF171092AF101092BB
:10DB3000AE101092B9101092B5101092EA178091A1
:10DB4000DF0082FD04C08091DF0081FF0FC0809163
:10DB5000DF008B7F8093DF008091DF008D7F8093DB
:10DB6000DF008091DD0081608093DD008091D8002E
:10DB70008F7E8093D800779A6F9A8091D7008F7E9E
:10DB80008093D7008091DF0080FF91C48091DF00F7
:10DB90008E7F8093DF008091D80080618093D800D1
:10DBA0008091DD0082608093DD0081E07BC4809104
:10DBB0009F0080FD05C08091B810813009F0C3C07E
:10DBC0008EEF80939F009091EF171092AF101092FC
:10DBD000AE101092B9101092B8108091A00082601F
:10DBE0008093A0007894987F9093EF1780919E0087
:10DBF000816080939E008091A00080628093A0004D
:10DC00001092BC101092BB1020E030E019C080913F
:10DC1000AE109091AF1091FF0BC08091AE1090911B
:10DC2000AF109D7F9093AF108093AE102F5F3F4F4A
:10DC30008091D90081FD78C08091DF0082FD74C0A1
:10DC40002436310520F38091A0008D7F8093A000C1
:10DC500080919E00826080939E008091AE10909192
:10DC6000AF109D7F9093AF108093AE1080919E0077
:10DC700081FDFCCF8BEF80939F001092BC1010921F
:10DC8000BB1020E030E017C08091AE109091AF1033
:10DC900091FF0FC080919F0081FF0BC03093BC109B
:10DCA0002093BB108EEF80939F008DEF80939F0099
:10DCB0000AC02F5F3F4F8FEF2F3F380729F7309370
:10DCC000BC102093BB108091A00082608093A000C4
:10DCD0001092A7001092AD0080E060E30E944F0810
:10DCE0001092BC101092BB104091F01720E030E071
:10DCF00020C08091AE109091AF1091FF0BC0809129
:10DD0000AE109091AF109D7F9093AF108093AE10A6
:10DD10002F5F3F4F8091D90081FD06C04A3021F02E
:10DD20008091DF0082FF05C03093BC102093BB10B0
:10DD30000AC024363105E8F282E08093F017109291
:10DD4000BC101092BB108091DF0082FD08C0809152
:10DD5000DF0081FD04C08091D90080FDA8C38091BF
:10DD6000DF008B7F8093DF008091DD008B7F8093CD
:10DD7000DD001092F0178091DD0081608093DD005E
:10DD80008091D8008F7E8093D8008091D8008061E8
:10DD90008093D8008091DF008D7F8093DF00809199
:10DDA000DD0082608093DD008091DD0084608093DF
:10DDB000DD0080919E008E7F80939E0078C38091CD
:10DDC000AE109091AF1091FF72C38091AE10909100
:10DDD000AF109D7F9093AF108093AE108091BB10D9
:10DDE0009091BC1001969093BC108093BB1001974A
:10DDF0008436910508F45BC383E054C31092B510D8
:10DE00008091B2168093A10088E08093B31680E8D9
:10DE10008093551986E08093561980E091E09093A5
:10DE200058198093571910925A191092591980E471
:10DE300090E090935C1980935B1981E080935D1969
:10DE400081EF97E10E94C460882309F0C7C1109256
:10DE5000BC101092BB104091F01720E030E01BC0C6
:10DE60008091AE109091AF1091FF0BC08091AE10D9
:10DE70009091AF109D7F9093AF108093AE102F5F65
:10DE80003F4F8091D90081FD09C04A3039F080911F
:10DE9000DF0082FD03C02431310510F33093BC1044
:10DEA0002093BB108091A0008D7F8093A000809173
:10DEB0009E00826080939E008091AE109091AF1082
:10DEC0009D7F9093AF108093AE1080919E0081FD56
:10DED000FCCF8BEF80939F001092BC101092BB1070
:10DEE00020E030E017C08091AE109091AF1091FF0C
:10DEF0000FC080919F0081FF0BC03093BC10209316
:10DF0000BB108EEF80939F008DEF80939F000AC01F
:10DF10002F5F3F4F8FEF2F3F380729F73093BC100B
:10DF20002093BB108091A00082608093A00010928B
:10DF3000BC101092BB101092A7001092AD0080E0B0
:10DF400060E30E944F084091F0172091BB10309180
:10DF5000BC101BC08091AE109091AF1091FF0BC010
:10DF60008091AE109091AF109D7F9093AF108093F1
:10DF7000AE102F5F3F4F8091D90081FD09C04A301C
:10DF800039F08091DF0082FD03C0283C310510F399
:10DF90003093BC102093BB108091F8178093B31678
:10DFA0001092551915E01093561985E090E0909362
:10DFB00058198093571910925A19109259191092A2
:10DFC0005C1910925B1910925D1981EF97E10E9424
:10DFD000C4601093B21684E065C280E8809355193E
:10DFE00086E08093561980E091E0909358198093D1
:10DFF000571910925A191092591982E190E0909392
:10E000005C1980935B1910925D1981EF97E10E9472
:10E01000C460882309F0E2C00E94405F813029F487
:10E020008091EF1781608093EF1785E03BC280E815
:10E030008093551916E01093561980E092E0909362
:10E0400058198093571910925A19109259194FEF75
:10E05000E42EF12CF0925C19E0925B1910925D199C
:10E0600081EF97E10E94C460882309F0B7C00E9445
:10E07000A35F882309F4B2C08091B1168F5F8093AB
:10E08000B1160E94B963882309F411C21092551980
:10E0900089E080935619C1E0D0E0D0935819C0931D
:10E0A000571910925A191092591910925C1910921E
:10E0B0005B1910925D1981EF97E10E94C46088237B
:10E0C00009F08CC01093F0178091EF178260809355
:10E0D000EF178091A00082608093A0008091B5101E
:10E0E00090E02AE430E0829FF001839FF00D929F40
:10E0F000F00D1124EF54F94E86859785099709F0A4
:10E1000066C080899189892B09F061C082899389D1
:10E11000892B09F05CC080EA809355191093561939
:10E1200080E099E2909358198093571910925A19E8
:10E1300010925919F0925C19E0925B1910925D19D6
:10E1400081EF97E10E94C460882309F045C0809167
:10E15000F3178093BD10D093BC10C093BB1003E2A3
:10E1600013E0C8E0D0E01FC0009355191093561972
:10E17000D0935819C093571930935A1920935919AD
:10E1800010925C1910925B1910925D1981EF97E162
:10E190000E94C4608091BB109091BC100196909336
:10E1A000BC108093BB102091BB103091BC108091AB
:10E1B000BD1090E082179307B8F681E08093EA17CC
:10E1C00085E08093EB1780E00E94266505C01092E1
:10E1D000EA1781E08093B910789469C187E062C141
:10E1E0001092B9101092B6108091EA17882309F4A2
:10E1F0005EC18091BA10882309F059C18091B51091
:10E200008093EB1881E08093BE10CAE4D0E07FC019
:10E210001092BD1020E0A62FB0E0A651B84E12C05B
:10E22000322F3F5F822F90E08C9FF0018D9FF00D89
:10E230009C9FF00D1124EF54F94E91818C91981709
:10E2400019F0232F243060F32093BD102093B510D4
:10E25000822F90E08C9FF0018D9FF00D9C9FF00D20
:10E260001124EF54F94E81818093A1008689809317
:10E27000A7008091A6008F7B8093A6008091A600C6
:10E280008E7F8093A6008091A9008F7B8093A90048
:10E290008091A6008F778093A6009091F0178091CF
:10E2A000A60086FD0AC08091D90081FD06C09A3083
:10E2B00021F08091A60080FFF2CF8091A9008064B8
:10E2C0008093A9008091A60086FF05C08091A600DA
:10E2D0008F7B8093A6008091A60080FF13C0809161
:10E2E000A60081FD06C08091AF008093BB10109204
:10E2F000BC108091A6008E7F8093A6008091BB10F9
:10E300000E9428688091BE108F5F8093BE1060913C
:10E31000BE108091EA17861708F07ACF8091EB182B
:10E320008093B51090E02AE430E0829FF001839F53
:10E33000F00D929FF00D1124EF54F94E81818093DE
:10E34000A100B5C08091B51090E02AE430E0829F32
:10E35000F001839FF00D929FF00D1124EF54F94EC0
:10E36000828585FF19C01092551983E08093561954
:10E3700081E090E0909358198093571990935A191F
:10E380008093591910925C1910925B1910925D19C3
:10E3900081EF97E10E94C4608091A00090E035E099
:10E3A000969587953A95E1F7817090709093BC109F
:10E3B0008093BB108091A0008F7D8093A0008091FE
:10E3C0009F008F7D80939F0080919E008E7F809321
:10E3D0009E0080919F008F7B80939F008091A00082
:10E3E00080648093A0008091D80080628093D800E0
:10E3F00089B58D7F89BD19BC89E054C08091AE106C
:10E400009091AF1092FD05C08091B710813009F056
:10E410004EC08091B7108130A1F48091A0008F7B15
:10E420008093A0008EE089BD09B400FEFDCF8091ED
:10E43000D8008F7D8093D80080919F008F7B809340
:10E440009F0080919E00816080939E0080919E003D
:10E45000846080939E0080919F0083FFFCCF809119
:10E460009F008F7E80939F001092B71080919F0035
:10E47000877F80939F008091AE109091AF109B7F1B
:10E480009093AF108093AE108091BB109091BC1010
:10E49000892B29F08091A00080628093A00086E003
:10E4A00001C08BE08093F01702C01092F017DF914B
:10E4B000CF911F910F91FF90EF9008958EE089BD4D
:10E4C00009B400FEFDCF8091D8008F768093D800EC
:10E4D0008091D80080698093D8008091D8008F7D8A
:10E4E0008093D8008091E0008E7F8093E00080913F
:10E4F000D70080618093D7008091D800806480939A
:10E50000D8008091DD0084608093DD008091A000C0
:10E5100082608093A0001092F0170C9498631F9370
:10E5200082E08093E90012E00AC01092E900809135
:10E53000E80083FF02C00E94645C1093E9008091B0
:10E54000EB0085FDF2CF83E08093E90013E00AC081
:10E550001092E9008091E80083FF02C00E94645C91
:10E560001093E9008091EB0085FDF2CF82E080936B
:10E57000E90004C08091EB0080FF38C08091E80082
:10E5800085FFF8CF85E58093F10093E59093F10046
:10E5900082E48093F1009093F1008091BF1080930A
:10E5A000F1008091C0108093F1008091C1108093A0
:10E5B000F1008091C2108093F10080918D168093BC
:10E5C000F10080918E168093F10080918F168093D8
:10E5D000F100809190168093F1008091A1168093B4
:10E5E000F1008091E8008F778093E8001F910895F3
:10E5F00083E08093E9002091F1008091F100833560
:10E6000019F490E0253509F091E08091F100823411
:10E6100009F091E08091F100833411F49923B1F075
:10E620008091E8008B7F8093E8008091E8008F77ED
:10E630008093E80082E08093E9008091EB008062A3
:10E640008093EB0081E08093A81608958091F100FB
:10E650008093BF108091F1008093C0108091F100F1
:10E660008093C1108091F1008093C2108091F100DD
:10E6700080938D168091F10080938E168091F10029
:10E6800080938F168091F100809390168091F10015
:10E69000882321F081E08093611902C010926119F2
:10E6A0008091F1008093601980916219882321F490
:10E6B0000E949840809360198091F100E1E9F6E1B1
:10E6C0008091F100819386E1E13AF807C9F78091E2
:10E6D000E8008B7F8093E8008091E8008F7780933B
:10E6E000E80080916119813019F482E08093E9009B
:10E6F0000E949559813089F08091EB00806280936F
:10E70000EB0080916119813011F0E3E001C0E2E09B
:10E71000F0E0EA55F94E81E0808308958091AD16CE
:10E72000882349F083E08093E9008091E80082FF2C
:10E7300002C05EDFF4CE08958AB1806F8AB9E2EE3E
:10E74000F0E08081846080830C94280980E0089543
:10E75000009751F481E08093E9008091EB008061A3
:10E760008093EB0082E01EC08130910529F582E0A4
:10E770008093E9008091EB0080618093EB0084E05E
:10E780008093EA001092EA008091EB008860809309
:10E79000EB0083E08093E9008091EB00806180933F
:10E7A000EB0088E08093EA001092EA008091EB0091
:10E7B00088608093EB000895029721F584E08093B0
:10E7C000E9008091EB0080618093EB0080E1809311
:10E7D000EA001092EA008091EB0088608093EB00E1
:10E7E00085E08093E9008091EB0080618093EB00ED
:10E7F00080E28093EA001092EA008091EB0088604A
:10E800008093EB000895833031F5613069F0613019
:10E8100028F0623079F06330F1F412C084E0809324
:10E82000AE1684E69DE011C08CE08093AE1682E0C7
:10E830009DE00BC08AE38093AE168EE09DE005C09C
:10E840008CE18093AE1688E49DE09093B01680939F
:10E85000AF1681E0089580E00895DF93CF9300D054
:10E8600000D0CDB7DEB78091F1008B838091F100AD
:10E870008C838B819C81892B31F484E38093AE1649
:10E8800088E69DE005C085E38093AE168CE99DE0A7
:10E890009093B0168093AF168091F1008983809198
:10E8A000F1008A838091E800877F8093E8002981C6
:10E8B0003A818091AE1690E08217930770F48F73BF
:10E8C0009070892B11F461E001C060E02091AF16D7
:10E8D0003091B0164091AE161CC02093AE16F5CF05
:10E8E0008091E80080FFFCCFF90190E00AC0542F2E
:10E8F0005150903449F09F5F84918093F10031969C
:10E90000452F9F01442399F78091E8008E7F8093E3
:10E91000E800442359F08091E80082FFE1CF209382
:10E92000AF163093B0164093AE1606C02093AF16C4
:10E930003093B0161092AE168091E80082FD0FC0A1
:10E94000613049F48091E80080FFFCCF8091E800BD
:10E950008E7F8093E8008091E80082FFFCCF809159
:10E96000E8008B7F8093E8008091E8008F778093A8
:10E97000E8000F900F900F900F90CF91DF910895C6
:10E980008091E800877F8093E8008091E8008E7F87
:10E990008093E8008091E80082FFFCCF8091E8003E
:10E9A0008B7F8093E8008091E8008F778093E80068
:10E9B0008091E8008E7F8093E8000895DF93CF93E5
:10E9C00000D0CDB7DEB78091F10089838091F1004E
:10E9D0008A838091E800877F8093E8006093C41069
:10E9E0008091E8008E7F8093E8008091E80080FFAE
:10E9F000FCCF0F900F90CF91DF910895DF93CF93CD
:10EA000000D000D0CDB7DEB78091F1008B8380912C
:10EA1000F1008C838091F10089838091F1008A83D9
:10EA20008091E800877F8093E80089819A81892B13
:10EA300049F08091C4108093F1008091E8008E7FAE
:10EA40008093E8008091E80082FFFCCF8091E8008D
:10EA50008B7F8093E8008091E8008F778093E800B7
:10EA60000F900F900F900F90CF91DF9108958091AC
:10EA7000E800877F8093E8008091E8008E7F809394
:10EA8000E8008091E80082FFFCCF8091F10085359D
:10EA900079F48091F1008A3A59F48091F10085353A
:10EAA00039F48091F1008A3A19F481E08093C3101F
:10EAB0008091E8008B7F8093E8008091E8008F7759
:10EAC0008093E8008091E8008E7F8093E800809139
:10EAD000E80080FFFCCF0895DF93CF9300D000D0F3
:10EAE000CDB7DEB78091F1008B838091F1008C83EC
:10EAF0008B819C81892B31F489E08093AE168BEB5E
:10EB00009CE005C089E08093AE168BEE9CE090936C
:10EB1000B0168093AF168091F10089838091F10047
:10EB20008A838091E800877F8093E80089819A81B9
:10EB30008A30910538F02091AF163091B01640918F
:10EB4000AE161CC08093AE16F6CF8091E80080FF11
:10EB5000FCCFF90190E00AC0542F5150903449F095
:10EB60009F5F84918093F1003196452F9F0144234C
:10EB700099F78091E8008E7F8093E800442359F054
:10EB80008091E80082FFE1CF2093AF163093B0165A
:10EB90004093AE1606C02093AF163093B016109275
:10EBA000AE168091E80082FFFCCF8091E8008B7F59
:10EBB0008093E8008091E8008F778093E8000F90C1
:10EBC0000F900F900F90CF91DF9108950F931F93A7
:10EBD00009EE10E081E0F801808381EC60E00E94A2
:10EBE000210882E0F801808381E864E30E94210823
:10EBF00083E0F801808380E864E30E94210884E0D8
:10EC0000F801808381EC60E00E94210885E0F80132
:10EC1000808380EC60E00E9421081F910F9108958D
:10EC2000DF93CF9300D0CDB7DEB72091F100909164
:10EC3000F100813869F4663009F083C0913221F027
:10EC4000923209F07EC002C047DF42C006DE40C0FB
:10EC5000813299F4693019F06A30C1F40AC09230F7
:10EC600021F0933009F06DC002C08ADE31C0FFDEB2
:10EC70002FC0822F692FA2DE2BC0813A29F4623087
:10EC800059F5822FBBDE24C0813221F56F3F09F098
:10EC900058C0222309F055C0992309F052C0809131
:10ECA000F10089838091F1008A8389819A8101979B
:10ECB00009F047C08091E800877F8093E800809149
:10ECC000E8008E7F8093E8008091E80080FFFCCF11
:10ECD00081E038C0813AA9F56E3F99F5222389F584
:10ECE000992379F58091F10089838091F1008A83DD
:10ECF00089819A81019729F58091E800877F809327
:10ED0000E8000E94434181508093F1008091E80027
:10ED10008E7F8093E8008091E80080FFFCCF809197
:10ED2000E80082FFFCCF8091E8008B7F8093E800B1
:10ED30008091E8008F778093E80081E080936219EA
:10ED400001C080E00F900F90CF91DF9108958091E6
:10ED5000D90081FF05C08091E20084608093E200C9
:10ED600008950F931F9310926719109268191092CB
:10ED7000691910926A19629903C081E0809367193A
:10ED80001D9905C0809167198260809367191E994B
:10ED900003C08DEF80936819649905C0809168194C
:10EDA0008D5F809368191F9903C08DEF8093691957
:10EDB000659905C0809169198D5F809369190091EB
:10EDC000631910916419065F1F4F0E94BF0808174E
:10EDD000190770F480916319909164190A969093C1
:10EDE00064198093631980916A198D5F80936A1901
:10EDF00000916319109164190A5010400E94BF08D5
:10EE00008017910770F480916319909164190A97A3
:10EE1000909364198093631980916A198350809349
:10EE20006A1980916719882389F480916819882369
:10EE300069F480916919882349F490E080916A19F6
:10EE4000882309F491E081E0982701C091E0892F9F
:10EE50001F910F9108958091AD16882309F44AC03F
:10EE600080916619882331F47CDF882319F081E0D2
:10EE70008093661990916619992321F48091651900
:10EE80008823C1F121E02093E9008091E80085FF0B
:10EE900031C0992359F0109266191092651980912A
:10EEA0006719882369F0209365190AC010926719C1
:10EEB000109268191092691910926A1910926519C6
:10EEC000809167198093F100809168198093F10017
:10EED000809169198093F10080916A198093F10003
:10EEE0008091E8008E7F8093E8008091E8008F7722
:10EEF0008093E80008951F938091C6109091C710E9
:10EF000001969093C7108093C6108091C5108F5FB3
:10EF10008093C5108091C510823039F41091E900BA
:10EF20009ADF1092C5101093E9001F910895E2EE48
:10EF3000F0E080818460808384B18F7184B985B171
:10EF4000806E85B98DB18F7C8DB98EB180638EB99D
:10EF50008AB1806F8AB96A98729A0E94A3070E9448
:10EF6000BF0890936419809363191092661981E029
:10EF70008093651908958AB1806F8AB984B18F71C1
:10EF800084B985B1806E85B98DB18F7C8DB98EB114
:10EF900080638EB9089584E08093E9008091E80051
:10EFA00085FF36C01F9B0CC0659B0AC0649B08C0D0
:10EFB00093B192959695969593709095917001C0A6
:10EFC00091E08091C810981719F19093C810909310
:10EFD000F1008AB58093F1008AB58093F1008AB57B
:10EFE0008093F1008AB58093F1008AB58093F10097
:10EFF0008AB58093F1008AB58093F1008091E80092
:10F000008E7F8093E8008091E8008F778093E800FE
:10F010000895DF93CF9300D000D0CDB7DEB785E061
:10F020008093E9008091E80082FF33C09091F10065
:10F030009F708091F1008F70823081F0833018F4DE
:10F040008130E9F405C0833079F08430C1F412C016
:10F05000992311F05C9A13C05C9811C0992311F0A8
:10F060005D9A0DC05D980BC0992311F05E9A07C0A0
:10F070005E9805C0992311F05F9A01C05F98809156
:10F08000E8008B7F8093E8008091E8008F77809381
:10F09000E8008091C310882319F18BB18F708BB970
:10F0A0008091E00081608093E00019821A821B82C7
:10F0B0001C820BC089819A81AB81BC810196A11D04
:10F0C000B11D89839A83AB83BC8389819A81AB818B
:10F0D000BC8180579141A140B04060F30E94070875
:10F0E0000F900F900F900F90CF91DF910895809126
:10F0F000AD16882311F08DDF4ECF089584B18F7146
:10F1000084B985B1806E85B98DB18F7C8DB98EB192
:10F1100080638EB98AB1806F8AB91092C910089540
:10F12000EF92FF920F931F93DF93CF9300D000D005
:10F13000CDB7DEB79A8389837C836B837A0183E0C2
:10F140008093F1171092F2178A818093F3178981C7
:10F150008093F4178C818093F5178B818093F61739
:10F1600081E28093551981E08093561910925819C5
:10F170001092571910925A191092591986E090E07E
:10F1800090935C1980935B1910925D1981EF97E160
:10F190000E94C4600B811C810F5F1F4F89819A817F
:10F1A000081B190B81EA8093551982E08093561948
:10F1B000109258191092571910925A191092591901
:10F1C00010935C1900935B1910925D1981EF97E120
:10F1D0000E94C460E1EFF7E198012E0F3F1F04C0C9
:10F1E0008191D7018D937D01E217F307C9F70F9045
:10F1F0000F900F900F90CF91DF911F910F91FF9083
:10F20000EF900895DF93CF9300D000D0CDB7DEB755
:10F210009A8389837C836B83DA0181E08093F11781
:10F220001092F2178A818093F31789818093F417E3
:10F230008C818093F5178B818093F617E7EFF7E1C8
:10F24000119288E1E131F807D9F749815A81342FC9
:10F250003F71632F70E0CB0120E207C0E22FF0E0A6
:10F26000EF50F84E10822F5F01970097B9F7932F58
:10F27000905E2B813C81241B350BA9014F5F5F4FB2
:10F2800009C0E92FF0E0EF50F84E8D918083415096
:10F2900050409F5F41155105A1F781E280935519B8
:10F2A00081E08093561910925819109257191092B4
:10F2B0005A19109259192F5D3F4F260F371F30935F
:10F2C0005C1920935B1910925D1981EF97E10E9400
:10F2D000C4600F900F900F900F90CF91DF91089521
:10F2E0000F931F93909100138091FE122091FF12B3
:10F2F000309100136091FD127091FE12981721F465
:10F30000C9014CED50E118C0062F10E0615070406B
:10F31000601B710BC9014CED50E174DF6091FD126F
:10F320007091FE124091CA1050E0401B510B4552A3
:10F330005F4ECB01801B910B65DF6091FD127091D8
:10F34000FE128091FF12909100134CEE51E1E8DE25
:10F350004091CA103091FC1220E010C0E22FF0E082
:10F36000DF01A451BE4EE452FF4E90818C9198175C
:10F3700021F08BB1806F8BB930E02F5F241770F3D1
:10F380003093FC124C9A1092CB101092CA101F911D
:10F390000F9108952F923F924F925F926F927F92BA
:10F3A0008F929F92AF92BF92CF92DF92EF92FF9295
:10F3B0000F931F93CF93DF9381E08093FC1289E03A
:10F3C0000E94424054E0252E312C13C10E942B3F55
:10F3D00009C00E942B3F182F0E94773D882309F017
:10F3E0000DC1812F8A33A9F726C1182F105302C0EF
:10F3F000182F17550E942B3F80628A3310F48053D8
:10F4000001C08755E12EE29440EFE422E80E0E940D
:10F410002B3F80628A3318F430ED432E02C029EA74
:10F42000422E480E0E942B3F80628A3318F490EDE2
:10F43000592E02C009EA502E580E0E942B3F8062BE
:10F440008A3318F410ED612E02C0B9EA6B2E680EF3
:10F450000E942B3F80628A3318F4A0ED7A2E02C0FE
:10F46000F9EA7F2E780E0E942B3F80628A3318F4CF
:10F47000E0ED8E2E02C079EA872E880E0E942B3F87
:10F4800080628A3318F460ED962E02C059EA952EF8
:10F49000980E4CECC42E40E1D42EE6010E2D10E067
:10F4A0005601A00EB11E17C00E942B3F80628A3306
:10F4B00010F4805301C08755F82EF29430EFF322F8
:10F4C000F8820E942B3F80628A3310F4805301C07F
:10F4D00087558F0D8993CA15DB0531F7882D8295E5
:10F4E000807F890D21F0843009F083C059C0C42D7C
:10F4F000D0E024E0CC0FDD1F2A95E1F7C50DD11D2A
:10F5000094E0CC0FDD1F9A95E1F7C60DD11D84E084
:10F51000CC0FDD1F8A95E1F7C70DD11D8091FD123B
:10F520009091FE120196C817D90729F08091CB104F
:10F53000882309F0D5DE2091CB1090E00AC0E92F96
:10F54000E20FF0E0E452FF4ED6018D916D01808311
:10F550009F5F9E15A0F32E0D2093CB108091CA10B3
:10F560008E0D8093CA10E81658F48091FD12909188
:10F57000FE12800F911F9093FE128093FD120CC01B
:10F58000015010400C0F1D1F1093FE120093FD122E
:10F59000D0930013C093FF12203A58F1A1DE29C086
:10F5A0008091CB10882309F09BDEB6E0B093F11771
:10F5B00083E08093F2171092F3178091CD1080931F
:10F5C000F417A1E2A0935519B1E0B0935619109227
:10F5D00058191092571910925A19109259193092BD
:10F5E0005C1920925B1910925D1981EF97E10E94DE
:10F5F000C4600E94773D882309F4E8CE8091CB1047
:10F60000882309F06DDE0E941A3E5C988091FC12FE
:10F61000DF91CF911F910F91FF90EF90DF90CF90EE
:10F62000BF90AF909F908F907F906F905F904F9022
:10F630003F902F9008950E942B3F80628A3308F4F8
:10F64000D4CED6CE8091F017863009F061C080917B
:10F65000B9108823F9F08091B51090E02AE430E0E9
:10F66000829FF001839FF00D929FF00D1124EF54C3
:10F67000F94E808591858B5E934051F48681978108
:10F680008B5F9F4229F481E08093C9105E9A02C08B
:10F690001092C9108091C9108823D1F11F9B02C01C
:10F6A0001E9936C00E94593D80E00E94BD3A0E94DA
:10F6B0008A3A882369F181ED9DE060E040E00E9494
:10F6C000C217882329F15C9A84E08093F117109285
:10F6D000F2178FEF8093F31781E28093551981E041
:10F6E00080935619109258191092571910925A195E
:10F6F0001092591983E090E090935C1980935B1904
:10F7000010925D1981EF97E10E94C4605C9842DE1F
:10F710008091F0178A50823020F08091B6108823B3
:10F7200019F01092C9105E98089510926C191092F9
:10F730006B190895EF92FF920F931F93DF93CF936E
:10F74000CDB7DEB728970FB6F894DEBF0FBECDBF9A
:10F750008091F017863009F0D0C08091B9108823CD
:10F7600009F489C010926B1910926C198091B51030
:10F77000482F50E08AE490E09C01429FC001439FE3
:10F78000900D529F900D1124FC01EF54F94E6581AC
:10F79000FC01E154F94E20E030E06AC080819181A3
:10F7A000039709F062C082819381892B09F05DC0C3
:10F7B00084819581892B09F058C081E080936B1971
:10F7C00085E190E0289F8001299F100D389F100D42
:10F7D00011248AE4E82EF12C4E9DF0014F9DF00D8E
:10F7E0005E9DF00D1124E00FF11FEF54F94E858955
:10F7F00087FF14C00E947760809301138091B51039
:10F8000090E08E9DF0018F9DF00D9E9DF00D1124D6
:10F81000E00FF11FEF54F94E818D14C0818D0E94CD
:10F820007760809301138091B51090E08E9DF00178
:10F830008F9DF00D9E9DF00D1124E00FF11FEF54F0
:10F84000F94E85890E94776080930213809101139D
:10F850008093A7008091A90080628093A900809185
:10F86000A9008F7B8093A90006C02F5F3F4F75963C
:10F87000261708F493CF80916B198823F1F18091BA
:10F8800001138093A7008091A60080FF10C0809193
:10F89000A60081FD02C08091F1008091A6008E7FBC
:10F8A0008093A6008091A6008F778093A600809118
:10F8B0006C19813011F595E599838AEA8A839B83D7
:10F8C0008C8381E28093551989E08093561980E0FA
:10F8D00093E0909358198093571910925A191092E7
:10F8E000591984E090E090935C1980935B19109211
:10F8F0005D19CE0101960E94C4608091F0178A5074
:10F90000823020F08091B610882339F08BB18F704F
:10F910008BB910926B1910926C1928960FB6F89447
:10F92000DEBF0FBECDBFCF91DF911F910F91FF9032
:10F93000EF9008958AB1806F8AB90895CF93DF93CD
:10F940008091F017863009F0ECC08091B9108823BF
:10F9500009F48BC0109203138091B51090E02AE453
:10F9600030E0AC01429FC001439F900D529F900D2B
:10F970001124FC01EF54F94E2581FC01E154F94EAC
:10F98000C0E0D0E06FC080819181039709F068C02A
:10F9900084819581029709F063C081E0809303130D
:10F9A00081E2809355198AE0809356191092581974
:10F9B0001092571910925A191092591910925C19F5
:10F9C00010925B1910925D1981EF97E10E94C4605B
:10F9D00081E88093551986E08093561980E092E281
:10F9E000909358198093571910925A1910925919D7
:10F9F0008AEF90E090935C1980935B1910925D19E7
:10FA000081EF97E10E94C4602091B51030E085E15C
:10FA100090E0C89FF001C99FF00DD89FF00D112410
:10FA20008AE490E0EC012C9FC0012D9F900D3C9F3B
:10FA3000900D1124E80FF91FEF54F94E85890E94AB
:10FA4000776080936D198093A7008091A9008062F0
:10FA50008093A9008091A9008F7B8093A90005C0A5
:10FA600021967596C21708F48ECF809103138823D0
:10FA700009F457C080916D198093A7008091A6006A
:10FA800080FF42C08091A60081FD34C0A091AF00EC
:10FA90002091AF004091AF006091AF008DB79EB74D
:10FAA0000A970FB6F8949EBF0FBE8DBFEDB7FEB795
:10FAB00031968FE897E0CDB7DEB79A838983A2832A
:10FAC0001382332727FD309535832483552747FD3F
:10FAD000509557834683772767FD709571876087B8
:10FAE0008FD14DB75EB7465F5F4F0FB6F8945EBFDC
:10FAF0000FBE4DBF8091A6008E7F8093A60080919F
:10FB0000A6008F778093A6008091A60086FF09C08B
:10FB10008091A6008F7B8093A6005C985D985E988C
:10FB20005F988091F0178A50823020F08091B61053
:10FB3000882329F08BB18F708BB910920313DF915A
:10FB4000CF91089580916E198F5F80936E19809187
:10FB50006E19882321F48091041381114F9A08951E
:10FB60008091F017863071F58091B910882321F0CB
:10FB70000E94C51581115D9A0E94CD0E882311F156
:10FB800064990FC05C9A81E0809304138EED9DE030
:10FB900065EF7DE041E00E94D017109204135F985A
:10FBA0005C981E990FC05C9A81E0809304138DEEDF
:10FBB0009DE066EE7DE041E00E94D01710920413B4
:10FBC0005C985F988091F0178A50823020F0809185
:10FBD000B610882319F00E94A10E5D9808958AB18D
:10FBE000806F8AB984B18F7184B985B1806E85B90F
:10FBF0008DB18F7C8DB98EB180638EB90C94970EC8
:10FC00000E94EC070E94290780E090E020E80FB6F0
:10FC1000F89420936100809361000FBE0E947807E2
:10FC200080E090E00895629FD001739FF001829F71
:10FC3000E00DF11D649FE00DF11D929FF00D839F7B
:10FC4000F00D749FF00D659FF00D9927729FB00D18
:10FC5000E11DF91F639FB00DE11DF91FBD01CF012B
:10FC600011240895991B79E004C0991F961708F094
:10FC7000961B881F7A95C9F780950895AA1BBB1B10
:10FC800051E107C0AA1FBB1FA617B70710F0A61B9C
:10FC9000B70B881F991F5A95A9F780959095BC01BD
:10FCA000CD010895A1E21A2EAA1BBB1BFD010DC0B8
:10FCB000AA1FBB1FEE1FFF1FA217B307E407F5071C
:10FCC00020F0A21BB30BE40BF50B661F771F881FF8
:10FCD000991F1A9469F760957095809590959B018E
:10FCE000AC01BD01CF0108959111089581568A514B
:10FCF00008F4805285580895FB01DC0104C08D9101
:10FD00000190801921F441505040C8F7881B990B8D
:10FD100008950F931F93CF93DF938C01EB0100970E
:10FD200031F46115710519F420E030E037C081E04D
:10FD300090E06EE070E0A3D2FC019C01009771F1AD
:10FD400080E88383209771F0D387C28781E883831B
:10FD500080918D1990918E19892B21F4F0938E1931
:10FD6000E0938D1901151105C9F011870087838172
:10FD70008260838380918F1990919019892B71F4FF
:10FD8000F0939019E0938F198091911990919219A5
:10FD9000892B21F4F0939219E0939119C901DF9115
:10FDA000CF911F910F9108950F931F93CF93DF93DE
:10FDB0008C01EB018B8181FF1BC082FF0DC02E8166
:10FDC0003F818C819D812817390764F4E881F9818E
:10FDD0000193F983E88306C0E885F985802F0995AA
:10FDE000892B31F48E819F8101969F838E8302C07F
:10FDF0000FEF1FEFC801DF91CF911F910F91089571
:10FE0000DF93CF93CDB7DEB7FE0135966191719147
:10FE100080918F1990919019AF0138D0CF91DF91D7
:10FE200008950F931F93CF93DF938C01E0918F1967
:10FE3000F0919019838181FF21C0C0E0D0E00DC016
:10FE4000E0918F19F091901920853185BF01F9015A
:10FE50000995892B11F0CFEFDFEFF80181918F0128
:10FE6000882371F7E0918F19F091901920853185E1
:10FE70008AE0BF01F9010995892B11F0CFEFDFEF7F
:10FE8000CE01DF91CF911F910F9108952F923F9254
:10FE90004F925F926F927F928F929F92AF92BF929A
:10FEA000CF92DF92EF92FF920F931F93DF93CF9346
:10FEB000CDB7DEB72B970FB6F894DEBF0FBECDBF20
:10FEC0003C012B015A01FC0117821682838181FDBE
:10FED00003C06FEF7FEFB9C19AE0892E1E0108942D
:10FEE000211C311CF3012381F20123FD859123FFA5
:10FEF00081912F01882309F4A5C1853239F423FDAE
:10FF0000859123FF81912F01853221F490E0B30187
:10FF10004BDFE8CF982FFF24EE249924FFE1FF1553
:10FF2000D0F09B3269F09C3228F4903259F0933231
:10FF300091F40EC09D3249F0903369F441E024C041
:10FF400052E0F52A84E0F82A28C098E0F92A25C072
:10FF5000E0E1FE2A22C0F7FC29C0892F80538A30B5
:10FF600070F4F6FE05C0989C902C1124980E15C0D4
:10FF7000E89CE02C1124E80EF0E2FF2A0EC09E322D
:10FF800029F4F6FC5FC140E4F42A07C09C3619F45A
:10FF900050E8F52A02C0983649F4F20123FD959104
:10FFA00023FF91912F01992309F0B8CF892F855410
:10FFB000833018F08052833038F444E050E0A40ECF
:10FFC000B51E5FE359830FC0933631F0933779F054
:10FFD000933509F052C01FC0F5018081898342E04A
:10FFE00050E0A40EB51E610101E010E011C0F50162
:10FFF000C080D180F6FC03C06FEF7FEF02C0692D97
:020000021000EC
:1000000070E042E050E0A40EB51EC60169D28C013A
:100010005FE7F52213C0F501C080D180F6FC03C074
:100020006FEF7FEF02C0692D70E042E050E0A40E58
:10003000B51EC60143D28C0150E8F52AF3FE06C076
:1000400018C080E290E0B301AFDEEA948E2D90E01C
:1000500008171907B0F30DC0F601F7FC8591F7FEFC
:1000600081916F0190E0B3019FDEE110EA940150AD
:1000700010400115110581F7E2C0943611F0993650
:1000800061F5F7FE08C0F50120813181428153817D
:1000900084E090E00AC0F501808191819C014427B1
:1000A00037FD4095542F82E090E0A80EB91E9FE6E0
:1000B000F92257FF09C050954095309521953F4F43
:1000C0004F4F5F4FE0E8FE2ACA01B901A1012AE0C3
:1000D00030E011D2D82ED2183FC0953729F41F2D09
:1000E0001F7E2AE030E01DC01F2D197F9F3661F072
:1000F000903720F4983509F0A5C00FC0903739F03B
:10010000983709F09FC004C028E030E00AC01061B1
:1001100014FD146020E130E004C014FD166020E1FD
:1001200032E017FF08C0F5016081718182819381FF
:1001300044E050E008C0F50180819181BC0180E07D
:1001400090E042E050E0A40EB51EA101D4D1D82E1B
:10015000D2188FE7F82EF122F6FE0BC05EEFF522E3
:10016000D91438F4F4FE07C0F2FC05C08FEEF82273
:1001700002C01D2D01C0192DF4FE0DC0FE01ED0DB4
:10018000F11D8081803319F499EEF92208C01F5FB8
:10019000F2FE05C003C08F2D867809F01F5F0F2D7A
:1001A000F3FC13C0F0FE0EC01E1510F09D2C0AC00B
:1001B0009D2C9E0C911A1E2D05C080E290E0B3018B
:1001C000F3DD1F5F1E15C8F304C01E1510F4E11AFD
:1001D00001C0EE2404FF0EC080E390E0B301E4DD33
:1001E00002FF1BC001FD03C088E790E00EC088E558
:1001F00090E00BC0802F867881F001FF02C08BE277
:1002000001C080E2F7FC8DE290E0B301CDDD05C0D6
:1002100080E390E0B301C8DD9A94D914C8F3DA946E
:10022000F101ED0DF11D808190E0B301BDDDDD2018
:10023000B1F705C080E290E0B301B6DDEA94EE20AC
:10024000C9F750CEF30166817781CB012B960FB6AB
:10025000F894DEBF0FBECDBFCF91DF911F910F91FC
:10026000FF90EF90DF90CF90BF90AF909F908F90D6
:100270007F906F905F904F903F902F9008950F93D5
:100280001F93CF93DF93689F8001699F100D789F24
:10029000100D1124C8010DD0EC01009721F060E091
:1002A00070E0A80116D1CE01DF91CF911F910F917F
:1002B0000895CF93DF93BC018230910510F462E082
:1002C00070E0A0919519B0919619ED01E0E0F0E091
:1002D00040E050E021C0888199818617970769F432
:1002E0008A819B81309719F09383828304C0909315
:1002F000961980939519FE0134C06817790738F470
:100300004115510519F08417950708F4AC01FE0159
:100310008A819B819C01E9012097E9F641155105ED
:10032000A9F1CA01861B970B049708F4BA01E0E013
:10033000F0E02AC08D919C91119784179507F9F4EC
:100340006417750781F412968D919C9113973097DD
:1003500019F09383828304C0909396198093951922
:10036000FD0132964FC0CA01861B970BFD01E80FB5
:10037000F91F6193719302978D939C9343C0FD0184
:10038000828193819C01D9011097A1F680919319E4
:1003900090919419892B41F48091A3079091A4071F
:1003A00090939419809393194091A5075091A607B3
:1003B0004115510541F44DB75EB78091A107909169
:1003C000A207481B590B20919319309194192417B7
:1003D0003507B0F4CA01821B930B8617970780F08C
:1003E000AB014E5F5F4F8417950750F0420F531FCC
:1003F0005093941940939319F9016193719302C03A
:10040000E0E0F0E0CF01DF91CF910895CF93DF934B
:10041000009709F450C0EC0122971B821A82A09128
:100420009519B0919619109709F140E050E0AC177A
:10043000BD0708F1BB83AA83FE0121913191E20F30
:10044000F31FAE17BF0779F48D919C911197280F78
:10045000391F2E5F3F4F3983288312968D919C91CF
:1004600013979B838A834115510571F4D093961994
:10047000C093951920C012968D919C911397AD0150
:10048000009711F0DC01D3CFFA01D383C28321910D
:100490003191E20FF31FCE17DF0769F4888199814C
:1004A000280F391F2E5F3F4FFA01318320838A8145
:1004B0009B8193838283DF91CF910895FC01059006
:1004C000615070400110D8F7809590958E0F9F1F56
:1004D0000895DC0101C06D9341505040E0F708954C
:1004E000FC016150704001900110D8F78095909503
:1004F0008E0F9F1F0895FA01AA27283051F120314D
:1005000081F1E8946F936E7F6E5F7F4F8F4F9F4FA7
:10051000AF4FB1E03ED0B4E03CD0670F781F891FE9
:100520009A1FA11D680F791F8A1F911DA11D6A0FB7
:10053000711D811D911DA11D20D009F468943F916A
:100540002AE0269F11243019305D3193DEF6CF0169
:100550000895462F4770405D4193B3E00FD0C9F72F
:10056000F6CF462F4F70405D4A3318F0495D31FD9C
:100570004052419302D0A9F7EACFB4E0A6959795EF
:10058000879577956795BA95C9F7009761057105C5
:1005900008959B01AC010A2E06945795479537950F
:1005A0002795BA95C9F7620F731F841F951FA01D69
:0605B0000895F894FFCF4E
:1005B60000F00A0D0053656C65637420736F7572E5
:1005C6006365206469726563746F72790A0D0053FE
:1005D600656C6563742064657374696E6174696FB4
:1005E6006E206469726563746F72790A0D00476FD5
:1005F60020746F20706172656E740A0D0044697212
:1006060020666F756E64202D2063726561746520A7
:100616006469723A200046696C6520666F756E647F
:10062600202D20636F70792066696C653A2000463C
:10063600696C6520657869737473207468656E20CB
:1006460064656C657465732074686973206F6E6584
:100656002E0A0D00212121636F7079206661696C75
:100666000A0D00456E64206F6620636F70790A0D6F
:1006760000001000000100200000020040000004FD
:10068600A87F000008D020000000A87F000002001C
:10069600000400040000080008000010001000001C
:1006A6002000200000400040FFFFFFFF002804015B
:1006B6000000002008000100000001080000000200
:1006C600100000000420FFFFFFFF40EB00904D5399
:1006D60057494E342E31000200000002000000008F
:1006E600F800003F00000001810029000000004ED4
:1006F6004F204E414D4520202020464154202020A9
:1007060020205252614172724161F8FFFFF8FFFFEB
:10071600FFF8FFFF0FFFFFFF0FFFFFFF0F3A2A3F14
:10072600223C3E7C2B2C2E3B3D5B5DFF4E6F2064B6
:1007360061746120617661696C61626C65207769BC
:1007460074682074686973204849442067656E653B
:1007560072696320636F6E66696775726174696F2B
:100766006E2E0A0D000A0D446576696365202569BB
:1007760020403A3078253032580A0D005649443A1E
:10078600253034582C205049443A253034582C20F2
:10079600004D6178506F7765722069732025696D09
:1007A600412C2000436F6E74726F6C20456E64702E
:1007B6006F696E7420697320256920627974657388
:1007C6002C2000537570706F7274656420696E74A6
:1007D6006572666163652873293A253032690A0DA8
:1007E60000496E74657266616365206E623A2530F3
:1007F60032692C20416C7453206E623A253032697E
:100806002C20436C6173733A253032692C20537562
:1008160062436C6173733A253032692C2050726FD3
:10082600746F636F6C3A253032690A0D0020456E8D
:1008360064706F696E7428732920416464723A008B
:100846002025303258004E6F6E650020506879734F
:100856006963616C20706970652873293A00257593
:100866002066696C652873292064656C6574656407
:100876000A0D005472616E73666572742065727239
:100886006F720D005472616E7366657274207261C8
:100896007465202D2057524954452025346C754BDC
:1008A600422F730D0A005472616E7366657274206E
:1008B60072617465202D20524541442025346C75A3
:1008C6004B422F730D0A005472616E736665727423
:1008D60020746F6F20736C6F770D005472616E73A6
:1008E6006665727420726174652025346C754B429E
:1008F6002F73202D2073747265616D2073697A657C
:10090600202534694B420D0A00746D702E62696EA3
:1009160000416C6C6F6320612066696C65206F6EA8
:10092600206561636820646576696365730A0D00F6
:100936002121214572726F7220616C6C6F63617444
:10094600696F6E206F6E2064657669636520310A73
:100956000D002121214572726F7220616C6C6F63EC
:100966006174696F6E206F6E2064657669636520B9
:10097600320A0D005472616E73666572742064618A
:1009860074612066726F6D206465766963652031D7
:1009960020746F2064657669636520320D00547299
:1009A600616E736665727420646174612066726F2D
:1009B6006D20646576696365203220746F206465F6
:1009C6007669636520310D005472616E73666572D7
:1009D60074206C6172676520627566666572206F49
:1009E6006E205553420D00456E64206F6620746577
:1009F60073740A0D0053796E6368726F6E697A6557
:100A060020666F6C646572733A0A0D0053656C65F7
:100A1600637420736F7572636520646972656374AD
:100A26006F72790A0D0053656C6563742064657393
:100A360074696E6174696F6E206469726563746F40
:100A460072790A0D00476F20746F20706172656EAF
:100A5600740A0D0044697220666F756E64202D203D
:100A6600637265617465206469723A20000A0D003C
:100A760046696C6520666F756E64202D20636F7005
:100A8600792066696C653A200046696C6520657850
:100A960069737473207468656E2064656C6574652B
:100AA600732074686973206F6E652E0A0D0021210C
:100AB60021436F7079206661696C0A0D00456E648A
:100AC600206F6620636F70790A0D000A0D2D2D20A8
:100AD600737061636520666F72206D6F72652D2D70
:100AE600000D202020202020202020202020202033
:100AF6002020200D0025633A20766F6C756D6520E9
:100B0600697320000A0D44726976652075736573F2
:100B1600200046415431320A0D0046415431360A0E
:100B26000D0046415433320A0D00616E20756E6B1E
:100B36006E6F776E20706172746974696F6E20745F
:100B46007970650D00524F4F542064697265637465
:100B56006F72790A0D00446972206E616D652069B5
:100B6600732025730A0D002020202020202020201D
:100B76002053697A6520204E616D650A0D0044692F
:100B860072200020202020002531306C7520202581
:100B9600730A0D00202534692046696C65730D0AB9
:100BA6000020253469204469720D0A003A207370CA
:100BB6006163653A20256C754D42200A0D004D652E
:100BC6006D6F727920696E74657266616365206106
:100BD6007661696C61626C653A0D004672656520E6
:100BE60073706163653A20256C75204B4279746594
:100BF60073202F20256C75204B42797465730A0D7E
:100C060000467265652073706163653A202575201C
:100C160025250A0D00EB0302001C201420230103E6
:100C260000002000215812000000090000080250B0
:100C360008055008065003000203010203000025C0
:100C4600642C2025642C2025642C202564200D0A84
:080C56000020009B19000000C2
:00000001FF
